:020000040800F2
:10000000005000208D010008890100080000000058
:10001000890100088901000889010008000000002A
:10002000000000000000000000000000890100083E
:10003000890100080000000089010008890100080A
:100040008901000889010008890100088901000868
:100050008901000889010008890100088901000858
:100060008901000889010008890100088901000848
:100070008901000889010008890100088901000838
:100080008901000889010008890100088901000828
:100090008901000889010008890100088901000818
:1000A0008901000889010008890100088901000808
:1000B00089010008890100088901000889010008F8
:1000C00089010008890100088901000889010008E8
:1000D00089010008890100088901000889010008D8
:1000E00089010008890100088901000889010008C8
:1000F00089010008890100088901000889010008B8
:1001000089010008890100088901000889010008A7
:100110008901000889010008890100088901000897
:100120008901000889010008890100088901000887
:100130008901000889010008890100088901000877
:100140008901000889010008890100088916000852
:100150008901000889010008890100088901000857
:100160008901000889010008890100088901000847
:100170008901000889010008890100088901000837
:100180008901000889010008FEE70000684620F0A8
:1001900007018D4601B500230A4A0B499818884289
:1001A00004D20A49585898500433F5E7084B094AD5
:1001B000934203D2002043F8040BF8E700F00CF858
:1001C000FEE700BF000000203800002000390008D2
:1001D00038000020481C00202DE9F743002000F0E3
:1001E00061FF002001F008F9012001F09DF8684648
:1001F00001F075FE002401238DF805408DF80430D0
:100200008DF80640B5490A196058958802AE0583F5
:100210006946083446F8085D01F014FE182CF1D147
:100220000027AF4CE31938599A8802A9028341F894
:10023000082D0837694601F005FE302FF1D1002660
:10024000A84DAF197059BC8802AB44836946083683
:1002500043F8084D01F0F6FD182EF1D1A24D082605
:10026000284669460096802401F0ECFD2E839F4DC0
:10027000DFF87C8208264FF020094FF40057A8F8D9
:100280001A9001206F836E8301F0D8F8A8F81890B7
:1002900001202F832E8301F0D1F8013CE7D12046C5
:1002A0008F4A131881589D88083030284D83F7D124
:1002B000012001F0C3F80027894EF019BC5982884B
:1002C0000837302F2283F7D1012001F0B7F800253D
:1002D00001218DF804508DF80710804B5F1902AC96
:1002E000BE88E85844F8086D6946083501F0AAFD53
:1002F000182DF2D100257A48421902A9938828586E
:1003000041F8083D0835694601F09CFD302DF2D1D9
:100310000027744EF41902A8A588694640F8085DC4
:10032000B859083701F08EFD182FF2D1704F6420B4
:1003300001F022F83A6902F0010501F0B4F9C6B201
:1003400016B93B69D9070BD53DB18020012101F0D9
:1003500023FE8020002101F01FFE002001F0AAF9F9
:10036000002000F02FFB002000F024F9B6B960490E
:100370000C69E20770D45F480778422F6CD15E4A5F
:100380001678002E68D001F0D1FC0120002100F089
:10039000DFFF5A4BDF78082F46D103E0102000F032
:1003A000DDFA59E06FF00700012101F0E9FD6FF07F
:1003B0008000012101F0F0FD4FF0FF30012101F03C
:1003C000F7FD4FF0FF30012101F0FEFD4FF0FF304F
:1003D000002101F0D5FD4FF0FF30002101F0DCFDE0
:1003E0004FF0FF30002101F0E3FD4FF0FF3000211E
:1003F00001F0EAFD45B18020012101F0CDFD802012
:10040000002101F0C9FD08E001F04DF928B13C4898
:10041000D0F8E4550DB102F0C5FA3A4E346884F3D1
:10042000088836490A68904700F0CEFF012001464F
:1004300000F08EFF00F0D2FF40F2F31398421F4607
:10044000F8D900F0C1FF0120002100F081FF00F089
:10045000C5FFB842FBD9E7E700F0B6FF00F0BEFFEA
:100460003227B0FBF7F364210446B3FBF1F001FB44
:10047000103242F21073B4FBF3F1560841F28830A7
:1004800003FB11428242B4FBF7F307FB134188BF21
:10049000C6EB07060120B14294BF002101210A27C3
:1004A00000F056FFB4FBF7F607FB16440CB900F05A
:1004B000A9FD002000F03AFD00F090FF44F61F6116
:1004C0008842CBD900F080F80028C7D1002D3FF436
:1004D0005AAF074A1069C307C0D454E73036000842
:1004E0004836000818360008001002400004024098
:1004F00000000240D23F0008D33F0008044000083B
:10050000EC15002000400008124B1A78032A10B5A1
:100510000BD811490C6800F07F004FEAC41444EA7C
:10052000001008600FD104220EE0072A0FD80B49F3
:100530000C6800F07F004FEAC41444EA0010086021
:1005400001D1082200E001321A70002010BD4FF0E6
:10055000FF3010BDFC0400203800002044000020C3
:1005600070B5134B88B016461A7804460D468DF8C0
:1005700000209978DA7858781B798DF802108DF878
:1005800003208DF801008DF8043000F083FD8DF814
:100590000500F7208DF808006946204609228DF8ED
:1005A00006508DF8076000F087FA08B070BD00BFF4
:1005B0007837000810B9034B187070474FF0FF30C0
:1005C000704700BFFD040020014B1878704700BF42
:1005D000FD0400202DE9F04198460C4615460646DC
:1005E00000F04CFD00F0F0FEB8F1010F04D0B8F1BE
:1005F000020F40F0A38189E0B14B14B1012C0AD164
:1006000004E01C70AF4BB04A1C6092E019780729D7
:1006100000F2918197E01978082903D030460E2125
:100620000122E5E0A948AA4C02784378817822703B
:10063000C2780079A34FA44D6370A170E27020715D
:100640003F682D6800F026FD4FEA556E6071780E08
:100650000223E071C7F386417044A3712172C7F38E
:10066000C62341186372C7F3061253FA81F3C5F328
:100670008640A27252FA83F250FA82F1C5F3C62381
:1006800053FA81F22073C5F3061050FA82F16373B6
:100690000023A07384F80BE0C9B21A460F34184641
:1006A000A84221D010F807E04FF0080C01335200A7
:1006B000DBB242EADE12062B4FEA4E0ED2B25FFAEE
:1006C0008EFE0AD9C3F1070302FA03F2D2B251181F
:1006D000002304F8012BC9B21A460CF1FF3C1CF0B0
:1006E000FF0CE3D10130DBE71BB18B1804F8012BC1
:1006F000D9B24A42764902F07F00F723A21C20704B
:1007000063703046521A00F0D7F914E114B1012C8D
:1007100053D110E06A4B6B496B486E4A1C700C60F9
:1007200004606D4B6D496E4814706E4A1C700C600D
:1007300004601460FFE062480178072907D8654922
:1007400008782A180A702846FFF7DEFEF3E0082929
:100750002BD160480278AB18037060480368B3F58A
:10076000806F80F0E880584E5E4F5D4C3668386888
:10077000226807240132C5F380176D00072A47EA73
:100780004000EDB206D9524AD0540133B34228BFDB
:1007900009210022013CEDD1524C206050480260FA
:1007A0004E4A1360464B1970C5E0092902D14A4BE5
:1007B0001D70C0E00C220270BDE0434B47481F682B
:1007C0000168B942FFF42AAF3D4A13780C2B03D1DC
:1007D00030460E2142460BE03E4A3F4813780178EE
:1007E000584200F07F02914205D030460E2103228C
:1007F000FFF7B6FE9FE0334B3B4901240C701C68A9
:1008000044EA0700830740F08C80384A944202D8BB
:100810006FF0070087E000F0D9FC00F100614B1E8B
:100820009C426DD801F074FA00230C2159433048E2
:100830000A58944224D12F492F488C4201D10022DA
:1008400002600121006801FA03F1014203D02B4D3F
:100850004FF000082EE041EA000227490A60244ACE
:100860000C2000FB03230221586801F0B5FA082888
:10087000EDD04FF0FF3001F061FA6FF0030052E06D
:1008800001330C2BD1D1E2E76B7829781A0442EAC4
:10089000012315F8011CAA780B4343EA026101F019
:1008A0007DFA04350828E4D101F02AFA01F020FA93
:1008B00008F10408B84508EB0400E5D342E000BFA6
:1008C000FC04002038000020440000207837000895
:1008D0004C0000204000002048000020F8040020C8
:1008E000F404002000050020FD040020FF3F000864
:1008F00078360008004000083C0000204D00002031
:10090000B4F1005F84D300F069FC00F10050421E96
:1009100094423FF67DAF20460E493A4602F072FE01
:1009200010E06FF0080043420E213046DAB2FFF7C4
:1009300017FE00F067FB0020BDE8F0814FF0FF30AC
:10094000BDE8F0810449087842420F21304602F0A8
:100950007F02ECE74C0000204000002010B5114B56
:1009600088B01A7899788DF800200446DA7858789B
:100970001B798DF802108DF803208DF801008DF899
:10098000043000F087FBF7218DF8050001208DF879
:1009900006008DF8071020466946082200F08CF802
:1009A00008B010BD7837000808B52020FFF7D6FF43
:1009B0001020FFF7D3FF024B0020187008BD00BFC6
:1009C000FD04002010B5044600282CD1174A184910
:1009D000102313700B70174A174B184918601060DA
:1009E0000860174B174A184918601060086000F03B
:1009F00061FF164B164A1C70164B174914701C7079
:100A00000A78C00F422A04D114490A78110658BF47
:100A10001A70134B00211980124900220023C1E9EA
:100A20000023404210BD4FF0FF3010BD00000020F9
:100A300001000020040500200C05002030050020E6
:100A40003805002020050020100500201405002096
:100A50001805002015050020D03F0008D13F0008F0
:100A6000160500202805002010F0F00F38B50446C8
:100A70000D4604D101280CBF0C4B0D4B1C780D4BBF
:100A80001A6864F3071542B904F0F004102C0AD177
:100A90002846BDE8384000F07BBF204629469047F5
:100AA0000028F1D038BD4FF0FF3038BD01000020E4
:100AB00000000020040500202DE9F04180460E468C
:100AC00017460024BC4235D23B1B022B0DD0032B12
:100AD00019D0012B19D1325D052161F3030562F3B1
:100AE0000F2501346FF317450AE03119305D4A785C
:100AF000062363F3030560F30F2562F31745023401
:100B00006FF31F650FE0072000E0042060F303058A
:100B10003019335D4178827863F30F2561F317450F
:100B200062F31F65033440462946FFF79DFF002806
:100B3000C8DA00E00020BDE8F081000030B5A1B0C7
:100B4000F0238DF80030134B7E2232258DF80320E0
:100B50001A788DF8045000240F258DF801408DF887
:100B600002408DF805208DF8065002AB0D5D5A1E2F
:100B700035B101341A4603F8015C0133642CF5D118
:100B8000F72102F8011B6946521AFFF795FF21B0C1
:100B900030BD00BF1505002000B589B0F0238DF8E9
:100BA000003000238DF801308DF802307E238DF85F
:100BB000033032238DF80430084B8DF806101B7873
:100BC0008DF80720F7218DF80810092269468DF865
:100BD0000530FFF771FF09B000BD00BF150500200B
:100BE000F0B5454E8BB0337804460D461746FFF7F7
:100BF000F1FC00287CDA31780D295AD001D829B1CE
:100C000069E00E2974D00F2965D15AE03B4B1DB124
:100C1000012D03D11F706BE01D7069E01878052865
:100C200029D011D8022820D004D801283DD120464F
:100C3000334937E003281BD0042836D100F0C0FA2E
:100C400030490246684623E0082826D006D8062800
:100C500019D0072829D100F0C1FA16E009281FD0C1
:100C60007F2822D1FFF7A0FE42E02046264919E066
:100C70002046264916E0684600F0B4FA00282046CF
:100C800009DA23490EE000F0A1FA2249024668463B
:100C900001F004F82046694604E020461E4901E0C0
:100CA0001E492046FFF74AFF22E020460E210D2272
:100CB00004E0022D1CD120460E211022FFF76CFF0C
:100CC00016E0174A0DB1012D01D1556010E05268B0
:100CD00072B92046F2E70E210A462046FFF75CFF74
:100CE0000F49054B0A7800206FF307020A7018704D
:100CF00000200BB0F0BD00BF080500203405002027
:100D0000183700083A3700081F3700083037000846
:100D10003F370008413700084437000856370008BD
:100D200018050020F72910B50A465AD82E4B197815
:100D300001F0080303F0FF041BB12C4B1B78834226
:100D40004CD1A0F11103062B48D9284B187004BBD5
:100D50002548037803F00703042B03D82448C05C1C
:100D6000904221D101F00701052903D121480178E2
:100D7000914219D15A1C1C4B197802F0070060F3FC
:100D80000201052819702CD9CAB242F00800187067
:100D900027E0130611D5F72A06D101F01001CBB2D6
:100DA00013B10221FFF71CFF0F4B134A19780020E3
:100DB0006FF307011970107010BD01F01004E4B258
:100DC00044B9094B197841F0100119700A4B2146BA
:100DD0001A7000E00121FFF703FF02E04FF0FF303F
:100DE00010BD002010BD00BF180500201405002014
:100DF00078370008150500200805002001F00F03D2
:100E00002DE9F0470F46C1F30728C1F307494FEA20
:100E1000116A03F1080101F00F010629064602D804
:100E2000002A58D17AE0B8F1F00F05D003F10C0098
:100E300000F00F01032929D83A49D1E9004554EAC5
:100E4000050023D106F0F004302C4FF000000CD048
:100E5000502C13D0102C19D1334C208006F00F00E9
:100E6000012404FA00F0088010E02F4C208006F0E6
:100E70000F00012404FA00F0488007E02A4C20808B
:100E800006F00F00012404FA00F08880991E0D2955
:100E900044D8DFE801F01E1E071B242443434343CC
:100EA00043434307B8F1F70F13D83046414607F0E4
:100EB0000F07FFF737FF0F2F30D049463046FFF7B7
:100EC00031FF30465146FFF72DFF27E0B8F1F70F0D
:100ED00005D91AB3304627F0F00190471EE01A1FDB
:100EE00012F0FF041AD030464146FFF71BFF012CD9
:100EF0000CD030464946FFF715FF022C05D030468E
:100F00005146FFF70FFFD04600E0C846B8F1F70F93
:100F100004D1044800220023C0E900230020BDE8DA
:100F2000F08700BF280500201605002013B50446F1
:100F300001A800F045FD002807DB0199C1F303106B
:100F400010302246FFF75AFFF2E72849D1E9002383
:100F500052EA030047D0264B1888B0F57A7F42D971
:100F60000A8862B1002142FA01F313F0010003D1B3
:100F700001311029F7D101461031C8B21AE04B886F
:100F80005BB143FA02F010F0010103D10132102AE3
:100F9000F7D10A463032D0B20CE0888850B140FA1E
:100FA00003F111F0010203D10133102BF7D11346E5
:100FB0005033D8B20F4B1A7802F00801C9B249B1C8
:100FC0000D490978814205D16FF307021A700B4B66
:100FD00000221A700A490A6802B1904703480022A9
:100FE0000023C0E9002300201CBD00BF280500200D
:100FF0001605002018050020140500200805002013
:101000003805002010B500F007FD044600F048F850
:10101000054B1A884FF6FF718A4240EA040001D05E
:1010200001321A8010BD00BF16050020114BF7B524
:101030001C680746E4B1C1F30764C1F30720C1F39C
:1010400007420D4D8DF8064001F00F0100246E5C43
:101050008DF804008DF805202546B54208DA01AA6E
:10106000044B515D1B683846984701350443F4E74B
:101070002046FEBD0C05002008370008012803D0DB
:10108000034B1870002070474FF0FF30704700BFCF
:1010900001000020014B1878704700BF15050020A3
:1010A0000020704713B5044600287AD11F20012183
:1010B00000F036FF3C4B00949A6802F00C000828C0
:1010C00002D1012000905DE0196841F001021A6030
:1010D0009C60186820F08471344821F480321A60D2
:1010E0005860196821F480221A60DC600194186845
:1010F00040F4803119602C4B1A6802F400300090E3
:1011000001994A1C0192009818B90199B1F5A06F94
:10111000F1D11B6813F4003218BF0122009200982D
:1011200001282FD1204B2248196C41F080521A64BB
:10113000016841F48042026098689860996841F4BF
:1011400000429A6098681B4A40F4A05199605A6026
:10115000186840F0807119601868134A8101FBD546
:10116000154B40F205611960906820F00301916011
:10117000936843F0020090600B4A916801F00C0301
:10118000082BF9D10D48002100F0A2FD4FF440706A
:1011900000F094FD009A012A14BF4FF0FF300020A8
:1011A00001E04FF0FF301CBD003802401030002439
:1011B0000070004008544007003C02400000000856
:1011C000014B1868704700BF002004E0024B1888EC
:1011D00081B28802704700BF227AFF1F4FF440306F
:1011E0007047000000230B4A591089180A78D90764
:1011F00058BF120902F00F02092A94BF302137218B
:101200008A18C2540133182BEDD10021017608460B
:10121000704700BF107AFF1F074B1A681AB9EFF327
:101220001081064801604FF0010080F310881A68B1
:10123000511C196000207047400500203C0500202B
:10124000074A13683BB1581E106038B905490A684F
:1012500082F3108802E04FF0FF30704700207047A3
:10126000400500203C0500200F291CD80F4BDA68F0
:10127000D343C3F30222C2F1040301FA03F10901CB
:1012800000F16043CAB203F56141012381F80023F4
:1012900042B200F01F00510903FA00F2044840F87E
:1012A0002120002070474FF0FF30704700ED00E034
:1012B00000E100E073B5054668460E46144600F0AE
:1012C0000EFE02238DF805300096062C29D8DFE8A3
:1012D00004F02604090F13181D0003208DF80400E4
:1012E000002302E000238DF804308DF8073012E06F
:1012F00000228DF80420F8E700218DF80410012366
:10130000F3E701208DF80400002302E001238DF8AB
:1013100004308DF806302846694600F093FD002021
:1013200001E06FF001007CBDC30710B5044605D590
:1013300006484FF480510522FFF7BCFF34F00F033D
:1013400014BF6FF00100002010BD00BF000C024070
:10135000C20707D5074B11F0010F4FF4805214BF9D
:101360001A835A8330F00F0314BF6FF0010000207E
:10137000704700BF000C024030B5012185B0044623
:10138000102000F0E5FD54204443611E0D4CADF8E3
:1013900004104FF6FF730025204601A90293ADF813
:1013A0000C50ADF8065000F01BFE01210A46204605
:1013B00000F060FE2046012100F050FE284605B0F6
:1013C00030BD00BF001000400348012108B5416254
:1013D00000F064FE002008BD00100040054810B574
:1013E0000121446A00F04FFE00280CBF20464FF058
:1013F000FF3010BD001000401FB50446B8B90120F1
:10140000014600F0B1FDA7204FF6FF73ADF80400D0
:1014100001A909480293ADF80C40ADF8064000F070
:10142000DFFD0548012100F019FE204601E04FF0E4
:10143000FF3004B010BD00BF00000140044B596AEA
:1014400089B25A6A521A92B28242FAD9002070477F
:101450000000014012230B8000487047B437000899
:1014600004230B8000487047B0370008704770476E
:101470007047704770470020704700207047000099
:1014800065230B8000487047F337000810B50B4BFD
:101490008CB098781A888DF8060002A80C46ADF832
:1014A0000420FFF79FFE0028ACBF02A801A8044952
:1014B000224601F065F902480CB010BDE43700087F
:1014C000E41B002070B5164B86B00A4601AC03F150
:1014D000100618685968254603C50833B3422C46E0
:1014E000F7D11888002328800E495818017859B17F
:1014F00020395F298CBF002101210133202B06D028
:101500000029F1D101A805E0002BFBD001E0002962
:10151000F8D00448044901F033F9034806B070BD1F
:1015200044370008E03F0008E41B0020FFF7CABF73
:10153000FFF7C8BF1146FFF7C5BF00001FB5084C35
:101540000A462068616801AB03C3A068054C1860B7
:10155000214601A801F014F9204604B010BD00BFD7
:10156000E7370008E41B0020022908B503D108462C
:10157000002100F067FA002008BD012908B503D159
:101580000846002100F056FA002008BD10B50221DF
:10159000044601F046FD2046812101F042FD002075
:1015A00010BD002000F08CB9012000F089B90000C6
:1015B000022110B5402204460B4601F011FD8121A5
:1015C00040220223204601F00BFD0221034A044879
:1015D000402301F03FFD002010BD00BFAC150020EE
:1015E000EC15002073B50120244C014600F098FC56
:1015F00000204FF4D853022503268DF806008DF8FD
:1016000007006946204600938DF804508DF8056068
:1016100000F018FC204608210A2200F069FC204650
:1016200009210A2200F064FC20460B210A2200F066
:101630005FFC0A2220460C2100F05AFC4FF4806126
:1016400000918DF804502046012569468DF8075019
:101650008DF8056000F0F6FB0A210A46204600F0EE
:1016600047FC29464FF4804000F07EFC802029464C
:1016700000F062FC284600F035FB7CBD0000024013
:1016800043200821FFF7F0BD014801F06FBD00BF06
:10169000EC15002080B2FFF7D1BE4FF47A735843A7
:1016A00080B2FFF7CBBE4FF0A0431868C0F3C04034
:1016B00070470000022837B5054642D8FFF7F3FF10
:1016C0000446FFF76EFF45BB14F0FF0F25D01E4CFC
:1016D0002046FFF787FF1D481D491E4AC4F8E40550
:1016E000C4F8E81520460121C4F8EC2501F0AEF855
:1016F000204601F050F9204601F0C0F92046FFF7DE
:10170000BFFF01210323204684F8101184F8123111
:10171000FFF74EFFFFF748FF11E00D4B0D4A009316
:1017200001210A4B084800F0BBFD074801F016FDF7
:101730004CF25030FFF782FE034801F007FD002015
:1017400001E04FF0FF303EBDEC150020803700086F
:1017500058380008C837000870B5254CD4F8E4356F
:10176000002B43D0FFF758FD22480178002939D0DB
:10177000D4F8DC63B608B3B2002B33D01E4A10880D
:1017800081B21BB2C1F5007293422BDA00241B4DCB
:1017900055F82450C5F3031010302946FFF746FCD6
:1017A00090B9174B174A198889B242F82150198805
:1017B0004A1C91B2B1F5007F198028BF18800E48ED
:1017C00003885A1C91B201800134301B03B2002BF4
:1017D000DDDC0849064800220A7040230221074A3E
:1017E00001F038FCBDE87040FFF72ABD70BD00BFB6
:1017F000EC1500205015002046050020AC150020F7
:1018000052150020500D0020234BD3F8E40510B5ED
:10181000002840D0FFF700FD20490A78002A36D181
:101820001F4B188881B2002931D01E4A1078002839
:101830002DD019888AB2102A98BF1988174B94BFE7
:1018400089B210210120187015480288531A9AB2E3
:10185000028000220BB29A4213DA134B13481C8801
:10186000A4B250F82440124840F8224018880130B1
:1018700080B2B0F5007F188001D3002018800132BB
:10188000E8E705480A4A81219B0001F000FCBDE819
:101890001040FFF7D5BC10BDEC1500204C0D00200A
:1018A000561500205A150020581500204C05002020
:1018B0005C150020002814BF4FF0FF300020704757
:1018C0000D49002310B50B800C4C0D4923800B8073
:1018D0000C4C0D4923700B800C4C0D4923801A468B
:1018E0000B800C4C0C4B012110B121701A7001E0DF
:1018F00022701970002010BD4605002052150020EE
:1019000048050020501500205615002044050020F1
:10191000581500205A1500204C0D002038B5184CE1
:101920002378054613B94FF0FF3038BD15480188BC
:101930008AB2B2F5FF7F07D9FFF766FF2378002B45
:10194000F1D06FF0010038BDFFF766FC0E4B0F4978
:10195000188882B2501C41F8225082B21A8019882D
:1019600088B2B0F5007F01D300221A80054B198898
:10197000481C82B21A80FFF763FC002038BD00BF0C
:101980005A15002056150020440500204C05002063
:1019900010B504462046FFF7C1FF831C08D1074B52
:1019A0001A8842F20F718A4207D8501C1880F1E75A
:1019B000002802DB014B00221A8010BD54150020C4
:1019C000124B10B50446188881B2D9B1FFF724FC38
:1019D0000F4B10491A8890B251F8202022601C88C1
:1019E000601C81B2B1F5007F198001D300221A80FA
:1019F000064C2388581E81B22180FFF721FC2288E3
:101A000090B210BD4FF0FF3010BD00BF4605002062
:101A100048050020500D002008B5054801F01EF8CB
:101A200018B9FFF799FEFFF7EFFE002008BD00BFD1
:101A3000EC150020024B00221A70FFF7E5BE00BF34
:101A40004C0D0020024B01221A70FFF785BE00BF2B
:101A50005015002020B10368197001684A1C02600B
:101A600070472DE9F843141E8046894601DC202783
:101A70000FE0002219F8021009B10132FAE7A24280
:101A8000B4BFC2EB04040C4613F0020F0CBF2027B6
:101A90003027DB070CD42546002D05DD40463946AE
:101AA000FFF7D8FF013DF7E724EAE476A41B00E046
:101AB00000263546C6EB0903595D21B14046FFF7C4
:101AC000C9FF0135F6E72646002E05DD40463946BA
:101AD000FFF7C0FF013EF7E7002CACBF2819281C18
:101AE000BDE8F8832DE9FF470C9EDDF83480814680
:101AF0000C4651B930228DF804208DF8051032467D
:101B000001A94346FFF7ADFF35E033B10A2A04D1FE
:101B1000002902DA4C42012700E0002704AD00232F
:101B200005F8013DAA466CB1B4FBF2F302FB134485
:101B3000092C02DD0E993A396418303405F8014D4C
:101B40001C46EFE787B14EB118F0020F06D04846A9
:101B50002D21FFF77FFF013E012705E02D2005F134
:101B6000FF3A05F8010C00274846514632464346E5
:101B7000FFF777FF381804B0BDE8F087F0B589B0FB
:101B800006460D46059200242B7823B1252B79D1EA
:101B900068786A1C28B9002E7BD030680022027059
:101BA00077E025286DD02D2802D1AA1C012300E062
:101BB0000023174601323978302902D143F002035D
:101BC000F7E700223978A1F130005FFA80FC3D464A
:101BD0000137BCF1090F03D80A2505FB0202F1E722
:101BE000732909D1059F391D059139682A4F30465F
:101BF000002908BF394641E064290ED18DE80C0068
:101C0000059961230293081D096805900A22304650
:101C10000123FFF767FF241839E0782906D10599D9
:101C2000081D8DE80C000590612207E058290AD1B3
:101C30000599081D8DE80C0005904122029230465E
:101C4000096810220BE075290BD18DE80C0005996D
:101C500061230293081D096805900A22304600237B
:101C6000D7E7632913D10599081D0968059000205D
:101C70008DF81C108DF81D0007A93046FFF7F1FE06
:101C8000C9E7154630462978FFF7E4FE01340135EF
:101C90007AE7204609B0F0BD743800080EB40FB5DD
:101CA00005AA019052F8041B01A80392FFF766FFF2
:101CB00004B05DF804EB03B07047000040F0BF6073
:101CC000024B40F40031D960704700BF00ED00E0E6
:101CD00021F0604121F07F02014B10439860704772
:101CE00000ED00E0014B5861704700BF003C01402F
:101CF000024B1A6842F4006018607047003C0240D2
:101D0000024B1A6842F4805018607047003C024051
:101D1000044B1A69002A04DA034800F1883158603C
:101D200059607047003C024023016745024B1A6925
:101D300042F0004018617047003C0240014BD860FF
:101D4000704700BF003C02400B4BDA68D0030DD453
:101D5000D868C1060CD4D96811F0EF0F0AD1DB683E
:101D600013F0020F0CBF08200720704701207047B6
:101D70000520704706207047003C024007B5082345
:101D80008DF80730FFF7E0FF8DF807009DF807009A
:101D90000128F7D09DF807000EBD000070B505467C
:101DA0000E46FFF7EBFF082813D10A4C236923F4F2
:101DB00040702061216941F400722261236943F07F
:101DC000010020612E60FFF7D9FF216921F0010297
:101DD000226170BD003C024070B5064641B1012948
:101DE00008D0022914BF4FF440754FF4007503E08A
:101DF0000D4601E04FF48075FFF7C0FF08281ED1A3
:101E00000F4C236923F44070206121690D43256143
:101E1000226922F0F8032361206940F002010E4399
:101E20002661226942F480332361FFF7A7FF21690D
:101E300021F002022261236923F0F801216170BDC3
:101E4000003C0240F0B50E680022012303FA02F3C1
:101E500003EA06059D423ED107680C79530027FA34
:101E600003F707F00307A7420DD007684FF0030CF4
:101E70000CFA03FC27EA0C070760076804FA03FC66
:101E80004CEA07070760013C012C17D88768032438
:101E900004FA03F427EA040787604C79876804FA98
:101EA00003F43C438460446824EA05058C7945606A
:101EB000456804FA02F4A4B22C434460C5680324C4
:101EC00004FA03F425EA0405C560CD79C46805FA6F
:101ED00003F32343C3600132102AB6D1F0BD0021C1
:101EE0004FF6FF730360017141718171C1717047D9
:101EF00001F00703C908083130B59B0050F82150A4
:101F00000F2404FA03F425EA040440F8214050F8B1
:101F1000214002FA03F2144340F8214030BD000092
:101F2000044B1A6B09B1104301E022EA0000186368
:101F3000704700BF00380240044B5A6B09B1104390
:101F400001E022EA00005863704700BF00380240F9
:101F5000044B1A6C09B1104301E022EA0000186436
:101F6000704700BF00380240044B5A6C09B110435F
:101F700001E022EA00005864704700BF00380240C8
:101F8000044B1A6909B1104301E022EA000018610C
:101F9000704700BF00380240044B5A6909B1104332
:101FA00001E022EA00005861704700BF003802409B
:101FB000044B1A6A09B1104301E022EA00001862DA
:101FC000704700BF00380240044B5A6A09B1104301
:101FD00001E022EA00005862704700BF003802406A
:101FE0001C4A038890429BB212D002F58062904254
:101FF0000ED0B0F1804F0BD0A2F58032904207D0C6
:1020000002F58062904203D002F58062904203D1D3
:102010004A8823F0700313430F4A904208D002F518
:102020008062904204D023F440730A899BB2134328
:1020300003804B680A88C362064B0285984203D02E
:1020400003F58062904201D1897A0186012383825F
:10205000704700BF0000014000100040038819B124
:1020600099B241F0010303E023F001010A04130CCB
:102070000380704783899BB20AB1194301E023EAC8
:10208000010181817047038A828911EA030092B2BB
:1020900003D011420CBF002001207047C9438AB20F
:1020A00002827047D0F8E83510B5044618698047B9
:1020B000032184F81211002010BD08B590F81231E8
:1020C000042180F8133180F81211D0F8E805C268B5
:1020D0009047002008BD08B5D0F8E435D96901B1B2
:1020E0008847002008BD08B5D0F8E435196A88474C
:1020F000002008BD08B5D0F8E435596A88470020AB
:1021000008BD002110B5402204460B4600F068FFD0
:10211000802140220023204600F062FFD4F8E80529
:10212000012384F812314168A0788847002010BD4F
:1021300013B56946044600F023F99DF8001001F03C
:102140001F03012B0CD006D3022B0ED1204669466B
:1021500000F046F90EE02046694600F0BBF909E0C0
:102160002046694600F09EF904E0204601F0800117
:1021700000F0A8FF00201CBD70B50446002947D11F
:1021800090F81131022B37D1D0F83821D0F8243112
:102190009A4211D9D21AC0F83821C078012804D146
:1021A000D4F82811CB18C4F828312046D4F82811C7
:1021B00092B200F0B5F81FE0D0F83C51B5FBF3F651
:1021C00003FB16565EB99D4209D3D0F840219542D3
:1021D00005D2324600F0A4F8C4F840610CE0D4F80F
:1021E000E405C16829B194F81231032B01D12046CE
:1021F0008847204600F0B5F894F81621012A10D13E
:10220000094920690B680022436084F8162108E020
:10221000D0F8E4355B6923B190F81221032A00D18C
:102220009847002070BD00BFE01B002010B5044699
:1022300059BB90F81111032930D1D0F89023D0F870
:102240007C339A4214D9D21AC0F89023C07801285E
:1022500004D1D4F88013C818C4F880039A4228BF68
:102260001A462046D4F8801392B200F062F815E0C6
:10227000D0F8E4150B6923B190F81221032A00D19C
:102280009847204600F05EF808E0D0F8E4359B69F6
:1022900023B190F81221032A00D19847002010BDE5
:1022A0002DE9F041069F0446164698460D46FFF775
:1022B00099F920462946C4F8E485C4F8E875C4F8BD
:1022C000EC6500F042FED4F8E835186880472046F7
:1022D000BDE8F041FFF7D4B9D0F8E43510B50446B5
:1022E0001A689047D4F8E80581688847002010BD37
:1022F00008B5D0F8E4355A689047002008BD38B5D5
:1023000004460D46C4F83C21C4F838211346022285
:1023100080F8112100212A4600F0B9FE002038BDC6
:1023200010B50C4613460021224600F0B0FE0020F6
:1023300010BD10B50C4613460021224600F08AFE5F
:10234000002010BD0021042310B50A46044680F881
:1023500011310B4600F09BFE204600F0D8FD002016
:1023600010BD0021052310B50A46044680F811313E
:102370000B4600F06FFE204600F0C9FD002010BDA6
:1023800090F8CC350B7090F8CD254A7090F8CE358A
:1023900090F8CF2503EB02224A8090F8D03590F8D0
:1023A000D12503EB02228A8090F8D23590F8D3250C
:1023B00003EB022293B2CB800121C0F8403180F8B8
:1023C0001111704710B58021044600F07BFE2046B5
:1023D000002100F077FE2046BDE8104000F097BDD8
:1023E00070B54E788A88012E04460D46D3B211D0BE
:1023F00029D3032E51D190F81221022A2AD0032A80
:1024000049D14988A9B9A3B1802B12D0194600F04F
:1024100059FE0EE090F81221022A1BD0032A3AD16D
:102420004988002939D153B1802B08D0194600F0D2
:1024300067FED4F8E405294683682046984720467D
:10244000FFF780FF29E090F81251022D02D0032DF2
:1024500021D106E00BB3802B1FD0194600F032FECD
:102460001BE012F0800F4FF0280006D002F07F0230
:1024700000FB024191F81E3103E000FB034393F897
:102480007633074803B10123036005492046022241
:10249000FFF735FF01E0FFF795FF002070BD00BF9B
:1024A000A415002038B590F81231032B04460D46D0
:1024B0000CD10A79012A09D8D0F8E4359A689047F6
:1024C000E88828B92046FFF73DFF01E0FFF77AFFD3
:1024D000002038BD70B54B78052BA2B004460D46E0
:1024E00000F0838008D8012B00F01581C0F0DA805D
:1024F000032B40F03381E6E0082B00F0C58003D8C1
:10250000062B40F02B8106E0092B00F08E80552B26
:1025100040F024810FE14888010A4B1E062B00F28F
:102520001D81DFE813F007001A0027001B011B01C3
:102530001B011B01D4F8EC15A0780A680DF1060107
:1025400090470146E888402803D094F81231012BC7
:102550003BD10822ADF8062037E0D4F8E4050DF1B0
:102560000601826AA0789047022343700146C4F8AE
:10257000F0052AE0C1B2A07805291FD8DFE801F0F4
:1025800003070B0F1317D4F8EC25536812E0D4F8A7
:10259000EC158B680EE0D4F8EC35DB680AE0D4F873
:1025A000EC25136906E0D4F8EC154B6902E0D4F889
:1025B000EC2593690DF10601984705E0D4F8E43560
:1025C0000DF10602DB6A98470146BDF806000028B7
:1025D00000F0C880EA88002A00F0C480824228BF48
:1025E0000246ADF806202046B5E08A88002A40F071
:1025F000B580C988002940F0B1806E8890F812211A
:1026000006F07F03032A1E4600F0A88080F81431EC
:10261000194600F093FD2046FFF794FE0EB102200C
:1026200000E0012084F812019CE08B784F4A012BD6
:10263000137000F2938090F81221022A03D0032A2B
:1026400040F08E8008E0002B61D00121032380F848
:10265000101180F8123114E043B9022180F81211F0
:1026600080F810311946FFF743FE50E090F8101142
:1026700001294CD0FFF73CFE3C480178204684F805
:102680001011FFF729FE42E0CA88012A66D190F8AE
:102690001231022B04D0032B62D100F588715AE06D
:1026A000334958E090F81221931E012B58D8314835
:1026B000D4F81821002101600AB1022303602046EA
:1026C0002C49022247E04B88012B2DD0022B49D107
:1026D0008A8812F0FF0F45D10069110A4A1E43682B
:1026E000042A0FD8DFE802F0030507090B000120D8
:1026F00006E0022004E0032002E0042000E00520C0
:1027000060F306131C490B60012384F81631204640
:10271000FFF718FE26E090F81221931E012B1FD818
:102720004A88012A1ED10023D4F8E425C4F81831C0
:1027300093689847EBE70978C0290FD16B886BB98C
:10274000EE88802E0AD10D49324602A800F05AFFC9
:10275000204602A93246FFF7D2FD03E02046294673
:10276000FFF730FE002022B070BD00BFA015002092
:10277000A81500209C150020E01B00207B380008D5
:1027800030B5C0B10023C55CDCB20133002DFAD1F5
:10279000631C5B00138003220B704A700138022314
:1027A00010F8012F3AB15C1CCA54E2B20233002483
:1027B0008C54DBB2F4E730BD37B50023104C0193E5
:1027C00005460320FEF766FFE8680269013C0192B6
:1027D00013D001990029F4DA019B43F00102019220
:1027E0000199074A01610369013A019302D00199F5
:1027F000C907F8D40320FEF74DFF00203EBD00BFFF
:10280000410D030030B5C4786CB900EB820003338E
:10281000D0F8D0509B1022469A4204D051F82200A2
:1028200001322860F8E7002030BD10B50332D0F83F
:10283000D0409210002393424FEA830004D02068D6
:1028400041F823000133F6E7081810BDF0B5002366
:10285000012240240129C370827084800CD102239C
:10286000082604224FF4A0740372C17206704270ED
:10287000C4804FF0A04309E041B90C23C17203703A
:1028800006214FF4A065204B4170C58003F500611F
:1028900045780161C3600246194600240432AC4207
:1028A00001F1200608D201F5106701F530611165CC
:1028B000576101343146F1E703F5806403F588611F
:1028C00044610478C0F8CC10002203F5A061A24254
:1028D00006D200EB82050132C5F890102031F6E7F0
:1028E00003F580510022A24207D200EB820501329B
:1028F000C5F8D01001F58051F5E703F56063C0F825
:102900000C310020F0BD00BF0000044038B5037A50
:102910000025012B0446C3681FD1986B617A65F3CB
:10292000104009B140F480109863DA686FF38612A2
:102930006FF396526FF351426FF3D342DA60204641
:10294000FFF73AFFE378012B19D1052161F3440524
:10295000E06845F02005856011E0DA6842F040014A
:10296000D960FFF729FF607AE36800280CBF4FF4B5
:1029700034124FF474129A631420FEF78EFEE2783C
:10298000012A06D1E368996821F03E0040F02A024E
:102990009A60002038BDC3689A6842F001009860D0
:1029A00000207047C3689A6822F0010098600020F8
:1029B0007047000007B500230193019A42F02003FD
:1029C0000193019A094B61F38A120192C26801983E
:1029D00010611169013B019102D001988006F8D481
:1029E0000320FEF757FE00200EBD00BF410D03007F
:1029F00007B500230193019941F010020192C068CC
:102A0000019B074A03610169013A019102D0019BD0
:102A1000D906F8D40320FEF73DFE00200EBD00BF0E
:102A2000410D0300C26808B5D36801296FF35D73D7
:102A30006FF39E7302D143F0005302E009B943F0F3
:102A400080433220D360FEF728FE002008BDC36813
:102A5000586900F0010181F001007047C3685869AE
:102A600000F001007047C3685A69986910407047C8
:102A700003691A6861F301021A60704710B5C368F0
:102A800000226FF080414FF0FF349A6159615C6021
:102A900059610A499961C07890420CBF10211146D2
:102AA00041F4872040F00811986941F4401120EA70
:102AB000010001439961104610BD00BF000800806D
:102AC00038B5D0F80C31016900221A6015460A6841
:102AD00065F3CC220A60C37A012B04461BD1032183
:102AE000FFF7C6FFE068C02380214FF4800263F344
:102AF0000F05416261F31F4561F30F024FF4A071AE
:102B00008262C0F8045161F30F056FF31F45C0F8EE
:102B10000851C0F80C5110212046FFF74BFF20460A
:102B2000FFF766FF206900234FF0FF320361436126
:102B30008261C36161788B4214D204EB830201335A
:102B400090690168C1F3076202F08001CAB2002AED
:102B500014BF4FF09041002101600022FF2102616B
:102B60008160E7E700236078834214D204EB83009E
:102B70000133426D1168C1F3076000F08001C8B2F3
:102B8000002814BF4FF09041002111600020FF2168
:102B900010619160E7E723691A6942F48071196155
:102BA000E078012804D1054A402161F359421A63B3
:102BB0002046FFF763FF002038BD00BF030101007E
:102BC00003699868C0F341014B1E022B02D8024AE8
:102BD000D05C704703207047FB38000803698169A7
:102BE00010B59C680A68C4F34100022802D06FF354
:102BF0000A0202E0032060F30A020A60596841F405
:102C000080725A60002010BD30B54D780B780022DC
:102C1000012D00EB830405D105FA03F5A46965F3E2
:102C20000F0205E0012505FA03F3646D63F31F420B
:102C30002368C3F3072505F08005EDB26DB98D68F3
:102C400065F30A03CD78C98865F3934361F399531B
:102C500043F0805343F4004121600069C3691A4383
:102C6000C261002030BD30B54D780B780024012DB5
:102C7000224600EB830105D105FA03F3896963F36A
:102C80000F0205E0012505FA03F3496D63F31F42C6
:102C900000696FF3CF340C60C16921EA0202C2619E
:102CA000002030BD70B54E780A78012E0B4600EB3F
:102CB000820148D18D695C6929682A6964F312022E
:102CC00014B966F3DC420BE09E68A419013CB4FB26
:102CD000F6F6DC7866F3DC42012C08BF64F35E7222
:102CE0002A61C278012A06D11A7800EB82041A6997
:102CF000A46962610CE0DA78012A09D05A693AB114
:102D000002691C78556B012606FA04F42C435463BF
:102D1000DA78012A07D102699268D20554BF41F0DE
:102D2000005141F080511A7800EB820241F00441D9
:102D300092691160D978012937D1D9681A789B8AAC
:102D4000FFF760FD31E04D6D5E692A689C68296976
:102D50002EB964F31201012464F3DC410AE0361950
:102D6000013EB6FBF4F666F3DC41B605B60D7443DE
:102D700064F312012961C178012905D11C7800EBA7
:102D800084014C6D19696161D978012906D159799D
:102D900011B142F0005201E042F080521B7800EB8A
:102DA000830042F00441426D1160002070BD73B594
:102DB0004D78012D3DD183694A691E681C690094D4
:102DC000E4B242B962F306049DF802208DF8004097
:102DD00065F3C4020EE08D68AA428ABF4D6162F3BA
:102DE000060465F306049DF802208DF800400124D6
:102DF00064F3C4028DF80220009A1A61C278012A95
:102E000005D10C7800EB840294690A69626146F08E
:102E100004461E60C378002B34D14A69002A31D0A1
:102E200003690A78586B012101FA02F202435A63DE
:102E300028E00B784E6900EB8302536D8A681D68A9
:102E40001C690094E4B206B14A6162F306049DF87D
:102E500002208DF80040012464F3C4028DF80220A2
:102E6000009A1A61C378012B05D10A7800EB82031E
:102E70005A6D0B695361097800EB810045F00445F8
:102E8000426D156000207CBD4B780978012B00EB6A
:102E900081000DD180690368C3F3076202F08001ED
:102EA000CAB20AB143F0804343F40011016004E068
:102EB000436D1A6842F400111960002070474B7886
:102EC000012B0B78C97800EB83000CBF8269426D3F
:102ED0001368881E6FF35553012898BF43F0805341
:102EE00013600020704703699A69D8691040000C8C
:102EF000704700EB810102694B6D99685069084089
:102F0000704703699869D969084080B2704782B0F8
:102F100000230093C021012200238DF8031062F3E7
:102F2000C40318218DF802308DF80010436D009A0B
:102F30001A61C178012906D100F2CC5058611A6893
:102F40004FF080221A6002B0704710B50446FFF7B8
:102F50007DFC012384F81231002384F81431627857
:102F6000934213D2282202FB034101F58E72012005
:102F700081F81D0181F81C31A1F822314020002187
:102F8000D1709060D16051610133E8E7002360782F
:102F9000834213D2282101FB034000F55D7200211A
:102FA00080F87433A0F87A3380F8751380F87713BB
:102FB00040209060D16051610133E8E72046FFF77F
:102FC000F1FC2046FFF7A2FC00212046FFF72AFD76
:102FD0002046FFF775FD2046BDE81040FFF7DBBC3B
:102FE00070B5CDB201F07F044FF0280606FB040453
:102FF00015F0800F14BF04F58E7404F55D7401F0B4
:103000007F01ED0921706570A260E37005B1E18078
:10301000022B01D1002323712146FFF7F5FD00208B
:1030200070BD10B5CAB201F07F034FF0280404FB55
:10303000030312F0800F14BF03F58E7303F55D7365
:1030400001F07F01D20919705A701946FFF70BFE83
:10305000002010BD38B501F07F04282505FB0405CC
:1030600005F55D7185F874434B610023CA608B617F
:103070004B70C378012B05F55C7508BF0A6114B964
:10308000FFF795FE01E0FFF70DFE002038BD70B59B
:1030900001F07F04282505FB040505F58E71012646
:1030A000CA600A61002285F81C414E7005F58C75D6
:1030B0008A614B6114B9FFF77AFE01E0FFF7F2FD78
:1030C000002070BDCAB212F0800F10B54FF0280377
:1030D00006D001F07F0403FB040303F58E7303E0C5
:1030E00003FB010404F55D73D209012401F07F01A3
:1030F00019709C705A701946FFF7C6FE002010BD6B
:10310000CAB212F0800F10B54FF0280306D001F0BC
:103110007F0403FB040303F58E7303E003FB010448
:1031200004F55D730024D20901F07F0119709C70D1
:103130005A701946FFF7C3FE204610BD02690023EE
:1031400061F30A1311680B431360704703695A68EF
:1031500003206FF341025A60FEF79FBA03695A6871
:1031600042F0020058600320FEF797BA2DE9F04FB5
:1031700085B00446FFF76BFC08B900203AE2204610
:10318000FFF771FC07460028F7D0C0F3074A0AF0A2
:103190000800C0B2002856D02046FFF7A4FEA34680
:1031A000804626464FF00009B8F1000F4AD018F0CB
:1031B000010F3FD05FFA89F3194620460093FFF7CD
:1031C00098FE10F0010F0546009B20D0706D012580
:1031D0008560E178A94207D10269DBF87C13C2F36C
:1031E00012000A1ACBF88C237148016820460A683D
:1031F00019469047E378012B09D1B9F1000F06D1A8
:1032000094F81101052802D12046FFF780FE05F051
:103210000201CAB212B1736D02259D6005F008006B
:10322000C1B239B1624A15682046AB689847706DE3
:103230000821816009F101094FEA580804360BF1B1
:10324000280BB1E701200AF0040A5FFA8AF3002B89
:1032500000F0B1802046FFF754FE264681464FF02D
:103260000008B9F1000F00F0A58019F0010F00F07F
:1032700099805FFA88FA236904EB8A0019695D6B0B
:10328000826925FA0AF59068EA01D5B20D43054036
:10329000EA071BD5586B464A012505FA08F120EAD2
:1032A00001005863B36910689D6051464368204629
:1032B0009847E178A94209D1B8F1000F06D194F8F6
:1032C0001121042A02D12046FFF721FE05F0080053
:1032D000C3B213B1B16908258D6005F01002D0B2F8
:1032E00010B1B36910259D6005F04001CAB212B15A
:1032F000B0694025856005F00203D9B211B1B26909
:103300000225956025F07F0010F0FF0F4AD028239A
:1033100003FB084101F58C75019504356869AB69BB
:10332000AA68C11AB069914238BF0A4602F1030C7B
:1033300082694FEA9C0C93B2634530D9A9696A69E6
:1033400091422CD25AB3A868C1EB020B834528BF27
:1033500083460BF1030E4FEA9E0CE968CDF800C0DE
:1033600052461FFA8BF32046FFF74CFAEB68AA6926
:10337000DDF800C003EB0B010BEB0200E960A86174
:103380006969B36988429A69D5D301982569027938
:103390006B6B012101FA02F023EA00036B63B5694C
:1033A0008022AA6008F101084FEA5909043658E75B
:1033B000040000200120FDB205F00201CAB212B1E2
:1033C000E36802215961C7F3076202F08003D9B2B2
:1033D000C9B1A07A40B1D4F80C31D4F80C216FF304
:1033E00041036FF3000313602169844A486820F0A9
:1033F00001034B60116820468B699847E0684FF0E5
:10340000004242610120C7F3072808F00801CBB24F
:103410006BB37A4994F812210B6800208DF80F00E5
:103420008DF80F2020465A6990472069E36882682A
:103430004FF400615961A07AC0B1D30716D594F852
:103440001521012A12D19DF80F30032B0ED1D4F88B
:103450000C11086840F001020A600B6843F0030099
:10346000086067490A6942F006030B61012005F014
:103470000801CAB242B1614803682046D96888474A
:10348000E06808224261012005F01005EDB2002D30
:1034900035D0E668B36923F01001B161366A28229D
:1034A00006F00F00C6F3434302FB0045022B05F56F
:1034B0005D750DD0062B1CD104F2CC51204608229C
:1034C000FFF7B3F9A969C6F30A168819A86110E0D5
:1034D00047F6F072324062B1C6F30A16E968324626
:1034E0002046FFF7A2F9EB68A86999198619E960E7
:1034F000AE61E3689A6942F010019961012008F019
:103500001003DAB2002A34D026697068002520F052
:103510000101716020462946FFF74CFA23462A46EE
:1035200066780433B24206D25E69FF21B160186D3D
:1035300001328160F4E70126206966F30F050B2153
:103540004FF0FF3266F31F458261C5614161016141
:1035500003686FF30A1303602046FFF7D8FC27497E
:10356000E0680B684FF4805242611A692046904728
:10357000304608F020085FFA88F1E9B12046FFF7ED
:103580002DFBE5682046ED68FFF71AFB032806D1FE
:1035900000214FF40070A170A080092204E00120F6
:1035A0004023A070A3800522E36862F38D254FF4C9
:1035B0000052DD6001205A61C7F3074707F0100190
:1035C000CBB24BB10D4802682046D1698847E36809
:1035D0004FF480105861012007F02007FFB24FB16F
:1035E000064A116820460B6A9847E0684FF40012BB
:1035F0004261012005B0BDE8F08F00BF040000204B
:1036000000ED00E010B50023934203D0CC5CC4541D
:103610000133F9E710BD0000000002408000000007
:10362000000402400080000000040240200000006E
:1036300000000240200000000004024000200000C2
:1036400000040240080000000004024004000000E2
:10365000000C0240000800000004024000100000BE
:10366000000C024000040000000002400080000046
:103670000004024000010000FFFFFFFF0000000007
:1036800000000000004000080800000000000000EA
:1036900000800008100000000000000000C00008CA
:1036A00018000000000000000000010820000000D9
:1036B00000000000000002082800000000000000D8
:1036C00000000408300000000000000000000608B0
:1036D0003800000000000000000008084000000062
:1036E0000000000000000A08480000000000000080
:1036F00000000C08500000000000000000000E0850
:103700005800000000000000000002030301020353
:1037100003030303020203014D494F5333320053A5
:10372000544D33324634444953434F564552590061
:1037300053544D3332463478780025303878003F82
:10374000002564004D494F53333220426F6F746C33
:103750006F6164657200286329203230313420544F
:103760002E204B6C6F7365002025303258002020CE
:103770002000253038582000F000007E3200000084
:10378000B11500088D15000877140008000000002E
:103790007B1400087B150008691500080000000074
:1037A000000000000000000081140008351500082A
:1037B000040309041201000200000040C016FE03C9
:1037C00010100102030100005514000861140008E4
:1037D0003D150008C51400088D14000831150008B7
:1037E0002D1500083432006D696469626F782E6FA0
:1037F00072670009026500020104803209040000BA
:10380000000101000209240100010900010109046D
:103810000100020103000207240100014100062407
:10382000020101000624020202000924030103012F
:10383000020100092403020401010100090502023A
:10384000400000000005250101010905810240003A
:1038500000000005250101036D1400086F14000825
:10386000A9150008731400087514000871140008E5
:10387000A3150008286E756C6C2900D10FED54CF8C
:10388000C5FBB89752389138910E7D0FED389301F2
:10389000910E9100C11F020E91F7041040006E10AE
:1038A0006EE76A0000000000000000000000000059
:1038B0000000000000000000000400000000000004
:1038C000000000000000002F55461F00D848403778
:1038D0006AF76A00300000C7062E734A2C137BE992
:1038E0007F32002A280D9BFE0B21EF422A2F73B551
:1038F000B8DA76E679BF0FEB793E0B0201020000E1
:1039000010100000080000202D2200087921000876
:1039100031210008D720000803210008BB2000083F
:10392000A5200008E7200008F5200008000000009E
:103930000000000000000000FFFFFFFFFFFFFFFF8F
:10394000FFFFFFFFFFFFFFFFFFFFFFFFFFFFFFFF87
:10395000FFFFFFFFFFFFFFFFFFFFFFFFFFFFFFFF77
:10396000FFFFFFFFFFFFFFFFFFFFFFFFFFFFFFFF67
:10397000FFFFFFFFFFFFFFFFFFFFFFFFFFFFFFFF57
:1040000000000220711F01086D1F01080906010848
:104010006D1F01086D1F01086D1F010800000000E1
:10402000000000000000000000000000B5190108B9
:104030006D1F0108000000002D1A0108691A01080F
:104040006D1F01086D1F01086D1F01086D1F01081C
:104050006D1F01086D1F01086D1F01086D1F01080C
:104060006D1F01086D1F01086D1F01086D1F0108FC
:104070006D1F01081D870108F98601086D1F0108E1
:104080006D1F01086D1F01086D1F01086D1F0108DC
:104090006D1F01086D1F01086D1F01086D1F0108CC
:1040A0006D1F01086D1F01086D1F01086D1F0108BC
:1040B0004D890108758901086D1F010881A3010858
:1040C00019A5010885A10108FDA201086D1F0108BD
:1040D0006D1F01086D1F0108FD9F0108BDA00108AB
:1040E0006D1F01086D1F01086D1F01086D1F01087C
:1040F0006D1F01086D1F01086D1F01086D1F01086C
:104100006D1F01086D1F01089D8901086D1F0108C1
:104110006D1F01086D1F01086D1F01086D1F01084B
:10412000158D01086D1F0108D58601086D1F010856
:104130006D1F01086D1F01086D1F01086D1F01082B
:104140006D1F01086D1F01086D1F0108E591010831
:104150006D1F01086D1F01086D1F01086D1F01080B
:104160006D1F01086D1F01086D1F01086D1F0108FB
:104170006D1F01086D1F01086D1F01086D1F0108EB
:084180006D1F01086D1F01080D
:020000040801F1
:100000002DE9F04740F22815C2F20005002646F619
:10001000C4642F46B046C2F200044FF0030A4FF00A
:100020000209012000F024FF2B7803B3206801218E
:1000300001F08CFC0128F9D12B78DBB2022B1ED009
:10004000032B17D0012B09D100201FF005F9002840
:10005000ACBF87F8009087F800A00026206801F068
:1000600011FB012000F004FF2B78002BDED121F0E2
:10007000EFFED6E709F008F987F80080EEE71FF0F9
:10008000EFF836B930461FF0F1F8061C18BF01260C
:10009000E4E700201FF0EAF80028DFD187F800A08D
:1000A000DCE700BF08B5012000F0E2FE21F0CAFE47
:1000B000F9E700BF08B5012000F0DAFE21F04EFE9E
:1000C000F9E700BF10B582B000F032FD02AC44F891
:1000D000040D2046012100F069FE00F029FD019B7E
:1000E000421F9A4288BF019021F028FFF1E700BF2C
:1000F00030B540F2281385B00024C2F2000304207A
:100100001C7001F09DFA46F6C463C2F20003186049
:10011000042001F095FA46F6CC63C2F200031860A1
:10012000042001F08DFA46F6C863C2F2000318609D
:10013000042001F085FA46F6C063C2F2000318609D
:10014000032240F2C5004FF650612346009201940D
:1001500002940394C0F6030102F5BA72C0F60100DE
:1001600000F0F2FA022540F2B5004FF65461234642
:100170000194029403940095C0F6030140F27712B3
:10018000C0F6010000F0E0FA012240F2A5004FF6AF
:100190005C6123460092019402940394C0F603012B
:1001A00002F5BB72C0F6010000F0CEFA40F2010089
:1001B0004FF6646100950194029403942346C0F6BF
:1001C000030140F27712C0F6010000F0BDFA2046AC
:1001D00005B030BD10B5044607F018FC40F22813F6
:1001E000C2F200031A784AB9A4B91A78022A08D1CF
:1001F00003221A7007F01EFC002010BD1A78022A94
:1002000003D007F017FC002010BD002CF9D1032209
:100210001A70EFE701221A7007F00CFC002010BDE5
:1002200040F22813C2F200031878831E5842584146
:10023000704700BF10B504461FF016F800280CBF29
:100240002D205520207000201FF010F800280CBF32
:100250002D204D206070FA201FF00AF800280CBFF6
:100260002D205220A070FA201FF004F8002398429D
:100270000CBF2D205720E0702371184610BD00BF21
:10028000F0B5012483B02746FF260025204602F062
:1002900037FAC0F3042367F301036FF3840301907B
:1002A0008DF805308DF804608DF8065020460199D0
:1002B000013402F015FA402CE8D1002003B0F0BD63
:1002C00010B582B000F034FC02AC44F8040D0121FA
:1002D000204600F06BFD00F02BFC019B421F9A4270
:1002E00088BF019041F64550C0F6030001F0CCFFF5
:1002F00041F64D50C0F6030002F06EFB05F0E8F841
:1003000021F0D8FCE3E700BF10B582B000F010FC8C
:1003100002AC44F8040D0121204600F047FD00F036
:1003200007FC019B421F9A4288BF019004F070FDB8
:1003300041F60550C0F6030004F016F921F0E0FC88
:10034000E9E700BF30B5002085B007F015FA0020BE
:1003500008F062FB002007F0EDF9002008F0F0F94A
:10036000002007F0A1FB002001F08CFE002001F02E
:1003700059FF002002F016F8002002F075F9002065
:1003800005F01CFC002008F075FB002005F012FCB5
:10039000002002F041FE002008F076FF002004F06B
:1003A0001FFF002005F05AF8002002F03BFB01205F
:1003B00002F0F0FB002010F0DDF8002002F0EAFB74
:1003C0002FF00AFC21F024FB02F0E6FC4FF4FA6463
:1003D0004FF47A7008F042FB013CF9D1032540F25A
:1003E000C12040F66C612346019402940394009569
:1003F000C0F6040140F27712C0F6010000F0A4F943
:1004000040F2093040F67461C0F6040140F2771200
:1004100023460095019402940394C0F6010000F075
:1004200093F900F095FA204605B030BD07F08CB97D
:1004300021F03EBC2DE9F04141F2597548F21F57B9
:10044000CDF2B715C5F2EB17012442F210764FF04A
:10045000640841F60550C0F6030004F085F8A5FBDA
:1004600004235B0B06FB13432BB908F07FF9C14350
:10047000012008F077F90134A7FB04235B0908FB8E
:100480001343002BE5D104F0C3FCE2E7F0B5D0F84C
:1004900000E0046947688668C56889B000F1140106
:1004A000CDF800E00EC9019740F6E460029603958E
:1004B0000494059148F6E474069207930699C0F6F1
:1004C0000404C0F6040003F039FE204603F036FEB3
:1004D00040F6FC60C0F6040003F030FE204603F056
:1004E0002DFE40F610700099C0F6040003F026FEC1
:1004F00040F61C700199C0F6040003F01FFE40F6A0
:1005000028700299C0F6040003F018FE40F634701B
:100510000399C0F6040003F011FE40F64070049900
:10052000C0F6040003F00AFE40F64C700599C0F6D0
:10053000040003F003FE40F658700699C0F604006C
:1005400003F0FCFD40F664700799C0F6040003F068
:10055000F5FD4EF63853CEF2000340F67070196880
:10056000C0F6040003F0EAFD4EF62853CEF2000375
:1005700040F680701968C0F6040003F0DFFD4EF607
:100580002C53CEF2000340F690701968C0F60400B8
:1005900003F0D4FD4EF63053CEF2000340F6A070C7
:1005A0001968C0F6040003F0C9FD4EF63C53CEF2C4
:1005B000000340F6B0701968C0F6040003F0BEFDF9
:1005C0006FF07F4002F01AFD002002F019FD0020BC
:1005D00002F0E0FA02F0D8FC0020014602F0E2FA54
:1005E00040F6C070C0F6040002F032FB012100208A
:1005F00002F0D8FA40F6D4700699C0F6040002F072
:1006000073FBFFF717FF00BF1EF0040F0CBFEFF3E3
:100610000880EFF30980FFF739BF704740F22410DC
:10062000C2F200002DE9F00FD0F800C00E4600E045
:100630002646344614F8015B0CEB0500407800F0C8
:10064000080000F0FF0B0028F2D12D2D67D02B2DD4
:1006500004BF7578B41C33F0100010D1D3F1010041
:1006600038BF0020302D03D048B10A239A4607E056
:10067000267806F0DF06582E56D000B108239A4699
:10068000BBF1000F0CBF6FF000494FF00049B9FB00
:10069000FAF800270AFB189938460CE04D45D4BFFC
:1006A00000260126404518BF0026EEB90AFB00507F
:1006B000012714F8015B0CEB0506767816F0040FA1
:1006C00018BF303D07D116F0030610D0012E14BF1D
:1006D00057263726AD1BAB4209DD404594BF0026A7
:1006E000012656EAD776D9D04FF0FF37E1E77B1CD9
:1006F00008D0BBF1000F10D10AB167B91160BDE895
:10070000F00F7047BBF1000F14BF4FF000406FF0C7
:100710000040002AF3D0611EF0E74042ECE7B41C31
:1007200075784FF0010B96E7102365789A460234EE
:10073000A6E700BF10B40C4613460146224600202F
:100740005DF8044BFFF76ABF2DE9F04F814683B097
:1007500048200E4693469A460C9FDDF834800E9D45
:1007600001F03AFB0446002800F0AF80002D00F0B5
:100770009E8005634FEA8B022846A5212FF06DFA73
:10078000206B0BF18042013A314600EB820B1022C4
:1007900004F134002FF006FB042F34BF3D4604253E
:1007A0000023261D84F84330E5626564304600F07E
:1007B000B5FD2BF0070B04F11800C5F1050500F09D
:1007C000ADFD5846A561246164624946524601F078
:1007D000E1F82060B8F1000F01D0C8F8004001F046
:1007E00009F940F22823C2F200031A6840F2D0153A
:1007F00001321A60C2F200052A68002A4AD040F28B
:100800003818C2F20008D8F8003040F26819C2F275
:1008100000098BB3E36A4FF0010A0AFA03FE40F2C3
:100820002C22C2F20002116840F2F8148B4288BFF9
:10083000136040F2F412C2F20002C2F20004106827
:100840003146266803EB830306EB0A0C4EEA0006EA
:1008500009EB8300C4F800C0166000F063FD01F0EE
:10086000D9F8D8F800301BB12B68DB6A9F420DD84D
:10087000504603B0BDE8F08F2B6840F26819DB6A80
:10088000C2F200099F4228BF2C60C3E701F0A2F822
:100890005046EEE72C601B6840F26819012B19D016
:1008A00040F23818C2F20009C2F20008B2E74FEA7B
:1008B0008B021046019201F08FFA019A2063002802
:1008C0007FF45BAF204601F00FFA4FF0FF3003B02A
:1008D000BDE8F08FC2F20009C84609F1640A40463B
:1008E00008F1140800F00EFDD045F8D140F2FC1BD1
:1008F000C2F2000B40F2102A5846C2F2000A00F081
:1009000001FD504600F0FEFC40F2D410C2F200009F
:1009100000F0F8FC40F24010C2F2000000F0F2FCDF
:1009200040F25410C2F2000000F0ECFC40F234122D
:1009300040F2F013C2F20002C2F2000340F2381893
:10094000C2F800B0C2F20008C3F800A062E700BF1E
:100950002DE9F047482001F03FFA0446002800F056
:100960008E8040F2DC5001F037FA2063002800F05E
:10097000D180A52140F2DC522FF06FF9206B40F6B8
:10098000E471C0F604011022002500F5BB66271DA6
:1009900004F134002FF006FA384684F84350E5623B
:1009A000656400F0BBFC04F1180000F0B7FC26F011
:1009B0000706052340F615712A46A3613046C0F6A6
:1009C00001012461646200F0E5FF206001F012F88B
:1009D00040F22823C2F200031A6840F2D016013216
:1009E0001A60C2F200063268002A4AD040F2381576
:1009F000C2F200052B6840F26818C2F200083BB949
:100A0000336840F26818DB6A03B93460C2F2000848
:100A1000E36A4FF0010C0CFA03FC40F22C22C2F204
:100A20000002116840F2F8148B4288BF136040F254
:100A3000F412C2F20002C2F20004D2F800E0394619
:100A4000276803EB830008EB80007B1C4CEA0E0751
:100A50002360176000F066FC00F0DCFF2B6803B138
:100A6000336800F0BFFF40F2EC1301212960C2F2AD
:100A700000030022BDE8F0471A6001F017B8BDE896
:100A8000F08734601B6840F26818012B06D040F2F2
:100A90003815C2F20008C2F20005B9E7C2F2000838
:100AA000454608F164092846143500F02BFC4D45F5
:100AB000F9D140F2FC1AC2F2000A40F21029504665
:100AC000C2F2000900F01EFC484600F01BFC40F298
:100AD000D410C2F2000000F015FC40F24010C2F247
:100AE000000000F00FFC40F25410C2F2000000F0D1
:100AF00009FC40F2341240F2F013C2F20002C2F2DA
:100B0000000340F23815C2F800A0C2F20005C3F895
:100B100000907DE72046BDE8F04701F0E5B800BF52
:100B200040F2CC13C2F200031A6801321A60704717
:100B300010B500F05FFF40F2EC13C2F200031C6836
:100B400000F068FF204610BD2DE9F04F40F2CC13B5
:100B5000C2F200031B6883B0002B40F0908040F28B
:100B6000EC15C2F200052B6801332B602B68002BBB
:100B70005FD040F23002C2F20002019213462968AF
:100B80001A6840F2EC13914238BF40F23014C2F2BE
:100B9000000338BFC2F2000446D340F23417C2F259
:100BA00000073A681268002A36D03A68D268D468DA
:100BB0001A686368934278D840F2F41640F26818D5
:100BC000C2F20006C2F200084FF00109BA4607E07F
:100BD000DAF80030DB68DC682A686368934264D81E
:100BE00004F1040B584600F0C9FBA36A04F1180095
:100BF0000BB100F0C3FBE06A336809FA00F200EBC6
:100C000080001343594608EB8000336000F08AFBF4
:100C10003B681B68002BDBD1019A4FF0FF3340F299
:100C200030141360C2F2000423681BB303B0BDE8A4
:100C3000F08F40F2341340F2F011C2F20003C2F21E
:100C4000000118680C6840F2E8121C60C2F2000251
:100C500008601168013111601A681268CAB940F25F
:100C60003003C2F200030193019A4FF0FF33136087
:100C7000134684E703B0BDE8F04FFFF7D7BB40F25F
:100C80003014C2F20004236801332360FFF7CEFB67
:100C9000CAE71B6840F23002DB68C2F20002DB6880
:100CA00001925B681360134669E7019A40F23014C1
:100CB0001360C2F20004B7E72DE9F84F00F09AFE86
:100CC00040F2CC13C2F200031A68013A1A601A68A3
:100CD000002A4ED140F22823C2F200031B68002BE9
:100CE00047D040F2D417C2F2000740F2F41640F2A7
:100CF000681940F2D0189246BB46C2F20006C2F212
:100D00000009C2F2000821E0DBF80C30DC68251D88
:100D100004F1180000F032FB284600F02FFBE06AD7
:100D2000012202FA00FE336800EB80004EEA030362
:100D3000294609EB8000336000F0F4FAD8F800305F
:100D4000E16ADB6A994228BF4FF0010A3B68002B39
:100D5000DAD140F23014C2F200042368A3B9BAF128
:100D6000010F14D040F22423C2F200031A68012AB2
:100D700011D0002400F04EFE2046BDE8F88FFFF7AA
:100D8000E3FE2368013B23602368002BF7D140F288
:100D90002423C2F20003002201241A6000F01AFE8C
:100DA00000F038FE2046BDE8F88F00BF40F2CC13BB
:100DB000C2F200031A6870B5013240F2EC141A60F6
:100DC000C2F20004036822685D18934207D9AB425F
:100DD00007D80560FFF770FF00283AD070BDAB421E
:100DE00002D823689D42F4D940F2D016C2F2000620
:100DF00033680560181D00F0C1FA60B9336801213D
:100E0000DA6A40F2F41301FA02F2C2F2000319683E
:100E100021EA02021A603168226840F2D01395423A
:100E20004D60C2F2000318D340F23412C2F2000245
:100E300010681968043100F083FA40F23003C2F2FE
:100E400000031A68954238BF1D60FFF735FF002880
:100E5000C4D1BDE8704000F0BDBD40F2F012C2F256
:100E6000000210681968043100F06AFAB2E700BFA6
:100E700070B518B9BDE8704000F0ACBD40F2CC13BD
:100E8000C2F200031A6840F2EC15013240F2D014AD
:100E90001A60C2F20005C2F200042E6823680644FC
:100EA000181D00F06BFA60B923680121DA6A40F27C
:100EB000F41301FA02F2C2F20003196821EA0202F5
:100EC0001A6021682A6840F2D01396424E60C2F23E
:100ED000000315D340F23412C2F200021068196800
:100EE000043100F02DFA40F23003C2F200031A6818
:100EF000964238BF1E60FFF7DFFE0028BAD070BDF3
:100F000040F2F012C2F2000210681968043100F0D9
:100F100017FAF0E72DE9804840F2401640F23C1500
:100F200040F2282283B0C2F20006C2F2000540F26D
:100F3000CC1440F26819C2F20002B246A846C2F2CE
:100F400000040192C2F2000906E023680133236025
:100F50003768FFF7B1FE5FB92B68002BF5D1D9F8E0
:100F60000030012B01D900F035FDFFF761FAF3E7FE
:100F700000F040FDDAF80C30D3F80CB00BF10400AF
:100F800000F0FCF9019A1368013B1360D8F80030B7
:100F9000013BC8F8003000F03DFDDBF8300000F008
:100FA000A3FE584600F0A0FED6E700BF40F2CC13E7
:100FB000C2F200031B680BBB40F2F413C2F2000341
:100FC0001B68B3FA83F3DBB2C3F11F0340F268126C
:100FD000C2F2000203EB830302EB83035A6803F1BE
:100FE000080152688A425A6004BF52685A60D26847
:100FF00040F2D013C2F200031A60704740F224237B
:10100000C2F2000301221A60704700BF38B540F2F7
:10101000D014C2F2000423680D4603F1180100F059
:101020008FF92068043000F0A9F960B92368012124
:10103000DA6A40F2F41301FA02F2C2F2000319680C
:1010400021EA02021A606B1C2BD040F2EC13C2F2B0
:101050000003186821681A682C1840F2D0139442D3
:101060004C60C2F2000311D340F23412C2F200020B
:1010700010681968043100F063F940F23003C2F2DD
:1010800000031A68944238BF1C6038BD40F2F01269
:10109000C2F2000210681968BDE83840043100F05F
:1010A0004FB9216840F254100431C2F20000BDE88B
:1010B000384000F037B900BFF8B5C368DC6804F108
:1010C0001805284600F05AF940F2CC13C2F200038A
:1010D0001B682BBB261D304600F050F9E56A01273E
:1010E000AF4040F2F413C2F20003186840F26812F5
:1010F00005EB8505C2F20002314647EA000602EB25
:1011000085001E6000F00EF940F2D013C2F2000319
:101110001B68E06ADB6A984234BF00200120F8BDFA
:1011200040F2D4102946C2F2000000F0FBF8EBE7D1
:1011300040F2E81240F2EC13C2F20002C2F20003E5
:1011400012681B6880E80C00704700BF70B50D4640
:10115000044600F04FFC2868421C08BF002522D03E
:1011600040F2E812C2F20002116823688B4240F29A
:10117000EC13C2F2000308BF616803D01E68616807
:10118000B14214D91E6840F2EC13761AB042C2F292
:1011900000030CD91E681268801B1B68014429607B
:1011A00084E80C00002500F035FC284670BD0125C0
:1011B00000F030FC284670BD40F22423C2F2000348
:1011C00001221A60704700BF40F2D013C2F2000340
:1011D00018687047F8B50546D8B140F2D014C2F28D
:1011E00000042268C36AD26A934212D2226840F293
:1011F0006816D16A03EB8303C2F20006426906EB6C
:101200008303C1F105019A42816103D02368DB6A3F
:10121000C362F8BD071D384600F0B0F818BBEB6A92
:1012200003EB83029200B258EAB90121994040F2DF
:10123000F413C2F200031A6822EA01021A6022685B
:101240004FF0010CD26A1C680CFA02FC02EB82001F
:10125000EA624CEA0402394606EB80001A60BDE8F7
:10126000F84000F05FB840F2F413C2F20003E6E782
:101270002DE9F041044600283DD0C26A436C9A42F1
:1012800039D0061D304600F079F8F0B140F268150B
:1012900040F2F412C2F20005C2F20002636C4FF099
:1012A000010808FA03F8D2F800C0C3F1050703EB00
:1012B0008300E362314648EA0C03A76105EB800036
:1012C000BDE8F041136000F02DB8E36A40F2681504
:1012D00003EB83029200C2F20005AA586AB9012208
:1012E00002FA03F340F2F412C2F20002116821EA9A
:1012F00003031360D2E7BDE8F08140F2F412C2F2BA
:101300000002CBE700F108034FF0FF3100228160BB
:101310004360C36003610260704700BF0023036144
:10132000704700BF43685A688B604A605A68916092
:10133000596003684160013308610360704700BF72
:1013400010B40C68631C08BF03690AD0C26800F1BE
:1013500008031268944204D35B685A681268944286
:10136000FAD25A685DF8044B4A6091608B6059600C
:101370000368086101330360704700BF42688168F9
:10138000036910B4916081685C684A601A6884429D
:1013900008BF5960013A002101611A6018685DF8C0
:1013A000044B70472DE9F04F044685B001929A46F0
:1013B000894600F1240600F1100500F01BFBA26B2A
:1013C000E36B4FF0000B9A42D8464FF0FF3763D3E0
:1013D0000198002800F0B880BBF1000F71D000F038
:1013E00019FBFFF79DFB00F005FB636C013308BFA1
:1013F000C4F84480A36C013308BFC4F8488000F0EF
:1014000009FB02A801A9FFF7A1FE002840F0A38074
:1014100000F0F0FAA26BE36B9A4256D000F0FAFAB1
:1014200000F0E8FAA36C002B06DC0FE0A36C013B94
:10143000A364A36C002B09DD636A3BB13046FFF760
:101440003BFE0028F2D0FFF7B7FEEFE7A76400F0FD
:10145000E1FA00F0CFFA636C002B06DC0FE0636C5E
:10146000013B6364626C002A09DD23693BB12846B5
:10147000FFF722FE0028F2D0FFF79EFEEFE7676439
:1014800000F0C8FAFFF718FC00F0B4FAA26BE36BA7
:101490004FF0010B9A429BD2226C002A40F09F80B1
:1014A0002568002D00F0C680A36B0133A363636A37
:1014B000002B40F0A68000F0ADFA012005B0BDE899
:1014C000F08F02A8FFF734FE89E700F0A3FA284660
:1014D0000199FFF79BFD00F08DFAA36C002B06DC51
:1014E0000FE0A36C013BA364A36C002B09DD636ACE
:1014F0003BB13046FFF7E0FD0028F2D0FFF75CFE7D
:10150000EFE7A76400F086FA00F074FA636C002B32
:1015100006DC0FE0636C013B6364636C002B09DD48
:1015200023693BB12846FFF7C7FD0028F2D0FFF73B
:1015300043FEEFE7676400F06DFAFFF7BDFB00289C
:10154000A2D100F047FA9FE7009000F063FA0098FC
:1015500005B0BDE8F08F00F04DFAA36C002B14DD50
:10156000636A93B104F1240507E0A36C013BA36413
:10157000A36C002B09DD636A3BB12846FFF79CFD95
:101580000028F2D0FFF718FEEFE74FF0FF33A36417
:1015900000F040FA00F02EFA636C002B14DD236992
:1015A00093B104F1100507E0636C013B6364636C65
:1015B000002B09DD23693BB12846FFF77DFD00289C
:1015C000F2D0FFF7F9FDEFE74FF0FF33636400F06F
:1015D00021FAFFF771FB002005B0BDE8F08F494606
:1015E000BAF1000F17D1A0682EF02CFBA168236C74
:1015F00062680B449342A360FFF456AF2368A36074
:1016000052E704F12400FFF757FD01287FF453AFA0
:1016100000F0E0F94FE7E0682EF014FB236CE2687D
:101620005B4221681A448A42E2603EBF62689B18AE
:10163000E36039E76068FFF71BFE656034E700BFD1
:1016400038B54C2000F0C8FB0446C8B100254FF067
:10165000FF3301228563C263436445608364056090
:101660008560C56005641030FFF74CFE04F124006E
:10167000FFF748FE204629462A462B46FFF792FEF2
:10168000204638BD38B545680446FFF79DFD8542C4
:1016900001D0002038BDE1680139E16009B10120C5
:1016A00038BD20460A460B46FFF77CFE012038BDB8
:1016B0002DE9F04F044685B099468A46019200F123
:1016C000240500F1100600F095F9A36B4FF0000B14
:1016D000D8464FF0FF37002B6CD10198002800F05E
:1016E000D680BBF1000F00F0BD8000F093F9FFF74A
:1016F00017FA00F07FF9636C013308BFC4F8448027
:10170000A36C013308BFC4F8488000F083F902A835
:1017100001A9FFF71BFD002840F0C08000F06AF926
:10172000A36B002B6DD100F075F92368002B00F03E
:10173000A68028460199FFF769FC00F05BF9A36CCD
:10174000002B06DC0FE0A36C013BA364A36C002B11
:1017500009DD636A3BB12846FFF7AEFC0028F2D0F2
:10176000FFF72AFDEFE7A76400F054F900F042F913
:10177000636C002B06DC0FE0636C013B6364626CFE
:10178000002A09DD23693BB13046FFF795FC0028AC
:10179000F2D0FFF711FDEFE7676400F03BF9FFF7C8
:1017A0008BFA002868D000F025F9A36B4FF0010BED
:1017B000002B92D02368E56853B1226C6068A918A9
:1017C0008142E160504624BFE36019462EF03AFAA8
:1017D000B9F1000F40F0A680A26B2368013AA26322
:1017E000002B00F0AF802369002B00F09E8004F1F5
:1017F0001000FFF761FC012840F0978000F0EAF844
:1018000093E000F007F900F0F5F8A36C002B06DC7C
:101810000FE0A36C013BA364A36C002B09DD636A9A
:101820003BB12846FFF748FC0028F2D0FFF7C4FC84
:10183000EFE7A76400F0EEF800F0DCF8636C002B33
:1018400006DC13E0636C013B6364636C002B0DDD0D
:1018500023695BB13046FFF72FFC0028F2D0FFF779
:10186000ABFCEFE702A8FFF763FC3EE7676400F01C
:10187000D1F8FFF721FA96E700F0ACF893E700F013
:10188000B9F86068FFF7A6FC00F0C4F851E70090D3
:1018900000F0C0F8009805B0BDE8F08F00F0AAF89D
:1018A000A36C002B14DD636A93B104F1240507E0F7
:1018B000A36C013BA364A36C002B09DD636A3BB1FD
:1018C0002846FFF7F9FB0028F2D0FFF775FCEFE799
:1018D0004FF0FF33A36400F09DF800F08BF8636CC9
:1018E000002B14DD236993B104F1100507E0636C4C
:1018F000013B6364636C002B09DD23693BB128461F
:10190000FFF7DAFB0028F2D0FFF756FCEFE74FF0C5
:10191000FF33636400F07EF8FFF7CEF9002005B0D6
:10192000BDE8F08F636AE5602BB900F073F8012021
:1019300005B0BDE8F08F04F12400FFF7BDFB0028DF
:10194000F3D05BE7FFF740FC60604CE770B545689B
:1019500004460E46FFF738FC85420BD000210B46AB
:1019600032462046FFF7A4FE012802BFE368013398
:10197000E36070BDE36801200344E36070BD00BF15
:1019800003480068006880F3088862B600DF00BF83
:1019900008ED00E010B400234FF0807440F8044CD0
:1019A00040F8081C40F8202C40F80C3C5DF8044B33
:1019B00040387047064B19680868B0E8F00F80F3AC
:1019C00009884FF0000080F311884EF00D0E70472B
:1019D000D00100204EF60453CEF200034FF08052A7
:1019E0001A607047EFF311804FF0BF0181F3118847
:1019F0007047002008B5FFF7F5FF40F23403C2F24C
:101A000000031A6801321A6008BD00BF80F3118814
:101A1000704700BF40F23403C2F200031868013877
:101A2000186000B17047FFF7F1BF00BFEFF3098006
:101A30000C4B1A6820E9F00F10602DE908404FF0B8
:101A4000BF0080F31188FFF7B1FA4FF0000080F378
:101A50001188BDE8084019680868B0E8F00F80F305
:101A600009887047D001002008B54EF60453CEF225
:101A700000034FF080521A60FFF7B4FFFFF764F8DD
:101A8000BDE808400020FFF7C1BF00BF4EF21402BE
:101A900041F63F114EF21003CEF20002C0F20101F6
:101AA000CEF2000307201160186070474EF62053F5
:101AB000CEF200031A6810B542F47F021A601A6869
:101AC000002442F07F421A60FFF7E0FF40F2340347
:101AD000C2F200031C60FFF753FF204610BD00BF99
:101AE0002DE9F04F46F6D065C2F20005002487B01C
:101AF0008A4646F6DC680590C2F20008FFF710F847
:101B00002C606C60AC605046BAF1000F40F09180E0
:101B1000B8F80010C1F30E014F007B1838F82320ED
:101B20000C46C2F30E03002B6DD046F6D066C2F20F
:101B3000000623E071883289C4EB030901314A446D
:101B400007EB040C7180328108EB8C0BBAF1000FAB
:101B500036D109EB49018900584602F043FB3C4469
:101B600038F82440E888C4F30E0467003B1938F8BD
:101B700023202146C2F30E03002B44D0B5F800E029
:101B8000591A89B208440EF1010E1204E880A5F832
:101B900000E0CFD5B28870890132014407EB040917
:101BA000B280718108EB8909BAF1000F15D1059B4C
:101BB0004B45D4D1FFF780F8059807B0BDE8F08F0A
:101BC000BBF8022041F23C008DE80402594622464F
:101BD000C0F6040002F0B2FABBE7B9F80610B9F893
:101BE00002C0B9F804E01A1B41F208000391019207
:101BF000CDF800C0CDF808E049462246C0F6040002
:101C000002F09CFAD3E76B8900F2554003F255438A
:101C1000401A46F6D066591AE8806981C2F2000679
:101C2000BAF1000F27D1FFF747F8002007B0BDE851
:101C3000F08F40F6EC7046F6DC68C2F20008C0F6A1
:101C4000040002F07BFAB8F80030B8F80610B8F8D3
:101C50000270B8F80460C3F30E0341F20800039168
:101C600022460193009702964146C0F6040002F016
:101C700065FAE8884CE704EB440108EB81014F88E2
:101C80008D88CA88C4F58A63053341F2080003923F
:101C900001932246009702950023C0F6040002F04B
:101CA0004DFA41F2600031887288B388C0F60400B2
:101CB00002F044FA41F29C00F18832897389C0F63F
:101CC000040002F03BFA3289738902EB420203EB13
:101CD000430341F2D80092009B0043F2FC31C0F66E
:101CE000040002F02BFA9EE7F8B50446002862D003
:101CF000FEF716FF46F6DC63C2F200034AF6AB229B
:101D0000E01ACAF6AA22A2FB0010C0F3CF004400DA
:101D10002518AD00595B01EB410292009F5E9E18B1
:101D2000002F21DB0444A4001D196E8846F6DC62F6
:101D300006EB4606B6009B5FC2F20002002B3BDBBF
:101D40009388002103EB430602EB8606F080AB800C
:101D5000E9809080135B6FEA43436FEA5343135368
:101D6000BDE8F840FEF7A8BFF188B78801EB410154
:101D700003EB81018F80B188F68801EB410103EB11
:101D80008101CE80995AC1F30E0199525A5B02EB40
:101D9000420233F82220C2F30E0202EB420203EBAE
:101DA000820250805A5B02EB420233F82210C1F3E8
:101DB0000E015953B6E7F8BD6FEA41416FEA514150
:101DC0009153135B698803EB430302EB8302518059
:101DD000BDE8F840FEF770BF2DE9F0410746002846
:101DE00000F0A380FEF79CFE082F81BF4AF6AB23CC
:101DF000A7F10901CAF6AA23A3FB012146F6DC6775
:101E0000C2F2000788BFC908B7F804E086BF0231F4
:101E100089B2012147F6FF727346002412E037F8B9
:101E20002640C4F30E04E41AA4B294422CBF002549
:101E300001258C4238BF0025002D18BF9E4618BFD3
:101E40002246034603EB430607EB860080881D46C7
:101E50000028E4D147F6FF739A4214BF7546224624
:101E60004FEA450404EB05064FEA860637F806807C
:101E700046F6DC63C8F30E0808BFAE46B819C2F2D6
:101E80000003B8F1000F28D08A4250D0511A89B20D
:101E90000D4405EB4505AA00981823F80280A0F828
:101EA00002E09A5B8E441FFA8EFEC2F30E0202EB32
:101EB00042026FEA4E4103EB82026FEA5141A2F8FF
:101EC00002E075464FEA4E049953254407EB850717
:101ED000FEF7F2FE381DBDE8F081481940F253428A
:101EE000904237DCBEF1000F06D1012215461A8060
:101EF0009A809646881802246619B600BA19D388C3
:101F0000714403EB43031FFA81FC00EB400007EB35
:101F10008301A1F804C007EB800307CA83E8070028
:101F200027F806C0A3F802E0CFE7BDE8F081C28839
:101F3000818802EB420203EB820291808288C18891
:101F400002EB420203EB8202D1809A5BC2F30E02E3
:101F50009A53BAE741F218102A46C0F6040002F07C
:101F6000EDF8FEF7A9FE4046BDE8F081FEE700BFB0
:101F7000684620F007018D4601B50D4B0D4898428B
:101F800007D2C243134423F0030204320A492DF05E
:101F900059FE0A480A4B984207D2C243134423F021
:101FA0000302043200212DF058FEFEF7CBF9FEE7C4
:101FB0002801002000000020807E05082801002064
:101FC00040C00020704700BFF8B50021012440F256
:101FD0003623C2F200030A46204640F235251C7023
:101FE000C2F2000506F050FA20462246002106F013
:101FF0004BFA95F800C0BCF1000F18D04AF2D82176
:102000004AF21C524AF2FC40C2F20001C2F2000243
:10201000C2F200000023CE5CD45CC75C7C40344339
:10202000CC54C45CE4B2D45401336345F3D140F2E0
:102030003023C2F200031B6803B1984740F23423F7
:10204000C2F200031B78DBB140F23723C2F2000377
:102050001A78AAB12D78013A1A708DB100234AF28C
:10206000D8214AF21C521E46C2F20001C2F20002FE
:10207000D05CCC5C6040D054CE540133AB42F7D13D
:10208000F8BD00BFF8B500286BD140F2302240F215
:102090003523C2F20003C2F2000220264AF2FC25D8
:1020A0004AF21C5E4AF2FC474AF2D821044610600C
:1020B0001E70C2F200050346C2F2000EC2F2000713
:1020C000C2F20001FF202A192B5582F8203082F835
:1020D000403082F8603082F8803082F8A03082F898
:1020E000C03082F8E03082F8003182F8203182F886
:1020F000403182F8603182F8803182F8A03182F874
:10210000C03182F8E0310EF8040038550B55013427
:10211000202C4FF00006D6D1012040F2342540F2A9
:1021200037244AF2F823C2F2000302463146C2F2D3
:102130000005C2F200041E702E70267006F0A4F98D
:102140000321012005F06CFF03210622012006F087
:10215000BFF840F23623C2F2000301221A70304663
:10216000F8BD4FF0FF30F8BD40F23523C2F2000356
:102170001878704740F23423C2F200031A7840F214
:102180003723C2F200031A7000207047F0B540F206
:102190003525C2F200052B7883B00746002B3DD0D1
:1021A00040F23623C2F200031A78002A33D000240A
:1021B00040F2302621462246C2F2000601201C7061
:1021C000376006F061F901202146024606F05CF90D
:1021D0004AF2F823C2F20003197841F6C9700131BE
:1021E000C9B20F2994BF19701C702B784AF2FC25D4
:1021F00088BF2146C0F60100C2F200054AF2FC4247
:10220000009005EB4111C2F20002012006F0C6F970
:10221000002003B0F0BD6FF00100FAE74FF0FF308F
:10222000F7E700BF10B490B94AF21C524AF2D82323
:102230000446C2F20002C2F20003FF2111541C54F2
:1022400001302028FAD100205DF8044B70474FF090
:10225000FF30F9E770B504460D46FFF785FFA04251
:1022600001D8002070BD05F0D1FB4AF2D823C2F29C
:1022700000031E5D1A5D2E4022EA05051D5505F07E
:10228000D9FB304670BD00BF2DE9F84F8146FFF7FE
:102290006BFF8246002800F08180B9F1000F7DD0ED
:1022A00000244AF2D8274AF21C58A346C2F200077B
:1022B000C2F20008072604E00134544506F108067E
:1022C0002ADAFFF751FF8442F6D205F09FFB3D5D0D
:1022D0003B5DEDB207F804B005F0ACFB002DEBD090
:1022E000E90752D4AA0747D46B073CD4280731D456
:1022F000E90626D4AA061BD46B0610D4ED09DBD060
:1023000018F804103046C9090134C847FFF732FFF6
:10231000544506F10806D4DB0020BDE8F88F18F814
:102320000410701EC1F38011C847FFF723FFE5E7D3
:1023300018F80410B01EC1F34011C847FFF71AFF88
:10234000DAE718F80410F01EC1F30011C847FFF7D0
:1023500011FFCFE718F80410301FC1F3C001C847C0
:10236000FFF708FFC4E718F80410701FC1F38001DD
:10237000C847FFF7FFFEB9E718F80410B01FC1F314
:102380004001C847FFF7F6FEAEE718F80410E0007A
:1023900001F00101C847FFF7EDFEA3E74FF0FF3062
:1023A000BDE8F88F50BB01464AF2FC200B46C2F252
:1023B0000000435442180131202982F8203082F86D
:1023C000403082F8603082F8803082F8A03082F8A5
:1023D000C03082F8E03082F8003182F8203182F893
:1023E000403182F8603182F8803182F8A03182F881
:1023F000C03182F8E031DCD1002070474FF0FF306F
:10240000704700BF2DE9F04F85B004460F46FFF737
:10241000ABFEE608864280F0CC80F643E4434AF205
:10242000FC2504F0070406444FF00108C2F2000541
:1024300008FA04F8741905F0E9FA002F6DD0AA5DC6
:102440005FFA88F31A43AA5594F8802194F88080A3
:1024500094F820B043EA080894F840A0009294F859
:10246000A021CDF80480DDF8008043EA0B0B43EA9D
:102470000A0A039294F8609043EA080294F8A0C014
:1024800094F8C0E094F8E07094F8006194F820515A
:1024900094F8400194F86011DDF80C8084F820B0C5
:1024A00084F840A094F8C0B194F8E0A143EA090987
:1024B000CDF8089043EA0C0C43EA0E0E1F431E436E
:1024C0001D431843194343EA080943EA0B0B43EA47
:1024D0000A03DDF8088084F8A0C084F86080DDF885
:1024E000048084F8C0E084F8808084F8E07084F888
:1024F000006184F8205184F8400184F8601184F868
:10250000802184F8A09184F8C0B184F8E03105F00E
:1025100091FA002005B0BDE8F08FAA5D6FEA0803CC
:10252000DBB21A40AA5594F8802194F8808094F880
:1025300020B003EA080894F840A0009294F8A02183
:10254000CDF80480DDF8008003EA0B0B03EA0A0AE9
:10255000039294F8609003EA080294F8A0C094F8FB
:10256000C0E094F8E07094F8006194F8205194F879
:10257000400194F86011DDF80C8084F820B084F8F4
:1025800040A094F8C0B194F8E0A103EA0909CDF89D
:10259000089003EA0C0C03EA0E0E1F401E401D407B
:1025A0001840194003EA080903EA0B0B03EA0A037F
:1025B0008FE74FF0FF30ADE738B504460D46FFF723
:1025C000D3FDA0422CD941F23C13E243C0F60403F0
:1025D0004AF2FC245B5D1044C2F200040219235449
:1025E00082F8203082F8403082F8603082F8803003
:1025F00082F8A03082F8C03082F8E03082F80031F2
:1026000082F8203182F8403182F8603182F88031DE
:1026100082F8A03182F8C03182F8E031002038BD64
:102620004FF0FF3038BD00BF0F2870B504460D468F
:10263000164613D8FFF798FDA84212D941F23C1371
:10264000ED43C0F6040328449A5D4AF2FC2300EBF4
:102650004414C2F200031A55002070BD6FF001004F
:1026600070BD4FF0FF3070BD2DE9F001A0BB4AF204
:1026700040584AF24062C2F20008C2F2000212F868
:10268000301002EBC00341F00F016FF3041102F8A8
:10269000301018F820C0DF785E789D781C79597961
:1026A0006FF3070C07F0F00708F820C001306FF354
:1026B00007176FF307066FF307056FF307046FF350
:1026C00003014028DF705E709D701C715971D6D176
:1026D0000020BDE8F00170474FF0FF30F9E700BF80
:1026E0003F289DBF4AF24053C2F2000343F8201036
:1026F0004FF0FF3098BF002082B002B0704700BF9B
:102700003F2882B08BBF01234AF240530022C2F21D
:10271000000383BF00928DF80130009B53F82030F6
:102720001846019302B070473F2838B504460D465D
:1027300012D805F06BF94AF24063C2F2000313F8B5
:102740003400024660F3830265F3010203F834208B
:1027500005F070F9002038BD4FF0FF3038BD00BFE4
:102760002DE9F04F4AF21C524AF2405583B0C2F2B2
:1027700000054AF240644AF2D82AC2F2000205F586
:102780008076C2F20004C2F2000A01924FF0FF0C00
:102790004FF0030B18E095F80180013F4FEA5818FD
:1027A00008F006090BFA09F12278FFB21AF80700BF
:1027B0001346C9B262F38303084223706BD1043518
:1027C000B54204F1080459D02B78002BF7D0A37838
:1027D0000BB1013BA370AF78002FDCD12278C2F39C
:1027E000810302F003094B45E9D002F00F03012BEE
:1027F000297847D0072B48D00E2B49D0082B7FD102
:102800000806DCD5D20602D4A278E02AD7D8FF2960
:1028100000F0BA802179A2782778501A1428CCBF0A
:10282000143111466A78C8BFC9B247F01007C8BF53
:10283000A17012F0030027704DD002285CD1C2F3C2
:10284000820201F0C000C2F1070230FA02F294F9EC
:10285000010008BF0122821A6FF045008242B8BF12
:1028600002466270E278043563F30302B5422171D7
:1028700084F802C0E27004F10804A5D1002003B07E
:10288000BDE8F08FCF06BDD499E78806BAD496E7A5
:102890004F06B7D493E73846CDF800C0FFF7DAFC0F
:1028A000DDF800C0002899D0019A18F0010FD35D1F
:1028B00043FA09F909F003091EBF4FEA490303F07F
:1028C000020343EA5909237869F30103DAB223705A
:1028D000C2F3810387E76079C2F38202D24300F03A
:1028E0000F00801842BF627802F1FF326270627995
:1028F00060F303026271B5E76278013A6270B1E792
:10290000022B37D1CF077FF55AAFD20603D5A27875
:10291000E02A3FF654AFFF2952D0A17820792278DF
:102920000F1A142F6FF30412C8BF00F114012270A4
:102930006A78C4BFC9B2A17012F003002FD0022878
:1029400029D1C2F3820201F0C000C2F1070230FABD
:1029500002F294F9010008BF01220244462AA8BFEE
:1029600046226270E278217163F3071284F802C094
:10297000E27024E70B2B02D18807C6D41FE70D2B8A
:1029800023D14F07C1D41AE7E27802F00F029A422E
:102990007FF440AF13E7627801326270E2E760795A
:1029A000C2F38202013200F00F0010440F28C2BFB0
:1029B000627801326270627960F303026271D1E77A
:1029C000E278B3EB121FA8D1F9E6042B7FF4F7AE3F
:1029D00008077FF5F4AE98E7F8B50746F8B14AF274
:1029E0004066C2F20006002408E05A7005F022F8A2
:1029F000204669B20134B847402C0ED005F006F8E5
:102A000006EBC4035D782A466FF30702002DECD174
:102A1000013405F00FF8402CF0D10020F8BD4FF044
:102A2000FF30F8BD70B500286ED14AF64404C2F2FA
:102A3000000441F2F0222346C0F6040207CA03C391
:102A40004FF47F511A80C0F600010B78422B21D140
:102A500043F6C173C0F600031A7843F6C2732270BE
:102A6000C0F600031A7843F6C3736270C0F6000321
:102A70001A7843F6C473A270C0F600031B78FF2BCC
:102A800008BF4FF48073A38043F6C573C0F60003FC
:102A90001B78E3804AF650034FF48041C2F20003F2
:102AA000C5F2144140F23822C2F20002002419603B
:102AB0004CF25030948005F0D1FF20460DF05AFDC5
:102AC000002823DB0EF056F94AF656064AF64E0267
:102AD0004AF654034AF64005C2F20002C2F200036D
:102AE000C2F20006C2F200052146204614801C8076
:102AF00034802C800EF0BCFA2046214634802C8095
:102B00000EF038FA204670BD4FF0FF3070BD00BFA8
:102B100010B44AF64404C2F2000441F2F022234603
:102B2000C0F6040207CA03C34FF47F511A80C0F6EF
:102B300000010B78422B21D143F6C173C0F600038C
:102B40001A7843F6C2732270C0F600031A7843F66F
:102B5000C3736270C0F600031A7843F6C473A270A0
:102B6000C0F600031B78FF2B08BF4FF48073A380CF
:102B700043F6C573C0F600031B78E38000205DF8C0
:102B8000044B70474AF64403C2F2000393F9000075
:102B9000C00F704740F24423C2F2000318700020B7
:102BA000704700BF40F23823C2F2000330B44AF647
:102BB00054024AF64E049D88C2F20004C2F200029A
:102BC0002080118095B19C79EDB200FB05F501FBE9
:102BD00004F44AF656024AF64003C2F20002C2F278
:102BE000000315801C8030BC0EF042BA0824062574
:102BF000EBE700BF4AF656024AF64003C2F2000273
:102C0000C2F20003108019800EF0B4B94AF65003E6
:102C1000C2F200031A1D011D824288BF99428CBF77
:102C20000022012210F0030F14BF002202F0010263
:102C30001AB1026800201A60704702781A70427850
:102C40005A7082789A70C2780020DA70704700BF9C
:102C50002DE9F047047884B0002C3DD04AF64409B1
:102C60004AF64E0840F238250746C2F20009C2F281
:102C70000008C2F2000500260FE020460DF09CFE81
:102C80000028A9BFB8F80030064301330643A8BFA7
:102C9000A8F8003017F8014FFCB199F9002001ABFA
:102CA000002AEADAAA88E2B1B5F806C0B5F808E069
:102CB0004FEADC0A0EFB0AFA95E807000AFB040457
:102CC00083E80700ADF80AC00194ADF80CE093E882
:102CD00007000EF0AFFCD3E72646304604B0BDE84F
:102CE000F0874FF0FF36D5E70FB42DE9F04794B0E9
:102CF0001CAB53F8041B04A81A46009307F0FAFD16
:102D00009DF81040002C3DD04AF644094AF64E0882
:102D100040F2382504AFC2F20009C2F20008C2F244
:102D2000000500260FE020460DF046FE0028A9BF52
:102D3000B8F80030064301330643A8BFA8F80030B6
:102D400017F8014FFCB199F9002001AB002AEADA2B
:102D5000AA88F2B1B5F806C0B5F808E04FEADC0A77
:102D60000EFB0AFA95E807000AFB040483E8070053
:102D7000ADF80AC00194ADF80CE093E807000EF03E
:102D800059FCD3E72646304614B0BDE8F04704B0FE
:102D900070474FF0FF36D3E72DE9F04F4AF6540263
:102DA00089B0C2F2000240F244234FF000090292BF
:102DB000C2F200034AF6560083F80090C2F2000007
:102DC000029B0090A3F800904AF64E04009B4AF63E
:102DD0004002C2F20002C2F2000448464946019293
:102DE000A4F80090A3F80090A2F800900EF040F92B
:102DF00040F2382AC2F2000A41F2C8264AF64407D5
:102E00000390D046C0F60406C2F200074D250FE03D
:102E100028460DF0D1FD0028A9BF238840EA090902
:102E2000013340EA0909A8BF238016F8015F05B302
:102E300097F9002005AB002AEADABAF80420002A44
:102E400076D0B8F806C0B8F808E04FEADC0B0EFB05
:102E50000BFB98E807000BFB050583E80700ADF8BE
:102E60001AC00595ADF81CE093E807000EF0E2FBF0
:102E7000D1E70398BAF8042049EA000B029801212F
:102E800040F2382325800180C2F20003002A55D089
:102E90009B79019A4FF000091380009B484601215D
:102EA000A3F800900EF0E4F841F2DC2840F2382656
:102EB0004BEA000BCDF800B0C0F60408C2F20006E1
:102EC00028250FE028460DF077FD0028A9BF2388AC
:102ED00040EA0909013340EA0909A8BF238018F82C
:102EE000015FFDB197F9002005AB002AEADABAF8D4
:102EF000042002B3B6F806C0B6F808E04FEADC0BCF
:102F00000EFB0BFB96E807000BFB050583E80700AB
:102F1000ADF81AC00595ADF81CE093E807000EF077
:102F200089FBD2E7009B43EA090009B0BDE8F08FB6
:102F30004FF0FF3979E74FF0FF39D0E70823A8E7D2
:102F400038B505460024E0B22946013408350EF0B4
:102F50000BF910B9082CF6D138BD4FF0FF3038BD51
:102F600030B4827840F238230432C2F2000305788C
:102F70004478C178104401229A7218609D80DC80E8
:102F80000020198130BC70470DF0F4BEF0B54AF650
:102F90004403C2F2000393F9003085B0002B0446CD
:102FA0000DDB0DF009FD0028A1BF4AF64E03C2F269
:102FB00000031A880132A8BF1A8005B0F0BD40F2A4
:102FC0003823C2F200039A884FF0FF30002AF4D071
:102FD000DE881D89F70805FB07F793E8070001ABBA
:102FE00004FB070483E80700ADF80A600194ADF81C
:102FF0000C5093E807000EF01DFBD4E70EF012BB57
:103000000EF014BB84B001AB83E8070093E807001F
:1030100004B00EF00FBB00BF2DE9F04104460028BC
:103020007AD140F2390C40F23A0E40F2502740F289
:10303000482640F2782540F27C2140F2682240F296
:103040005423C2F20001C2F20002C2F20003C2F233
:10305000000CC2F2000E4FF01008C2F20006C2F2DD
:103060000005C2F200070860106018608CF800804C
:103070008EF8008030602860386006F0B9FBC50F1C
:10308000204602F02FFA00284FF00000B8BF45F0AC
:10309000020502F083FD00284FF00000B8BF45F0A4
:1030A000040502F06BFD40F26023C2F200031E78BB
:1030B00000284FF0000140F2582040F25A2261F3FC
:1030C0000706C2F20000C2F2000243F6D0741E707E
:1030D00001701170C0F600042378B8BF45F00805F0
:1030E000422B10D040F27021C2F2000100220023D6
:1030F000C1E9002340F25C24C2F2000400266842C9
:103100002680BDE8F08143F6D173C0F600031B783A
:10311000190658BF1370E5E74FF0FF30BDE8F081A6
:1031200010F0F0030CD101280BBF40F23A0340F23B
:103130003903C2F20003C2F20003187800F0F00372
:10314000202B14D00BD9302B05D0502B0DD100F0F3
:103150000F0002F017BD00F00F0002F023BD102B8E
:1031600003D100F00F0006F081BB0020704700F093
:103170000F0002F0EDB900BF10F0F00FF8B50446F3
:103180000D460AD101280BBF40F23A0340F2390341
:10319000C2F20003C2F200031C7840F24823C2F2DC
:1031A00000031B6804F00F06F7B22BB167F3071595
:1031B00029462046984778B904F0F004202C20D006
:1031C0000BD9302C15D0502C10D167F30715284699
:1031D000BDE8F84002F0DABCF8BD102C06D167F368
:1031E00007152846BDE8F84006F050BB4FF0FF3009
:1031F000F8BD67F3071529463046BDE8F84002F0F0
:10320000D5BC67F3071529463046BDE8F84002F003
:10321000D9B900BF41F0B001F8B50D09002465F33C
:10322000030461F30F2462F3174410F0F00F054616
:1032300063F31F640AD101280BBF40F23A0340F246
:103240003903C2F20003C2F200031D7840F24823A2
:10325000C2F200031B6805F00F06F7B22BB167F34B
:10326000071421462846984770B905F0F005202D2F
:103270001DD00AD9302D13D0502D0ED167F307146D
:10328000204602F083FCF8BDF8BD102D05D167F390
:103290000714204606F0FAFAF8BD4FF0FF30F8BDEB
:1032A00067F307142146304602F080FCF8BD67F34F
:1032B00007142146304602F085F9F8BD2DE9F04F9C
:1032C00085B0904600900F46002A00F0858040F2BD
:1032D0003903C2F20003029340F23A03C2F2000340
:1032E0000393009B40F2482903F0F003C2F2000967
:1032F0000193002524E0009B012B0CBF039B029B44
:103300001E78D9F8003006F00F0B5FFA8BFA2BB15C
:103310006AF3071421463046984768B906F0F0066C
:10332000202E46D03DD9302E4FD0502E48D16AF3B2
:103330000714204602F02AFC002843DB45454BD207
:10334000C5EB0803022B1FD0032B15D0012B22D075
:10335000AB1C7A19FB5C5278795D0420033560F36D
:10336000030461F30F2462F3174463F31F64019BAA
:10337000002BC0D0009EC4E7AB1C7A19795DFB5CC2
:10338000527807200335EAE76B1CFA5C795D00236D
:1033900002350620E3E70023795D1A460520013552
:1033A000DDE7102E0CD16AF30714204606F06EFA02
:1033B000C2E76AF307145846214602F003F9BBE757
:1033C0004FF0FF3005B0BDE8F08F6AF307145846A0
:1033D000214602F0EBFBAFE7002005B0BDE8F08F1F
:1033E0002DE9F04F0423002563F303056FF00F036D
:1033F00063F30F256FF3174510F0F00783B0044611
:10340000894690466FF31F6518BF83460BD101288C
:103410000BBF40F23A0340F23903C2F20003C2F29A
:10342000000393F800B040F24826C2F20006336869
:103430000BF00F0A5FFA8AF23BB162F307150092B4
:10344000294658469847009AA8B90BF0F00BBBF1F3
:10345000200F00F0D18053D9BBF1300F00F0C480B1
:10346000BBF1500F40F0B58062F30715284602F01B
:103470008DFB824600E082460422002540F25A235A
:1034800062F30305C2F200037E2262F30F251B786C
:10349000322262F3174563F31F65A3465FB9012C1F
:1034A0000BBF40F23A0340F23903C2F20003C2F20A
:1034B000000393F800B033680BF00F025FFA82FC50
:1034C0004BB16CF307158DE8041029465846984710
:1034D0009DE8041020BB0BF0F00BBBF1200F00F0B7
:1034E0009E806BD9BBF1300F14D0BBF1500F78D157
:1034F0006CF30715284602F049FB40EA0A0A11E07E
:10350000BBF1100F65D162F30715284606F0BEF92E
:103510008246B1E76CF307152946104602F046FBD8
:1035200040EA0A0A0423002563F303050D2363F32D
:103530000F2569F3174568F31F6557B9012C0BBFB9
:1035400040F23A0340F23903C2F20003C2F2000330
:103550001C78336804F00F06F7B22BB167F3071538
:10356000294620469847C0B904F0F004202C4BD0DF
:1035700018D9302C0BD0502C2ED167F307152846C4
:1035800002F004FB40EA0A0003B0BDE8F08F67F3E5
:1035900007152946304602F009FB40EA0A0003B04D
:1035A000BDE8F08F102C17D167F30715284606F0F9
:1035B0006DF940EA0A0003B0BDE8F08FBBF1100FCF
:1035C0000FD16CF30715284606F060F940EA0A0AA5
:1035D000A8E74FF0FF3A4FE74FF0FF3003B0BDE8E8
:1035E000F08F4FF0FF3A9DE762F3071550462946EA
:1035F00002F0DCFA82463FE762F30715504629469F
:1036000001F0E0FF824637E767F3071529463046A9
:1036100001F0D8FF40EA0A0003B0BDE8F08F6CF378
:1036200007152946104601F0CDFF40EA0A0A79E75E
:103630002DE9F04F87B09146029088461746002A40
:1036400069D040F24823C2F20003019340F23903EB
:10365000C2F20003049340F23A03C2F200030022D4
:10366000059300F0F0031546174603933EE04244ED
:10367000517803F07F0300293CD0927801F07F015C
:10368000002A38D002F07F02042060F3030463F3C1
:103690000F2461F3174462F31F64039A6ABB029B11
:1036A000012B0BBF059A049B16781E78019A06F031
:1036B0000F0B13685FFA8BFA2BB16AF307142146DC
:1036C0003046984708BB06F0F006202E33D026D9A6
:1036D000302E14D0502E2BD16AF30714204602F05E
:1036E00055FA07430335A9452A4614D918F802307C
:1036F000002BBCD100210022C6E7029ED6E76AF368
:1037000007145846214602F051FA0335A94540EA0C
:1037100007072A46EAD8384607B0BDE8F08F102ED2
:1037200006D16AF30714204606F0B0F80743D9E73C
:103730004FF0FF37D6E76AF307145846214601F0E9
:1037400041FF0743CEE700BFF8B50523002463F32C
:1037500003046FF0080363F30F246FF3174410F0B2
:10376000F00F05466FF31F640AD101280BBF40F22A
:103770003A0340F23903C2F20003C2F200031D789B
:1037800040F24823C2F200031B6805F00F06F7B2AF
:103790002BB167F3071421462846984770B905F006
:1037A000F005202D1DD00AD9302D13D0502D0ED16B
:1037B00067F30714204602F0E9F9F8BDF8BD102DB3
:1037C00005D167F30714204606F060F8F8BD4FF006
:1037D000FF30F8BD67F307142146304602F0E6F9E2
:1037E000F8BD67F307142146304601F0EBFEF8BD43
:1037F0002DE9F04F89B080462CF08DFA0426002583
:103800006FF00F0366F3030540F23A0963F30F25E7
:10381000C2F2000999F800A06FF3174598F800204C
:103820006FF31F652946074650460192FFF7A4FC37
:1038300040F25A237E21C2F200031B7861F30F2568
:10384000322161F3174563F31F65294683465046CD
:10385000FFF792FC0D2363F30F25019A402363F3D6
:10386000174562F31F6540EA0B0B29465046FFF7E8
:1038700083FC012F4BEA000BCDF818B098BF99F8E4
:10388000000063D999F8003000250293029B013FA4
:1038900003F0F003049340F2390340F2482AC2F2E5
:1038A0000003039708F101082F462A46C2F2000AD6
:1038B0000593CDF81C9018F80230002B5CD04244E0
:1038C000517803F07F03002956D0927801F07F01F0
:1038D000002A4ED10022042060F3030463F30F2476
:1038E000049B61F3174462F31F64002B46D1029BD3
:1038F000012B0CBF079B059B1E78DAF8003006F001
:103900000F0B5FFA8BF933B169F307142146304688
:10391000984700283AD106F0F006202E41D037D93A
:10392000302E2DD0502E44D169F30714204602F0DA
:103930002DF90743039B0335AB422A46BBD8069BB0
:10394000DDF81C903B4399F8000006930523002105
:1039500063F303016FF0080363F30F216FF3174163
:1039600021F07F41FFF708FC069B184309B0BDE832
:10397000F08F02F07F02AEE70021ABE7029EBCE7CA
:1039800069F307145846214602F010F90743D1E7BE
:10399000102E0ED169F30714204605F077FF074378
:1039A000C8E769F307145846214601F00BFE0743A8
:1039B000C0E74FF0FF37BDE72DE9F04340F24C245C
:1039C000C2F200042378ABB005460F2B00F2A080B2
:1039D000DFE803F0949E9E9E9E9E9E9E9E9E9E9ECF
:1039E0009E733E4240F23804C2F200042378002B5A
:1039F00000F06281012B05D140F25423C2F2000392
:103A00001B682BBB40F25A23C2F2000393F80080DC
:103A100028464FF0F00C00234FF07E0E32270E2682
:103A20001025F7240AA909228DF82D808DF828C0C9
:103A30008DF829308DF82A308DF82BE08DF82C7018
:103A40008DF82E608DF82F508DF83040FFF736FC42
:103A500000202BB0BDE8F083002900F08B80012905
:103A600000F0888040F26023C2F200035B68002B04
:103A7000EED140F25A22C2F2000292F800C04FF09A
:103A8000F00E7E273226F72428460AA90F250922A0
:103A90008DF829308DF82A308DF82F308DF82DC013
:103AA0008DF828E08DF82B708DF82C608DF82E5055
:103AB0008DF83040FFF702FCCAE7002969D00129E0
:103AC00090D140F23803C2F200031978FF2908BFF1
:103AD0001A70BDD0002900F032810129B8D140F21E
:103AE0005423C2F200031C68002CB1D040F25823CA
:103AF000C2F2000311461878A047A9E7002942D076
:103B000001294DD140F25923C2F200031A709FE7F8
:103B100040F25A23C2F2000393F800804FF0F00CF9
:103B20000E234FF07E0E284632270025F7260AA9DD
:103B300009228DF82E308DF82F308DF82D808DF8DC
:103B400028C08DF829508DF82A508DF82BE08DF87B
:103B50002C708DF83060FFF7B1FB40F26023C2F2A9
:103B600000031A78002065F3070225701A702BB045
:103B7000BDE8F08340F26023C2F2000300205960E8
:103B80002BB0BDE8F08340F25923C2F20003197054
:103B90005EE740F23803C2F20003FF221A7057E7D3
:103BA00040F25923C2F200031B78052B00F06D810F
:103BB00045D9082B00F0FE8000F2CA80062B00F0E9
:103BC0003181072B40F01E8103F0FAFE49F61021E7
:103BD0000246C0F60401684606F07AFE40F25A2317
:103BE000C2F200031E787E2000233221F0240F222F
:103BF0008DF829308DF82A308DF82B008DF82C1097
:103C00008DF82D608DF828408DF82E200DF1FF33B2
:103C10000DF163000DF12F0103E0834201F8012B48
:103C200003D013F8012F002AF7D10A46F72302F830
:103C3000013B0AA92846521AFFF740FB08E7022B6E
:103C400000F07A8140F28C80032B00F04D81042B30
:103C500040F0D88003F0A6FE40F6DC710246C0F6C4
:103C60000401684606F034FE40F25A23C2F2000313
:103C70001E787E2000233221F0240F228DF8293077
:103C80008DF82A308DF82B008DF82C108DF82D60D2
:103C90008DF828408DF82E200DF1FF330DF16300D3
:103CA0000DF12F0103E0834201F8012BBDD013F881
:103CB000012F002AF7D1B8E740F25A22C2F20002DF
:103CC00092F800904FF07E0C4FF0320E4FF0F0085B
:103CD0000F27F72628460AA909228DF829308DF8E2
:103CE0002A308DF82F308DF82D908DF828808DF8A2
:103CF0002BC08DF82CE08DF82E708DF83060FFF71A
:103D0000DDFA2378002B7FF4A3AE40F26823C2F2E1
:103D100000031B68002B7FF49BAE40F23A04C2F212
:103D20000004267841F26C30012DC0F6040018BF63
:103D30002570FFF75DFD012E18BF267088E640F262
:103D40006823C2F200031C68002C7FF4CFAE7FE62C
:103D5000092B00F019817F2B54D103F0CDFD77E6BC
:103D6000012B4FD140F25A23C2F200031878AC4B1A
:103D700000220F21F0277E2632248DF82D008DF8A9
:103D80002E1003F164008DF828708DF829208DF82D
:103D90002A208DF82B608DF82C400DF12F0104E0C6
:103DA000834201F8012B3FF440AF13F8012F002AA2
:103DB000F6D13AE740F25A23C2F200031878994B41
:103DC00000220F21F0277E2632248DF82D008DF859
:103DD0002E1003F164008DF828708DF829208DF8DD
:103DE0002A208DF82B608DF82C400DF12F0104E076
:103DF000834201F8012B3FF418AF13F8012F002A7A
:103E0000F6D112E740F25A23C2F2000393F8008081
:103E100028464FF0F00C00234FF07E0E32270E267E
:103E20000D25FEE503F0C4FD49F610210246C0F65B
:103E30000401684606F04CFD40F25A23C2F200032A
:103E40001E787E2000233221F0240F228DF82930A5
:103E50008DF82A308DF82B008DF82C108DF82D6000
:103E60008DF828408DF82E200DF1FF330DF1630001
:103E70000DF12F0104E0834201F8012B3FF4D5AE90
:103E800013F8012F002AF6D1CFE6684603F09CFD17
:103E900040F25A230028C2F20003C0F29D801E782F
:103EA0007E2000233221F0240F228DF829308DF856
:103EB0002A308DF82B008DF82C108DF82D608DF8A0
:103EC00028408DF82E200DF1FF330DF163000DF128
:103ED0002F0104E0834201F8012B3FF4A6AE13F852
:103EE000012F002AF6D1A0E640F25A23C2F20003C5
:103EF00018784D4B00220F21F0277E2632248DF8B2
:103F00002D008DF82E1003F164008DF828708DF8C7
:103F100029208DF82A208DF82B608DF82C400DF18A
:103F20002F0104E0834201F8012B3FF47EAE13F829
:103F3000012F002AF6D178E640F25A23C2F200039C
:103F400018783A4B00220F21F0277E2632248DF874
:103F50002D008DF82E1003F164008DF828708DF877
:103F600029208DF82A208DF82B608DF82C400DF13A
:103F70002F0104E0834201F8012B3FF456AE13F801
:103F8000012F002AF6D150E640F25A23C2F2000374
:103F90001878274B00220F21F0277E2632248DF837
:103FA0002D008DF82E1003F164008DF828708DF827
:103FB00029208DF82A208DF82B608DF82C400DF1EA
:103FC0002F0104E0834201F8012B3FF42EAE13F8D9
:103FD000012F002AF6D128E61878164B00220F216F
:103FE000F0277E2632248DF82D008DF82E1003F157
:103FF00064008DF828708DF829208DF82A208DF81E
:104000002B608DF82C400DF12F0104E0834201F864
:10401000012B3FF40AAE13F8012F002AF6D104E673
:104020005F130408C7120408431304084F1304085D
:10403000DB12040867130408F729F8B50B4621D8EA
:1040400040F26024C2F200042178C1F3C001D9B962
:10405000A0F11102D2B2062A1DD940F25822C2F2B2
:1040600000021070D1B11E0652D4227840F26024B2
:10407000C2F30015C2F20004002D3BD01A46012104
:10408000FFF79AFC0020F8BD40F25822C2F200026D
:1040900012788242DCD04FF0FF30F8BD207840F239
:1040A000602100F00702042AC2F2000110D9052A9B
:1040B00038D02378013202F0070262F30203052AA6
:1040C0002370DFD92378002043F008032370F8BD64
:1040D00041F26041C0F60401895C9942E9D022783E
:1040E00040F24C236FF30702C2F20003002022705B
:1040F0001870F8BD40F24C2642F01007C2F20006DC
:104100001A46294627703370FFF756FC2846F8BD3B
:10411000F72BE4D12278D506E1D51A460221FFF724
:104120004BFCDCE740F25A22C2F2000212789A42BB
:10413000D5D1062363F302000870C3E70FB430B58E
:10414000A3B0269C20462BF0E6FD64283CD827AB84
:1041500021461A4602A8019306F0CCFB02A82BF0D8
:10416000DAFD48B38208002A18BF03284FEA820309
:104170008CBF0024012432D901A94D68013405F017
:104180007F35A24241F8045FF7D81A4602A990424F
:104190000B4411D01C78511C04F07F0488421C7021
:1041A0000AD95978023201F07F019042597003D93F
:1041B0009A7802F07F029A7002A8FFF719FB23B0E9
:1041C000BDE8304004B0704741F2BC30C0F6040096
:1041D000FFF70EFB23B0BDE8304004B0704700226B
:1041E00002ABD7E72DE9F04F834697B00846002988
:1041F0005ED00BF1FF350D44AB455CD248F2F84779
:1042000041F210464FF00009C0F60407C0F604065C
:10421000CDF804B005F101085C46019B41F218415C
:10422000C0F6040102A8E21A06F052FB04F1100ADB
:104230000DF1110BAC428CBF3946314614F8012BFD
:10424000584606F045FB54450BF1030BF2D14FF0F5
:1042500020038DF841308DF84230544611AA0AF1FE
:104260000100AAF10F0313F8011C9646A1F1200CDE
:104270005FFA8CFCBCF15F0F88BF2E21434502F82A
:10428000011C03F1010302F1010201D09842EAD1BD
:104290004FF00A038EF800304FF0000302A88EF8AA
:1042A0000130FFF7A5FAAA4549EA0009B5D3484607
:1042B00017B0BDE8F08F0020FAE700BF2DE9F04FFE
:1042C00001F00F0707F1080303F00F030E46062B5A
:1042D00083B09046C1F30729C1F307454FEA116B3C
:1042E00082466FF3071606D80AB13146C047002050
:1042F00003B0BDE8F08FB9F1F00F05D007F10C0362
:1043000003F00F03032B13D840F27023C2F2000313
:10431000D3E9000150EA01020AD10AF0F001302984
:1043200000F0F880502900F0E880102900F0868025
:10433000BB1E0D2BDBD801A252F823F07B430108F2
:104340007B43010875430108854301088B4301083D
:104350008B430108EF420108EF420108EF420108D8
:10436000EF420108EF420108EF420108EF42010865
:1043700075430108B9F1F70F2CD9B8F1000FB6D089
:104380005046B2E7B9F1F70FF7D8043F17F0FF0234
:1043900061D140F2602493461746C2F200042378AC
:1043A000C3F3C003BBF1F70F0BD0002B9FD118F163
:1043B000000318BF0123002F18BF0023002B96D045
:1043C000DEE740F27022C2F2000200240025C2E9BA
:1043D0000045EAE750464946FFF72EFE0F2F07D06B
:1043E00029465046FFF728FE50465946FFF724FE5F
:1043F00040F26023C2F200031B781B073FF577AF42
:1044000040F27824C2F200042368002B00F0A88058
:104410004946504698470F2F814640F08F8010F054
:10442000FF0F14BF00230123B8F1000F0CBF0023BE
:1044300003F00103002B3FF45AAFA1E701210AF07A
:104440000F0401FA04F440F25C21C2F200010020E2
:104450001C8008806CE740F26024C2F200045046E1
:1044600049460192FFF7E8FD2378019A13F0080FFF
:1044700018BF00270AD140F27823C2F200031F6858
:1044800027B150464946B847019AC7B2012A69D9AF
:10449000504629460192FFF7CFFD2378019A13F089
:1044A000080F0BD140F27823C2F200031B682BB136
:1044B000504629469847019A3843C7B2022A36D057
:1044C00050465946FFF7B8FD237840F26024C3F305
:1044D000C003C2F200047BBB40F27822C2F20002A9
:1044E0001268002A3FF45EAF504659469047237841
:1044F0003843C7B2C3F3C00354E701210AF00F04E5
:1045000001FA04F440F25C21C2F2000100209C8018
:1045100008800DE701210AF00F0401FA04F440F2CB
:104520005C21C2F2000100205C80088000E7237853
:10453000AB46C3F3C00335E7012333E729462368BD
:10454000504698472368074659465046984738438F
:1045500040EA090515F0FF0F14BF0023012363E7AC
:10456000012361E7CB461AE72DE9F04F40F26023C3
:1045700095B0C2F20003039340F2782240F25C232C
:1045800040F27029C2F20002C2F20003C2F2000936
:104590008346059204930AA805F032FA002869DBE5
:1045A0009DF828700A9C07F00F0505F1080303F039
:1045B0000F033F09062B07F110076FF307149DF84F
:1045C00029609DF82A809DF82BA040D9F02E05D0B7
:1045D00005F10C0303F00F03032B12D8D9E90001F6
:1045E00050EA01020DD107F00F03012101FA03F394
:1045F000049A4FF00000108040F27020C2F20000D8
:104600000380AB1E0D2BC6D801A151F823F000BFCB
:104610004F4601084F460108494601081347010863
:1046200017470108174701089745010897450108F2
:1046300097450108974501089745010897450108E6
:104640009745010849460108F72E40F2FF81BBF16A
:10465000000FA0D065F3030466F30F2468F317443A
:104660006AF31F6421463846D8470AA805F0C8F9FE
:10467000002895DA41F2FC24C0F604040AAD0FCC00
:104680000FC50FCC0FC594E8030085E803009DF823
:104690002860002E62D040F27C23C2F20003039314
:1046A00040F25823C2F20003049340F24C23002549
:1046B00040F26027C2F20003A8462C462A46C2F206
:1046C00000070593B24614A8024452F8243C0AF0AD
:1046D0000F0009A9984710F10A0F00F05081002837
:1046E00006DB504609995A4601350134FFF7E6FDCD
:1046F000092D08F1010831DC4FEAC80214AB13445C
:1047000013F8280C40BB4CB3804604460246B24620
:10471000D9E7F72E9BD82B1F13F0FF0C40F0D78161
:1047200040F260236146CDF818C0C2F200031B7846
:10473000C3F3C003F72900F04381002B7FF42BAFB4
:10474000069A1BF1000318BF0123002A18BF00239B
:10475000002B3FF420AF7DE78246B4E740F26022B1
:1047600040F27823C2F20002C2F2000303920693E1
:1047700040F2702240F25C23C2F20002C2F2000357
:10478000049205930AA801F005FA002866DB9DF85B
:1047900028700A9C07F00F0505F10803C7F30317FB
:1047A00003F00F035037062BFFB26FF307149DF889
:1047B00029609DF82A809DF82BA03CD9F02E05D0C9
:1047C00005F10C0303F00F03032B0FD8D9E9000107
:1047D00050EA01020AD107F00F03012101FA03F3A5
:1047E000059A4FF000001080049A9380AB1E0D2BA9
:1047F000C8D801A050F823F037480108374801080D
:1048000031480108394901083F4901083F49010879
:104810008547010885470108854701088547010844
:104820008547010885470108854701083148010887
:10483000F72E40F2CA80BBF1000FA3D065F303044A
:1048400066F30F2468F317446AF31F642146384661
:10485000D8470AA801F09EF9002898DA40F27021A2
:10486000D9E9002352EA0300C2F2000160D040F20D
:104870005C23C2F200031B88B3F57A7F58D90B88FA
:10488000002B00F0F581DD0700F16E829C0700F13E
:104890007182580700F16C82190700F16782DA060D
:1048A00000F16A829F0600F16B825E0600F166826B
:1048B0001D0600F16982DC0500F16482980500F1B3
:1048C0006982590500F164821A0500F15F82DF04F4
:1048D00000F162829E0400F161825D0400F1288291
:1048E000DB0B18BF0F2440F024821024204640F236
:1048F0006023C2F200031A78110707D540F258214D
:10490000C2F200010978814200F01A8240F27C2351
:10491000C2F200031B6803B1984741F220402146D0
:10492000C0F60400FFF70AFC00220023C9E90023B7
:10493000002015B0BDE8F08FF72E3FF67CAF2B1F9F
:1049400013F0FF0C40F0238140F260236146CDF864
:104950001CC0C2F200031B78C3F3C003F7292AD09E
:10496000002B7FF40FAF079A1BF1000318BF012340
:10497000002A18BF0023002B3FF404AF5EE73B780A
:104980001A070CD4039803680BB15046984741F2BC
:1049900020405146C0F60400FFF7D0FBA8E604997A
:1049A0000A78524501BF6FF307033B70059B002255
:1049B00008BF1A70E6E700200021C9E90001CFE72F
:1049C00000200021C9E90001B7E638463146FFF76B
:1049D00033FB0F2D07D041463846FFF72DFB3846F5
:1049E0005146FFF729FB039A13781B073FF5CAAE20
:1049F000069A1368002B00F09F813846314698478D
:104A00000F2D034613D0069841460268029338469C
:104A10009047069984460A683846CDF804C0514646
:104A20009047DDF804C0029B4CEA0000034313F0FA
:104A3000FF0F14BF00230123BBF1000F0CBF0023A5
:104A400003F00103002B3FF49DAEF7E638463146F4
:104A5000FFF7F2FA0F2D07D041463846FFF7ECFA80
:104A600038465146FFF7E8FA039A137819073FF5DD
:104A700092AD059A1368002B00F0608138463146EC
:104A800098470F2D034613D00598414602680293BC
:104A900038469047059984460A683846CDF804C0E0
:104AA00051469047DDF804C0029B4CEA00000343E6
:104AB00013F0FF0F14BF00230123BBF1000F0CBF45
:104AC000002303F00103002B3FF465ADC2E531463E
:104AD0003846CDF804C0FFF7AFFA039A40F26023DE
:104AE0001178C2F2000311F0080F18BF0022DDF8A0
:104AF00004C018BF06920DD105980268002A00F084
:104B0000E9800293384631469047029BC0B2DDF8F7
:104B100004C00690BCF1010F40F27881384641464E
:104B2000CDF804C0FFF788FA039ADDF804C01378C3
:104B300013F0080F0BD1059A136843B1384641466C
:104B40009847069BDDF804C01843C0B20690BCF13C
:104B5000020F7BD038465146FFF76EFA039A13785E
:104B6000C3F3C003002B7DD1059851460268002A8B
:104B70003FF4E0AD514638469047039A51461378CA
:104B8000069AC3F3C0031043C0B20690D2E5314683
:104B90003846CDF804C0FFF74FFA039A40F260237D
:104BA0001178C2F2000311F0080F18BF0022DDF8DF
:104BB00004C018BF07920DD106980268002A00F0C1
:104BC0008B800293384631469047029BC0B2DDF895
:104BD00004C00790BCF1010F40F2168138464146EF
:104BE000CDF804C0FFF728FA039ADDF804C0137863
:104BF00013F0080F0BD1069A136843B138464146AB
:104C00009847079BDDF804C01843C0B20790BCF179
:104C1000020F21D038465146FFF70EFA039A137857
:104C2000C3F3C0030BBB069851460268002A3FF449
:104C300095AE514638469047039A51461378079AE5
:104C4000C3F3C0031043C0B2079087E6039A4146FE
:104C50001378C3F3C0036DE5039A41461378C3F399
:104C6000C0037BE65146012364E55146012375E606
:104C70004A88002A32D0D4076DD4900700F1908082
:104C8000510700F19D80130700F19880D70600F1CD
:104C90009380960600F18E80550600F189801406F7
:104CA00000F18480D0057FD491057BD4530500F1B9
:104CB0008D80170500F18880D60400F1918095045D
:104CC00048D454047ED4D20B18BF0F2343D13024D0
:104CD00020460CE606921DE707927BE78C8820466B
:104CE000002C3FF404AEE0073AD4A10770D4620769
:104CF00072D423076ED4E70670D4A60676D4650670
:104D000072D420066ED4E1057CD4A20578D4630564
:104D100074D4270570D4E6046CD4A50468D4600468
:104D20001DD4E40B18BF0F221AD150242046DEE513
:104D30000E2410342046DAE501237DE60123BCE68B
:104D400040F24C216FF30702C2F2000100251A70F5
:104D50000D70DBE50D233033DCB22046C7E50E22B3
:104D60005032D4B22046C2E50024E2E70324E0E753
:104D70000224DEE70124DCE70424DAE70624D8E78E
:104D80000524D6E70824D4E70724D2E70B24D0E78C
:104D90000A24CEE70924CCE70C24CAE70D24C8E78F
:104DA0000123D8E70923D6E70823D4E70723D2E76E
:104DB0000623D0E70523CEE70423CCE70323CAE785
:104DC0000223C8E70E23C6E70B23C4E70A23C2E782
:104DD0000122C5E70322C3E70222C1E70422BFE79D
:104DE0000C23B8E70722BBE70622B9E70522B7E79D
:104DF0000D22B5E70C22B3E70B22B1E70A22AFE799
:104E00000922ADE70822ABE73146A4E531468EE43E
:104E100010B504F01FFE044600F0A0FB044300F0B0
:104E2000C3FE044300F0B0FE40F25C23C2F2000374
:104E30001A884FF6FF718A4218BF013244EA000017
:104E400018BF1A8010BD00BF40F24823C2F2000311
:104E500018600020704700BF40F25023C2F20003E8
:104E600018600020704700BF08B540F25023C2F21E
:104E700000031B680BB1984708BD184608BD00BF6A
:104E80002DE9F04140F25026C2F20006336882B0AC
:104E900080462BB341F2243201F00F00C0F6040229
:104EA000175CC1F30720C1F30742C1F307618DF816
:104EB00000008DF801208DF802103D4667B10025F5
:104EC0002C461DF80410404698470134A74245EA95
:104ED000000501DD3368F4E7284602B0BDE8F08143
:104EE000184602B0BDE8F08101281FBF40F23A0326
:104EF000C2F200031870002008BF4FF0FF30704767
:104F000040F23A03C2F200031878704740F25A2385
:104F1000C2F200031878704740F27823C2F200030F
:104F200018600020704700BF40F26823C2F20003FF
:104F300018600020704700BF40F25423C2F2000303
:104F400018600020704700BF40F27C23C2F20003CB
:104F500018600020704700BF2DE9F84F8946097A94
:104F60008346072992466ED81A68984692B39BF8F2
:104F70000040002C18BF2F2C0CBF0026012660D04B
:104F80002A2C2AD015782A2D27D0FDB10BF1010744
:104F90009446012607E02A2C21D01CF8015F2A2D17
:104FA0001DD0013695B1AC423B4602EB060103D061
:104FB0003F2C01D03F2D3CD117F8014B2F2C18BFAF
:104FC000002CE8D10B780120002B37D058F8102F97
:104FD000002ACCD10020BDE8F88F5B460026194698
:104FE00011F8013F01362F2B18BF002BF8D199F88B
:104FF000084009EB8401631CCA6089F80830D8F8BE
:105000000C10D8F808304AEA010123B14846984705
:1050100089F80840DAE7D8F80430002BF8D0701C83
:105020000A4658444946FFF797FF0028F0DABDE8E2
:10503000F88F61460B780020002BC7D10028D6D10D
:10504000C4E71146BEE76FF00300BDE8F88F00BF6C
:105050002DE9F00F067882B02C2E904600F0BC802F
:10506000421C0192002E00F08E80002900F08B80FF
:10507000002402E08A4204D01446621C855C002DA4
:10508000F8D1012A7FD0825C002A7CD12F2E7AD1E0
:10509000661D26F07F4626F00306B142C8F82C00B4
:1050A00071D9875D00EB06098D1B002F6BD015B9F8
:1050B00069E0AA4205D09246013219F80240002C5C
:1050C000F7D119F80250002D5DD12C2F5BD1771D3F
:1050D000574427F07F47BAF1080F28BF4FF0080A5E
:1050E00027F0030788F83050BAF1000F57D0B942C3
:1050F00049D38C46EAB2494619F801BF08EB0206CB
:10510000C41908EB820286F831B0D4634A780135BD
:10511000463A2E2A43D8DFE802F03042423042427B
:1051200042423042424242183042424242424230BF
:105130004230424242424E4C3C424C423C4C424243
:10514000424C424242424C183C00C25DC7EB0C0B41
:10515000CAB1BBF1000F16D0002602E05A4504D0B8
:105160001646721CA15C0029F8D1A25C5AB9053719
:10517000374427F07F4727F00307554588F830501C
:105180000DD0BC45B6D26FF0010002B0BDE8F00F03
:105190007047554507F1080788F83050F1D101985C
:1051A0000022414688F8082002B0BDE8F00FFFF762
:1051B000D3BE0437E1E76278C15D1204E67842EAC3
:1051C0000162A1783243073742EA0122174427F0EF
:1051D0007F4727F00307D0E76FF00200D5E700BF55
:1051E000003818BF6FF00000704700BF43780178A7
:1051F000C2781B0443EA01638078134343EA00202A
:10520000704700BF10B40A0C0C0E0B0AC17004707A
:10521000427083705DF8044B043070474178037826
:10522000C278090441EA0361837841EA020040EA56
:105230000320704710B40A0C0C0E0B0AC1700470E6
:10524000427083705DF8044B0430704710B504461B
:105250002AF00BFD0130031B9A0705D0002200F84D
:10526000012B031B9B07FAD110BD00BF43780178C7
:10527000C2781B0443EA01638078134343EA0020A9
:10528000704700BF04307047D31C23F00303F0B411
:105290001E0E1D0C1C0AC370067045708470031D21
:1052A000002A40D008300C1D814238BFA34234BFD1
:1052B0000020012041EA0304092A94BF002000F0E5
:1052C000010014F0030F14BF002000F0010078B3B8
:1052D00095080020AE0004460F580134AC421F5020
:1052E00000F10400F8D39C19B24201EB060008BF9C
:1052F00020460ED011F82570711C8A4203F82570E3
:1053000014D941780236B24261700FD98178981869
:10531000A1709407034606D0002403F8014B9918A6
:10532000091A8907F9D11846F0BC70479818F0E7B8
:10533000981811F8014B03F8014B8342F9D1E8E7C3
:1053400002780023110961F303036FF30713417817
:1053500062F30F23827861F3174362F31F631846E9
:10536000704700BFC1F3072201F47F0343EA0263E1
:10537000090E43EA012110B40A0C0C0E0023090A9D
:10538000047042708170C3705DF8044B0430704744
:105390002DE9F043884641F2684199B09146C0F644
:1053A0000401424607462AF0E3FC00283AD1B8F14E
:1053B0000F0F42D97A7B7B7A387B397AFC7A1204D8
:1053C000FD7B1B0442EA006243EA0163B87BB97AC1
:1053D00023432A4342EA002243EA01230192009335
:1053E0001024251DA8456A464B4607EB040607EB2B
:1053F00005001ED396F801C0395D4FEA0C4CF478D5
:105400004CEA016CB1784CEA040646EA01267419AC
:10541000A045314611D3002EE3D0FFF719FE002836
:10542000DFDA07E0002201238DE80C00B8F1000F5D
:1054300008D1002019B0BDE8F0834FF0FF3019B05B
:10544000BDE8F083384641464B466A46FFF700FE0A
:105450000028EEDA19B0BDE8F08300BF10B490B9AF
:1054600040F2802140F23B0240F23C031024C2F2A1
:105470000001C2F20002C2F20003086014701C7046
:105480005DF8044B70474FF0FF30F9E700B510F0BE
:10549000F00F83B08DF807100AD101280BBF40F23E
:1054A0003C0340F23B03C2F20003C2F2000318784F
:1054B0000309022B18BF4FF0FF3006D100F00F0098
:1054C0000DF10701012204F03DFD03B05DF804FB7E
:1054D00001235A1C042BD2B201D900207047134675
:1054E000F7E700BFF8B5044670BB40F28823C2F26C
:1054F000000340F2A02240F2842640F2A425C2F22A
:1055000000021860187158719871D8711881D860AC
:10551000187458749874D8749882FF27C2F20006E1
:10552000C2F20005177002F071FA37702C8002F099
:1055300081FA02F06BFA77706C8002F07BFA2046F9
:1055400004F006FCC017F8BD4FF0FF30F8BD00BFF7
:1055500001288CBF00200120704700BF08B502F071
:1055600055FA40F2A422C2F2000213884FF6FF71EE
:105570008B421CBF0133138040F28823C2F2000328
:1055800019894FF6FF7081421CBF01311981518882
:105590004FF6FF70814240F2A42218BF0131C2F2DF
:1055A000000218BF51809A8A4FF6FF718A4240F27A
:1055B0008823C2F200031CBF01329A8202F03AFA39
:1055C000002008BD2DE9F04FC1F307254FF0010879
:1055D000F72DC1F307464FEA116785B0044601F085
:1055E0000F0108FA00F832D9012832D841F22433E9
:1055F0000F29C0F6040300F08A80072900F33E81DA
:1056000040F2A42840F2842913F801A0C2F2000855
:10561000C2F200094FF0FF0BBAF1000F13D038F8B7
:1056200014208DF80850B2F57A7F8DF809608DF856
:105630000A7000F2A080204602A9524604F082FCC3
:10564000831CE9D028B9002005B0BDE8F08F0128FF
:1056500004D94FF0FF3005B0BDE8F08F41F224339C
:105660000729C0F604032ADD0F2940F0AB8040F281
:10567000A42840F2842993F80FA0C2F20008C2F2D5
:1056800000094FF0FF0B40F28423BAF1000FDAD08B
:1056900038F814208DF80850B2F57A7F8DF809603B
:1056A0008DF80A7098BFC2F200036FD8204602A995
:1056B00052461D5504F046FC831CC3D1E3E740F27B
:1056C000A42840F2842913F801A0C2F20008C2F213
:1056D00000094FF0FF0B40F28423BAF1000FB2D063
:1056E00038F814208DF80850B2F57A7F8DF80960EB
:1056F0008DF80A7098BFC2F200032BD8524620469C
:1057000002A91D5504F01EFC821C9BD1E3E740F268
:10571000A42840F2842993F80FA0C2F20008C2F234
:1057200000094FF0FF0BBAF1000F8CD038F81420AD
:105730008DF80850B2F57A7F8DF809608DF80A70FF
:1057400035D85246204602A904F0FCFB821C7FF4A7
:1057500079AFE8E7009302F059F9009B4FF000029F
:10576000C2F2000309F804B028F81420009302F0F4
:1057700061F9009BC2E702F049F94FF0000309F814
:1057800004B028F8143002F055F954E7009302F001
:105790003DF9009B4FF00002C2F2000309F804B08B
:1057A00028F81420009302F045F9009B7EE702F0F0
:1057B0002DF94FF0000209F804B028F8142002F087
:1057C00039F9BEE713F801B040F2A4290BF1FF3319
:1057D00040F2842ADBB20193C2F20009C2F2000A4D
:1057E000BBF1000F3FF42FAF39F814308DF808509B
:1057F000B3F57A7F8DF809608DF80A702CD840F2E5
:10580000A023C2F200031B7818EA030F16D0BBF1E5
:10581000010F40F283801AF8042040F28423AA4248
:105820001CBF002229F81420C2F2000311BF5A46FF
:105830008DF808608DF80970019A04E040F2842325
:10584000C2F200035A4602A920461D5504F07AFB15
:10585000811C7FF4F7AEC3E702F0D8F840F284234E
:105860000022C2F20003FF2129F814200AF80410D4
:10587000009302F0DFF85A46009BE4E713F801B00A
:1058800040F2A4290BF1FF3340F2A02ADBB20193CE
:10589000C2F20009C2F2000ABBF1000F3FF4D3AE1E
:1058A00039F814208DF80850B2F57A7F8DF8096028
:1058B0008DF80A7023D89AF8002018EA020F1CD03D
:1058C000BBF1010F98BF01220FD940F28422C2F22E
:1058D0000002125DAA421CBF002229F814200CD13C
:1058E000019A8DF808608DF8097002A9204604F02D
:1058F00029FB811C7FF4A6AECEE75A46F5E702F0FD
:1059000085F840F28422C2F20002FF2000211055E7
:1059100029F8141002F08EF85A46E6E740F2842384
:10592000C2F2000301228EE701282DE9F84F044658
:105930000F4603D94FF0FF30BDE8F88F40F28825BD
:1059400000EB4006C2F20005B60041F2584941F2B0
:10595000343A05EB060BC0F60409C0F6040A4FF012
:105960000008204604F0C2FA002858DB0106C2B243
:1059700030D49BF80410F02958D09BF80600A0BB47
:105980009BF805C0ABF8080063460CF1FF30C0B2CD
:10599000012B8BF8060030D0002839D101F0F0003F
:1059A000F0288BF8032000F08B80AA5D080960F3D3
:1059B0000302AA558BF80110AA593A609BF80620F9
:1059C00000202AB1BBF80820B2F57A7F00F2BA8035
:1059D000BDE8F88FF72A42D93878002140F00F004F
:1059E0007A703870B970F970E8E79BF805300138C3
:1059F000C0B2012B8BF80600CED18BF802208BF8B9
:105A000003800028ADD101F0F002F02ACDD15AE098
:105A10008BF80220204604F069FA0028A6DA9BF8E9
:105A200006204FF0FF30002AD2D0CBE79BF80710BA
:105A30000131C9B201298BF807104AD00229E7D0F9
:105A40008BF80320AA5D042161F30302AA55A9592A
:105A5000002239608BF80720ABF80820AEE7C2F3CC
:105A6000021119F801108BF804208BF8051011BBF6
:105A700000F00F001AF80000F02A8BF8050037D06C
:105A8000F72A41D0B0B9A95D052464F30301A955F3
:105A90008BF801208BF802008BF80300AA593A60BA
:105AA0009BF8052000208BF80620ABF80800002AA0
:105AB0008ED087E701468BF80610ABF8088050E7D8
:105AC00053B1012B0ED1AA5D022060F30302AA5547
:105AD00070E78BF8012044E7AA5D052060F303021C
:105AE000AA5567E7AA5D032060F30302AA5561E7A0
:105AF0004FF0010301468BF801208BF807308BF83B
:105B00000610ABF808802CE79BF8070050B301287B
:105B10000ED0A95D072060F30301A9558BF803207F
:105B2000AA5900213A609BF805208BF80710B9E7C5
:105B3000A85D062464F30300A8558BF802208BF8B7
:105B40000310EDE70022AA518BF804208BF8052002
:105B50008BF806208BF807206FF00900ABF80820BF
:105B6000BDE8F88FA95D052464F30301A9558BF8FE
:105B700001208BF802008BF80300D1E74FF0FF30D3
:105B8000704700BF00207047002070474FF0FF3083
:105B9000704700BF4FF0FF30704700BF4FF0FF303D
:105BA000704700BF00207047002070474FF0FF3063
:105BB000704700BF4FF0FF30704700BF4FF0FF301D
:105BC000704700BF10B5044648B9014602F028FAF4
:105BD00020460321072202F07BFB204610BD4FF038
:105BE000FF3010BDF8B5030606460C4617463BD4F9
:105BF00000200246014602F047FC3146002002F038
:105C0000A7FC210E002002F0A3FCC4F307410020F2
:105C100002F09EFCC4F30721002002F099FCE1B2DF
:105C2000002002F095FC3946002002F091FC4D2E38
:105C300018BF082423D00020FF2102F089FCFF2890
:105C4000054631D1013CF6D1FF21002002F080FC55
:105C500000200122014602F017FCFF21002002F083
:105C600077FC4FF0FF30F8BD77200021FF22FFF7CF
:105C7000B9FF012800DDF8BD06F07F06B8E7FF2177
:105C8000002002F065FCFF21002002F061FC0020F2
:105C9000FF2102F05DFCFF280546D5D00020FF2142
:105CA00002F056FC2846E6E7482E01D07A2EF5D1C0
:105CB000FF21002002F04CFCFF210506002002F02D
:105CC00047FCFF210646002002F042FCFF2104466B
:105CD000002002F03DFC45EA0645284340EA042541
:105CE000FF21002002F034FC2846F8BD002070B5EA
:105CF0000146012202F0C8FB00200321072202F026
:105D0000E7FA0A240020FF2102F022FC013CF9D12D
:105D100021462246204602F0B7FB4FF47A7002F08B
:105D20009DFE402021469522FFF75CFF051E35DBD6
:105D300040F2A826C2F2000648204FF4D57187220F
:105D40003470FFF74FFFB0F5D57F32D0E920214600
:105D5000FF22FFF747FF0128CCBF0120022030704F
:105D600004E013D0B4F5804F3DD03078022803BF53
:105D7000E9200021FF2241201CBF0021F922FFF76A
:105D800031FF0028054604F10104EADA50204FF4FF
:105D90000071F922FFF726FF337853B30020012268
:105DA000014602F071FBFF21002002F0D1FB2846E2
:105DB00070BD4FF4804401E0013C1AD0E9204FF05F
:105DC0008041FF22FFF70EFF05460028F4D17A201C
:105DD0002946FF22FFF706FF10F0804F0CBF042377
:105DE0000C233370DAE750204FF40071F922FFF7EB
:105DF000F9FE6FF00105D1E738B50446002833D12C
:105E00000321072202F064FA20462146012202F013
:105E10003BFB0A240020FF2102F09AFB601E10F0D9
:105E2000FF04F7D121462246204602F02DFB4020F8
:105E300021469522FFF7D6FE051E07DB21460122EB
:105E4000204602F021FBFFF751FF0546002001220A
:105E5000014602F019FBFF21002002F079FBD5F189
:105E6000010038BF002038BD03210122002002F0CC
:105E70002FFA00200146024602F006FB4D200021C9
:105E8000AF22FFF7AFFE0546E0E700BF70B540F276
:105E9000A823C2F200031B7804461A0758BF440225
:105EA00082B001220E460020032102F011FA2146A1
:105EB0005120FF22FFF796FE051E0CD02DDB00209F
:105EC0000122014602F0E0FAFF21002002F040FB2F
:105ED000284602B070BD4FF4803401E0013C1FD071
:105EE0000020FF2102F034FBC0B2FF28F6D00024CE
:105EF00032464FF4007321460094204602F04EFBD8
:105F00002046FF2102F024FB2046FF2102F020FB67
:105F10002046FF2102F01CFBD1E76FF0FF05CEE722
:105F20006FF48075CBE700BF70B540F2A823C2F2D2
:105F300000031B780E461907044682B058BF44027E
:105F400003210122002002F0C3F921465820FF223C
:105F5000FFF748FE051E0CD037DB0020012201466A
:105F600002F092FAFF21002002F0F2FA284602B075
:105F700070BDFE2102F0ECFA2A464FF40073314660
:105F80000095284602F00AFBFF21284602F0E0FABD
:105F9000FF21284602F0DCFA2846FF2102F0D8FA59
:105FA00000F00F00052818D14FF4001401E0013C67
:105FB0000ED00020FF2102F0CBFA10F0FF0FF6D038
:105FC000FF21002002F0C4FAC7E76FF0FF05C4E725
:105FD0004FF6FE65CFF6FF75BFE76FF48075BCE73F
:105FE0002DE9F04F032187B001220546002002F081
:105FF0006FF94A200021FF22FFF7F4FD061E0FD0A3
:10600000B8BF6FF0FF0600200122014602F03CFA03
:10601000FF21002002F09CFA304607B0BDE8F08F67
:106020004FF4803401E0013C58D00020FF2102F001
:106030008FFAC0B2FF28F6D0002402AA102321460E
:106040000094204602F0AAFAFF21204602F080FACE
:10605000FF21204602F07CFAFF21204602F078FA68
:106060009DF812009DF811909DF815209DF814B030
:1060700006AB00049DF8168053F80D1D9DF813A083
:1060800040EA09699DF809E09DF80A709DF817003B
:1060900049EA0B0995F810C002F00F0B1B7949EA89
:1060A0000A2A48EA0B2B9DF808909DF810804CEACC
:1060B000121C47EA0E27400801226C72C5F80CA09A
:1060C0002B726960A5F812B085F810C06F80287532
:1060D00085F8009085F80A806A7594E76FF48076F9
:1060E000AAE700BF2DE9F04F032187B00122054642
:1060F000002002F0EDF849200021FF22FFF772FD99
:10610000061E0FD0B8BF6FF0FF0600200122014627
:1061100002F0BAF9FF21002002F01AFA304607B067
:10612000BDE8F08F4FF4803402E0013C00F0E380E2
:106130000020FF2102F00CFAC0B2FF28F5D00024A5
:1061400002AA102321460094204602F027FAFF21DC
:10615000204602F0FDF9FF21204602F0F9F9FF2167
:10616000204602F0F5F99DF80CA09DF80D109DF861
:1061700008209DF80E304FEA0A1A4AEA111A01F077
:106180000F0B9DF809E091099DF80A709DF80B002E
:10619000C2F383094FEAD31802F00302C3F3801C51
:1061A000A5F806A085F808B0C3F3401AC3F3001B96
:1061B00001296C73297085F80190AA7085F809800F
:1061C00085F80AC085F80BA085F80CB085F803E0C7
:1061D0002F71687178D09DF810109DF811209DF8EE
:1061E0000F709DF81240880940EA870702F0030EFD
:1061F000E00903F0030347EA832340EA4E0EC1F3AC
:10620000C207500901F00701C2F382022B6185F831
:1062100018E02F756975A875EA759DF814209DF82A
:1062200015109DF813009DF816304FEA501C4FEAE8
:10623000911E04F0030A02F003099DF817704CEA5E
:10624000CA0A4EEA89094FEAD218C2F3411C00F08B
:106250001F00C4F38404C1F3401E4FEAD31BC2F3F2
:10626000820201F001017F08E87685F81AA0C3F3E5
:106270008010C3F3401A6C7685F81F90C3F30014A6
:10628000C3F3810985F81C8003F003034FF0000875
:1062900085F81DC04FF0010CAA7785F820E085F83D
:1062A000221085F823B085F8240085F825A085F80C
:1062B000264085F8279085F8283085F8297085F8DC
:1062C000218085F82AC020E79DF810009DF8112054
:1062D0009DF80F109DF8123042EA002201F00301F0
:1062E00042EA01411A012C756C75AC75EC75296197
:1062F0002A761C4691E76FF4807606E72DE9F04F89
:1063000040F2B423C2F2000301241D88002040F2B1
:10631000A92385B0C2F20003024621461C7002F098
:10632000B3F89E21002002F013F94021034600201B
:10633000019302F00DF92146844622460020CDF853
:1063400008C002F0A1F800200246214602F09CF8A5
:10635000BF21002002F0FCF803218346002002F058
:10636000F7F8214622468246002002F08DF80020F0
:106370000246214602F088F89F21002002F0E8F84A
:1063800081460020014602F0E3F82146224680467D
:10639000002002F079F800200246214602F074F84D
:1063A0004C21002002F0D4F8013D40F6FF76ADB25A
:1063B000B54228BF3546E9B20746002002F0C8F8CA
:1063C000214622460646002002F05EF800200246E2
:1063D000214602F059F84D21002002F0B9F8290AAF
:1063E0000390002002F0B4F8214605462246002022
:1063F00002F04AF8019BDDF808C04CEA030343EAC7
:106400000B0B4BEA0A0A4AEA090949EA080848EA72
:106410000707039B3E4346EA0300284305B0BDE857
:10642000F08F00BF2DE9F04F0646002093B00146E3
:10643000012201F04DFF00280390C0F2ED80737837
:106440003578B2781D43F378154332791D4373795B
:1064500015431D4300F0E380306840F2AC24C2F2E3
:1064600000042060B388A38000200246012102F0CE
:106470000BF8BF21002002F06BF8032184460020B6
:10648000CDF804C002F064F8012103460A4600205A
:10649000029301F0F9FF00200246012101F0F4FF10
:1064A0009F21002002F054F803218346002002F0CF
:1064B0004FF801210A468246002001F0E5FF002046
:1064C00002460121257801F0DFFF4421002002F07F
:1064D0003FF829460490002002F03AF801210A46CC
:1064E0000590002001F0D0FF0020024601216578D0
:1064F00001F0CAFF4521002002F02AF82946069043
:10650000002002F025F801210A460790002001F042
:10651000BBFF002002460121A57801F0B5FF422112
:10652000002002F015F829460890002002F010F82B
:1065300001210A460990002001F0A6FF0020024632
:106540000121E57801F0A0FF4321002002F000F8CE
:1065500029468146002001F0FBFF01210A468046C2
:10656000002001F091FF002002460121257901F071
:106570008BFF4021002001F0EBFF29460746002059
:1065800001F0E6FF01210A460646002001F07CFFEB
:10659000002002460121647901F076FF41210020AC
:1065A00001F0D6FF21460546002001F0D1FF012170
:1065B00004460A46002001F067FFDDF804C0029B94
:1065C0004CEA0303DDF80CC043EA0C0343EA0B0377
:1065D000DDF810C043EA0A0343EA0C03DDF814C0F7
:1065E00043EA0C03DDF818C043EA0C03DDF81CC0D5
:1065F00043EA0C03DDF820C043EA0C03DDF824C0B5
:1066000043EA0C0343EA090949EA080848EA07078C
:106610003E43354345EA040013B0BDE8F08F0AA8B5
:1066200001F0D2F90AA829F076FB0B280FDC40F222
:10663000AC24C2F200040126022003210422052317
:1066400025706670A070E170227163710CE70DF126
:106650004808804418F822CC18F824ECACF137092B
:1066600018F8266C18F8281C18F82A3C18F8214C41
:1066700018F8237C18F8250C18F8272C18F829BCD2
:106680004FEA09194FEA0C185FFA89F908F0F00887
:10669000BCF1400F8CBFCC46C446A4F13709A4F12D
:1066A0003008AEF1370A5FFA89F95FFA88F8402CB2
:1066B0008CBF4C4644464FEA0A1AA1F137084CEA0F
:1066C000040C5FFA8AFA4FEA081840F2AC24C2F2CE
:1066D0000004CDF810A05FFA88F8CDF8148084F893
:1066E00001C0DDF810804FEA0E1C0CF0F00CBEF17A
:1066F000400F98BFE046C646A7F1300CA7F1370817
:10670000A6F137095FFA8CFC5FFA88F8402F8CBF3E
:10671000474667464FEA09194FEA061C0CF0F00C91
:106720005FFA89F9402E98BFE146A0F1370CA0F13D
:1067300030065FFA8CFCF6B240288CBF60463046CB
:106740000E01DDF814C006F0F006402998BFB446EB
:106750006146A2F13006A2F1370CA3F1370A5FFAC5
:106760008CFCF6B2402A8CBF624632464FEA0A1AC7
:106770004FEA031C5FFA8AFA0CF0F00C402B98BF2A
:10678000E246ABF13706ABF13003F6B2DBB2BBF158
:10679000400F88BF33464EEA070749EA00090A431B
:1067A0004AEA03032570A77084F80390227163718D
:1067B0005AE600BF40F2AC20C2F20000704700BFB2
:1067C0002DE9F04F8146002089B00F4690460146E2
:1067D00001221E4601F07CFD041E27DB40F2E73A51
:1067E00010E001F0B5FE012104460A46002001F048
:1067F0004BFE002C1ADB14F008051BD0BAF1010A7D
:1068000000F05C8100200246012101F03DFE1F21C5
:10681000002001F09DFE041E4FF0FF014FF000002C
:10682000DFDA01210A46002001F02EFE204609B0E1
:10683000BDE8F08F2A460121284601F025FEBF2140
:10684000284601F085FE032103462846029301F005
:106850007FFE012184460A462846CDF80CC001F08F
:1068600013FE2A460121284601F00EFE9F212846EC
:1068700001F06EFE29460490284601F069FE0121D0
:106880000A460590284601F0FFFD2A4601212846C8
:1068900001F0FAFD4221284601F05AFE29460690F1
:1068A000284601F055FE01210A460790284601F0CE
:1068B000EBFD2A460121284601F0E6FD432128464A
:1068C00001F046FE10218346284601F041FE0121D9
:1068D00082460A46284601F0D7FD029BDDF80CC02F
:1068E000049A4CEA03031343059A1343069A13438D
:1068F000079A134343EA0B0B4BEA0A0A54EA0A04C9
:1069000094D42A460121284601F0BEFD462128469E
:1069100001F01EFE06F5805ABA441FFA8AFA844630
:106920005FFA8AF12846CDF80CC001F011FE012172
:1069300003460A462846029301F0A6FD2A46012195
:10694000284601F0A1FD4721284601F001FE4FEA4B
:106950001A218346284601F0FBFD012182460A46A2
:10696000284601F091FD029BDDF80CC04CEA0303C0
:106970001C4344EA0B0454EA0A043FF557AF2A4685
:106980000121284601F080FD7A21284601F0E0FD32
:10699000072184462846CDF80CC001F0D9FD01211D
:1069A0000A468346284601F06FFD2A460121284603
:1069B00001F06AFD7A21284601F0CAFD3B46824675
:1069C00049462A460095284601F0E8FD0121074680
:1069D0000A46284601F058FDDDF80CC0002E18BF0D
:1069E000B8F1000F4CEA0B0C4CEA040444EA0A0A22
:1069F0004AEA070768D100200246012101F044FD60
:106A00009F21002001F0A4FD802103460020029375
:106A100001F09EFD01210A468346002001F034FD6D
:106A200000200246012101F02FFDBF21002001F0CE
:106A30008FFD80218246002001F08AFD01210A4657
:106A40008146002001F020FD00200246012101F0D6
:106A50001BFDBC21002001F07BFD0A2180460020A7
:106A600001F076FD01210A460646002001F00CFDEA
:106A700000200246012101F007FD9F21002001F0C6
:106A800067FD08210546002001F062FD0121044652
:106A90000A46002001F0F8FC029B3B4343EA0B0B43
:106AA0004BEA0A0A4AEA090949EA080848EA0606D6
:106AB00035432C43204609B0BDE8F08F6FF00F043A
:106AC000204609B0BDE8F08F2A460121284601F092
:106AD000DBFC7A21284601F03BFD41460446334663
:106AE0002A460095284601F059FD012104430A4633
:106AF000284601F0C9FC27437DE700BF2DE9F04F90
:106B00000546002087B00C460246012101F0BCFC7E
:106B1000BF21002001F01CFD03218346002001F06D
:106B200017FD012103460A460020009301F0ACFC4A
:106B300000200246012101F0A7FC9F21002001F066
:106B400007FD02218246002001F002FD01210A46D4
:106B50008146002001F098FC00200246012101F04E
:106B600093FC5421002001F0F3FC294680460020CC
:106B700001F0EEFC01210A460746002001F084FCEA
:106B800000200246012101F07FFC5621002001F087
:106B9000DFFCE1B20646002001F0DAFC01210A46E2
:106BA0000546002001F070FC00200246012101F0A2
:106BB0006BFC5721002001F0CBFC210A0290002041
:106BC00001F0C6FC01210A460390002001F05CFCA4
:106BD00000200246012101F057FCBF21002001F0F6
:106BE000B7FC03210490002001F0B2FC01210A4609
:106BF0000590002001F048FC00200246012101F030
:106C000043FC9F21002001F0A3FC032184460020C7
:106C1000CDF804C001F09CFC012104460A46002086
:106C200001F032FC009B029A43EA0B0343EA0A0399
:106C300043EA090343EA08033B4333432B4313432B
:106C4000039ADDF804C01343049A1343059A1343CF
:106C500043EA0C0C5CEA04040CD524E001F078FC57
:106C6000012104460A46002001F00EFC002C1ADB2C
:106C7000E30718D500200246012101F005FC0A2196
:106C8000002001F065FCFF210446002001F060FCBB
:106C900004434FF0FF014FF00000DFD501210A4609
:106CA000002001F0F1FB204607B0BDE8F08F00BFE7
:106CB0002DE9F04F01210A46B9B0002001F0E4FBB4
:106CC0000020014601F0ACF900200146012201F04C
:106CD000FFFA0028C0F2808300200246012101F063
:106CE000D3FBFF21002001F033FC012106460A46B8
:106CF000002001F0C9FB002EC0F276834FF47A70B9
:106D000001F0ACFE00200246012101F0BDFB002095
:106D10001D2101F01DFC061EC0F26A83FF21002028
:106D200001F016FC012105460A46002001F0ACFBEB
:106D3000002DB8BF2846C0F24F8305F00905012D8C
:106D400018BF6FF00F0040F047830020024629462D
:106D500001F09AFBBF21002001F0FAFB0321002083
:106D600001F0F6FB29462A46002001F08DFB0020A9
:106D70000246294601F088FB9F21002001F0E8FB34
:106D80000321002001F0E4FB29462A46002001F0FF
:106D90007BFB00200246294601F076FB12210020F1
:106DA00001F0D6FBFF210646002001F0D1FB06438F
:106DB00000F11583FF21002001F0CAFB2946074698
:106DC0002A46002001F060FB002FB8BF3846C0F211
:106DD0000383FAB2511E40F2AA23C9B2C2F20003E1
:106DE0001E291A7000F20D83002440F2A92640F2F9
:106DF000B423C2F200032246C2F20006294620460E
:106E00001C80357001F040FBBF21204601F0A0FB43
:106E10000321204601F09CFB29462A46204601F02A
:106E200033FB22462946204601F02EFB9F212046B7
:106E300001F08EFB2146204601F08AFB29462A46B6
:106E4000204601F021FB22462946204601F01CFB8A
:106E50004821204601F07CFB21460390204601F0AA
:106E600077FB294604902A46204601F00DFB224676
:106E70002946204601F008FB4921204601F068FB25
:106E800021460590204601F063FB294606902A46DC
:106E9000204601F0F9FA22462946204601F0F4FA8C
:106EA0004C21204601F054FBFF210790204601F0C1
:106EB0004FFB294608902A46204601F0E5FA224673
:106EC0002946204601F0E0FA4D21204601F040FB22
:106ED0000F210990204601F03BFB29460A902A46E3
:106EE000204601F0D1FA22462946204601F0CCFA8C
:106EF0004A21204601F02CFBFF210B90204601F097
:106F000027FB29460C902A46204601F0BDFA22466E
:106F10002946204601F0B8FA4B21204601F018FB23
:106F20000F210D90204601F013FB29460E902A46B2
:106F3000204601F0A9FA22462946204601F0A4FA8B
:106F40004421204601F004FB21460F90204601F029
:106F5000FFFA294610902A46204601F095FA22466B
:106F60002946204601F090FA4521204601F0F0FA2A
:106F700010211190204601F0EBFA294612902A4682
:106F8000204601F081FA22462946204601F07CFA8B
:106F90004221204601F0DCFA21461390204601F000
:106FA000D7FA294614902A46204601F06DFA224667
:106FB0002946204601F068FA4321204601F0C8FA2C
:106FC00010211590204601F0C3FA294616902A4652
:106FD000204601F059FA22462946204601F054FA8B
:106FE0007A21204601F0B4FA21461790204601F09C
:106FF000AFFA294618902A46204601F045FA224663
:107000002946204601F040FABF21204601F0A0FAAF
:1070100003211990204601F09BFA29461A902A462E
:10702000204601F031FA22462946204601F02CFA8A
:107030009F21204601F08CFA02211B90204601F08E
:1070400087FA29461C902A46204601F01DFA22465E
:107050002946204601F018FA4021204601F078FA2E
:107060000D211D90204601F073FA29461E902A46F4
:10707000204601F009FA22462946204601F004FA8A
:107080004221204601F064FA33211F90204601F08E
:107090005FFA294620902A46204601F0F5F922465B
:1070A0002946204601F0F0F94421204601F050FA2B
:1070B00015212190204601F04BFA294622902A46BC
:1070C000204601F0E1F922462946204601F0DCF98C
:1070D0004321204601F03CFA40212390204601F054
:1070E00037FA294624902A46204601F0CDF9224657
:1070F0002946204601F0C8F94921204601F028FA26
:107100003F212590204601F023FA294626902A4661
:10711000204601F0B9F922462946204601F0B4F98B
:107120004621204601F014FA12212790204601F052
:107130000FFA294628902A46204601F0A5F9224652
:107140002946204601F0A0F94721204601F000FA27
:107150000C212990204601F0FBF929462A902A4665
:10716000204601F091F922462946204601F08CF98B
:107170004A21204601F0ECF9EE212B90204601F047
:10718000E7F929462C902A46204601F07DF922464F
:107190002946204601F078F94B21204601F0D8F924
:1071A00005212D90204601F0D3F929462A462E903C
:1071B000204601F069F940F2AC20C2F20000FFF76E
:1071C00031F92246844629462046CDF804C001F014
:1071D0005BF9BF21204601F0BBF903212F90204627
:1071E00001F0B6F9294630902A46204601F04CF9C4
:1071F00022462946204601F047F99F21204601F00A
:10720000A7F903213190204601F0A2F929463290D6
:107210002A46204601F038F922462946204601F048
:1072200033F95521204601F093F921463390204649
:1072300001F08EF92A4634902946204601F024F9BF
:107240004FF480711020FFF759FC43F2724103465E
:1072500014200293FFF752FC4FF4807183462046BE
:10726000FFF74CFC224682462946204601F00CF9E5
:10727000BF21204601F06CF903213590204601F032
:1072800067F9294636902A46204601F0FDF8224645
:107290002946204601F0F8F89F21204601F058F9D0
:1072A00021468146204601F053F9294680462A4668
:1072B000204601F0E9F822462946204601F0E4F88C
:1072C0009F21204601F044F904213790204601F027
:1072D0003FF92A4606462946204601F0D5F8029B8A
:1072E000DDF804C0039A4CEA03033B4343EA0B0373
:1072F00043EA0A031343049A1343059A1343069A75
:107300001343079A1343089A1343099A13430A9A9B
:1073100013430B9A13430C9A13430D9A13430E9A7B
:1073200013430F9A1343109A1343119A1343129A5B
:107330001343139A1343149A1343159A1343169A3B
:107340001343179A1343189A1343199A13431A9A1B
:1073500013431B9A13431C9A13431D9A13431E9AFB
:1073600013431F9A1343209A1343219A1343229ADB
:107370001343239A1343249A1343259A1343269ABB
:107380001343279A1343289A1343299A13432A9A9B
:1073900013432B9A13432C9A13432D9A13432E9A7B
:1073A00013432F9A1343309A1343319A1343329A5B
:1073B0001343339A1343349A1343359A1343369A3B
:1073C000134343EA0909379B49EA080848EA0307D7
:1073D00047EA060000EAE07039B0BDE8F08F2946C0
:1073E0002A46002001F050F8304639B0BDE8F08F51
:1073F00001210A46002001F047F8304639B0BDE8C7
:10740000F08F6FF01000E7E758B940F2AC23C2F2FA
:107410000003187058709870D87018715871FFF781
:1074200047BC4FF0FF307047F0B50746002083B0EF
:1074300000240E460246012101F026F820463A219A
:1074400001F086F83A463346214605460094204628
:1074500001F0A4F8012105430A46204601F014F882
:10746000284603B0F0BD00BF2DE9F04F8046002054
:1074700087B089460122014600F02AFF041EC0F2AF
:10748000F88000200246012100F0FEFFBF2100200D
:1074900001F05EF803218246002001F059F8012135
:1074A0000A460746002000F0EFFF002002460121B7
:1074B00000F0EAFF9F21002001F04AF80121064672
:1074C000002001F045F8012105460A46002000F0A1
:1074D000DBFF00200246012100F0D6FF0020192129
:1074E00001F036F84AEA07073C4326432E43051EBF
:1074F000C0F2C580FF21002001F02AF801210A46D0
:107500000546002000F0C0FF00200246012100F0E7
:10751000BBFFBF21002001F01BF8032182460020A1
:1075200001F016F801210A460446002000F0ACFFE5
:1075300000200246012100F0A7FF9F21002001F05A
:1075400007F807460020014601F002F84AEA040461
:107550000121344383460A4600203C4300F094FF57
:1075600054EA0B0400F18580002D40F3868040F240
:10757000A925C2F200052E7856B9FEF7BFFE00EA33
:10758000E07515EA250038BF304607B0BDE8F08F3A
:10759000002040F2B42702460121C2F200073E88D3
:1075A00000F072FF4021002000F0D2FFF1B203464C
:1075B0000020039300F0CCFF01210A4683460020FF
:1075C00000F062FF00200246012100F05DFF412132
:1075D000002000F0BDFF310A8246002000F0B8FF15
:1075E000012106460A46002000F04EFF039B43EAB5
:1075F0000B0B4BEA040444EA0A04344339D4002058
:1076000000240246012100F03FFF3A21204600F00D
:107610009FFF214604AA06230094204600F0BEFFE7
:1076200001210A46204600F02FFFBDF81010B1F5E9
:10763000805F59D2CA0757D49DF81530DB0953D162
:10764000BDF8126040F2EE539E4250D932469DF88A
:1076500015409DF8143041F25C6000940193C0F62F
:10766000040040F2EE53FCF769FD6FF00F04FFF7E2
:107670001FFB204607B0BDE8F08F002681E70121FF
:107680000A46002000F000FF00200246012100F021
:10769000FBFEBF21002000F05BFF0321814600209C
:1076A00000F056FF01210A460746002000F0ECFEDC
:1076B00000200246012100F0E7FE9F21002000F09B
:1076C00047FF80460020014600F042FF01210446AA
:1076D0000A46002000F0D8FE49EA080333433B4342
:1076E0001C43C6D42846C5E7BDF81220AFE740F2D8
:1076F000A9244FF0000A3980C2F2000485F800A0E6
:10770000002E3FF43AAF9DF8143003F09003802B25
:107710007FF433AFB14538BF4E4640463146FFF7A0
:1077200083FE2378054613B15046054329E7FEF74B
:10773000E5FDFAE728B940F2B823C2F20003186069
:1077400070474FF0FF30704740F2B823C2F2000399
:107750001A68002001321A60704700BF40F2B82357
:10776000C2F200031868704740F2B823C2F2000367
:107770001B68181A704700BF002840F0AB8010B596
:10778000012186B004461F2003F08AFB534B00946E
:107790009A6802F00C02082A67D01A68504942F031
:1077A00001021A609C601A6822F0847222F480320E
:1077B0001A6059601A6822F480221A60DC60019411
:1077C0001A6842F480321A601A4603E0019BB3F54E
:1077D000A06F09D0136803F400330093019B0133B9
:1077E0000193009B002BF1D03C4B1B6813F400333A
:1077F00018BF01230093009B012B39D00021394889
:1078000003F08EF84FF4407003F080F801214FF040
:10781000805003F05DFB012003F0D2FA324803F000
:1078200021FB012003F036FB03A803F0D9FB632200
:1078300041F2873303A80492059303F091FB02A859
:1078400003F078FC002302A918468DF808308DF863
:1078500009308DF80A3003F0C9FB009810F1FF30B1
:1078600018BF4FF0FF3006B010BD01230093C5E7ED
:107870001A4B1E491A6C1E4842F080521A640A685C
:1078800042F480420A609A689A609A6842F4004220
:107890009A609A6842F4A0529A6058601A6842F05E
:1078A00080721A601A4611680C4B8901FBD5114A87
:1078B00040F2056111609A6822F003029A609A68AA
:1078C00042F002029A601A46936803F00C03082BF8
:1078D000FAD193E74FF0FF30704700BF0038024005
:1078E0001030002400400008000310000070004029
:1078F00008544007003C024010B5FAF77BF86FF0DF
:107900007F40FBF77BFB0020FBF77AFB0020FBF7B7
:1079100041F9FBF739FB00200146FBF743F91E480C
:10792000FBF796F900F072F84FF0FF30002100F0FD
:1079300019FF32244FF47A7001F090F8013CF9D12C
:107940006FF00100012103F0DBFA6FF080000121EC
:1079500003F0E2FA4FF0FF30012103F0E9FA4FF0B3
:10796000FF30012103F0F0FA4FF0FF30214603F021
:10797000C7FA4FF0FF30214603F0CEFA4FF0FF3048
:10798000214603F0D5FA21464FF0FF3003F0DCFA30
:10799000024B034ADA60FEE7C016040800ED00E07F
:1079A0000100FA05014B1868704700BF002004E091
:1079B000024B188880B28002704700BF227AFF1FF6
:1079C0004FF44030704700BF10B40022441E0E4BED
:1079D00051100B4412F0010F1B78DBB24FEA131168
:1079E00008BF0B4603F00F03092B8CBF3721302152
:1079F00001320B44182A04F8013FE8D10023037632
:107A00005DF8044B18467047107AFF1F074A136849
:107A10001BB9EFF31081064801604FF0010080F3BD
:107A20001088013313600020704700BFC00200209F
:107A3000BC020020074B186848B10138186020B913
:107A4000054B1B6883F310887047002070474FF088
:107A5000FF307047C0020020BC0200200F291CD854
:107A60000F4BDB68DB43C3F3022330B4C3F10403E1
:107A7000994000F1604543B205F561450901094CA3
:107A800000F01F005B090122C9B2824085F8001393
:107A9000002044F8232030BC70474FF0FF3070477F
:107AA00000ED00E000E100E02DE9F04F044697B062
:107AB000002840F0A68207A803F08CF8DFF8809336
:107AC000D54BD64FD64E3C604FF0040A4FF40068B9
:107AD000A3F818A002A8A9F8188003F02BF9052133
:107AE0000A46D0488DF80D408DF80E4003F030F96D
:107AF000CC480621052203F02BF9CA4807210522AC
:107B000003F026F94FF0020B202202A9C548029289
:107B10008DF80CB003F0BAF8802202A9C148029295
:107B2000012503F0B3F8BC48CDF808A002A98DF8F0
:107B30000C5003F0ABF8484602A9CDF808804FF08E
:107B4000400A03F0A3F802A9B6488DF80CB08DF8EE
:107B50000F50CDF808A003F099F829464FF4805053
:107B600003F0C2F929464FF4001003F099F92946B1
:107B70004FF4800003F094F92146AB4803F03CF841
:107B80004FF0C069A94BA84808934FF4803207A969
:107B90004FF48068119209940A940B940C940E94FB
:107BA0000F941094CDF81C90CDF8348002F0DAFFD9
:107BB00021469F4803F020F807A99D4809940B949B
:107BC000CDF828A0CDF81C90CDF8348002F0CAFF83
:107BD0002946304603F0DCFA2A463046032103F0FA
:107BE000E5FA05213A20FFF739FF4FF482704FF490
:107BF00000710722ADF80840ADF80C40ADF8164012
:107C0000ADF80A00ADF81210ADF81820ADF80EB0BE
:107C1000ADF8105033883022304602A99CB2ADF83E
:107C2000142003F08DFABDF80A30B3F5827F00F01E
:107C3000BE81794DDFF808B2DFF808824FF4805337
:107C40004FF4806900242B8302A80193ABF81890AD
:107C50007C6003F06FF828460C2105228DF80D405A
:107C60008DF80E4003F074F828460D21052203F02C
:107C70006FF828460E21052203F06AF828460F21E6
:107C8000052203F065F84FF0020A4FF4005228462F
:107C900002A902928DF80CA002F0F8FF4FF4004206
:107CA000284602A90292012602F0F0FF019B0293EE
:107CB000284602A98DF80C6002F0E8FF584602A998
:107CC0004FF4804BCDF8089002F0E0FF284602A95F
:107CD0008DF80CA08DF80F60CDF808B002F0D6FF3B
:107CE0005846314603F0F4F831464FF4001003F0E3
:107CF000D7F831464FF4800003F0D2F821464D48C2
:107D000002F07AFF4C4A4B4808924FF4803307A99F
:107D10001193079409940A940B940C940E940F9465
:107D20001094CDF8349002F01DFF2146434802F034
:107D300063FF402341480A9307A9079409940B94D1
:107D4000CDF8349002F00EFF3146404603F020FAA1
:107D500032464046032103F029FA05210E20FFF7A1
:107D60007DFE4FF482714FF400720723ADF8084096
:107D7000ADF80C40ADF81640ADF80A10ADF8122081
:107D8000ADF80EA0ADF81060ADF81830B8F80030BE
:107D90002822404602A99CB2ADF8142003F0D0F985
:107DA000BDF80A30B3F5827F00F0D7801A4EDFF8B5
:107DB00074A0DFF894804FF400494FF4807B0024D6
:107DC000AAF8189002A8A6F818B0BC6002F0B2FF9A
:107DD00050460F2106228DF80D408DF80E4002F01E
:107DE000B7FF30460321062202F0B2FF30460421DD
:107DF000062202F0ADFF06223046052102F0A8FF60
:107E00000823022730460DEB030102938DF80C7016
:107E100002F03CFF202319E000040240C4020020CD
:107E20000030014000000240406402400C3001403C
:107E300058640240586002400C38004070600240B4
:107E4000000C024000380040003C0040304602A9CF
:107E50000125029302F01AFF504602A9CDF80890BE
:107E60008DF80C5002F012FF304602A9CDF808B090
:107E700002F00CFF1023304602A902938DF80C701B
:107E80008DF80F5002F002FF4846294603F020F813
:107E900029464FF4001003F003F829464FF4800000
:107EA00002F0FEFF2146584802F0A6FE4FF480661D
:107EB000564A554808924FF4803307A91193079406
:107EC00009940A940B940C940E940F9410940D96AC
:107ED00002F048FE21464E4802F08EFE402307A9DC
:107EE0004B480A93079409940B940D9602F03AFEBE
:107EF0002946404603F04CF92A464046032103F048
:107F000055F905210D20FFF7A9FD4FF482714FF4BB
:107F100000720723ADF80840ADF80C40ADF81640EC
:107F2000ADF80A10ADF81220ADF80E70ADF8105093
:107F3000ADF81830B8F80030282202A940469CB2AB
:107F4000ADF8142003F0FCF8BDF80A30B3F5827FD9
:107F500019D0002017B0BDE8F08FB8F800306340AA
:107F60009D073FF423AFFF23A8F80C30B8F800308A
:107F700003F48273002B34D0B8F808301C06FBD40D
:107F8000244B9B8912E7B8F8003063409907E0D092
:107F9000FF23A8F80C30B8F8003003F48273BBB1AB
:107FA000B8F808301A06FBD41B4B9B89D1E73388FD
:107FB000634099073FF43DAEFF23B381338803F458
:107FC0008273BBB133891A06FCD4144B9B8930E60B
:107FD000B8F80830DB07E7D4B8F80830DB07F7D586
:107FE000E2E7B8F80830D807CAD4B8F80830D8079C
:107FF000F7D5C5E73389DB07E7D43389DB07F9D544
:10800000E3E74FF0FF30A5E7406002400C3C004042
:108010008860024000380040003C004000300140D1
:1080200070B582B005460C46684602F083FE072C08
:1080300000F24481DFE804F055A2AA04B3B5B7B159
:108040000024002201238DF805208DF80630012D33
:1080500050D0C0F0AE80022D40F0A78099480F218B
:10806000062202F075FE98480321062202F070FEF7
:1080700095480421062202F06BFE93480521062252
:1080800002F066FE082390488DF80450694600937C
:10809000002C40F0F18002F0F9FD20238A48009383
:1080A000694602F0F3FD01264FF400438548009332
:1080B00069468DF8046002F0E9FD4FF48073824850
:1080C0000093694602F0E2FD10237F488DF80760B7
:1080D00069468DF80450009302F0D8FD204602B0A6
:1080E00070BD002402220023012D8DF805208DF89B
:1080F0000630AED174480C21052202F029FE7248E8
:108100000D21052202F024FE6F480E21052202F007
:108110001FFE6D480F21052202F01AFE002C00F010
:10812000858002244FF400536946674800938DF818
:10813000044002F0ABFD4FF40043694662480093EF
:1081400002F0A4FD4FF4805369465F4800938DF818
:10815000044002F09BFD4FF4806369465B48009346
:1081600002F094FD4FF48043694657488DF804406F
:10817000009302F08BFD002002B070BD00240222AB
:1081800001238DF805208DF8063060E700240023D8
:108190008DF805308DF8063059E7012451E70124A8
:1081A000A0E70124EBE70124F1E76FF0010002B042
:1081B00070BD05210A46434802F0CAFD4148062128
:1081C000052202F0C5FD3F480721052202F0C0FD4F
:1081D000002C73D120233B480093694602268DF87A
:1081E000046002F053FD802336480093694602F094
:1081F0004DFD012504233448009369468DF8045051
:1082000002F044FD4FF4006330480093694602F0E9
:108210003DFD2C48694640238DF804608DF80750D9
:10822000009302F033FD204602B070BD4FF40053BE
:1082300025480093694602268DF8046002F026FD69
:108240004FF4004320480093694602F01FFD4FF4AD
:1082500080531D48009369468DF8045002F016FDC6
:108260004FF4806319480093694602F00FFD694698
:108270004FF480431448CFE702F008FD2023124852
:108280000093694602F002FD4FF400430D4800934D
:1082900069468DF8045002F0F9FC4FF480730A48E7
:1082A0000093694602F0F2FC102307488DF8045051
:1082B0006946009302F0EAFC002010E76FF002002C
:1082C0000DE700BF0000024000040240000C024025
:1082D00070B586B000234FF482764FF40075072402
:1082E000ADF80430ADF80830ADF81230ADF80660E6
:1082F000ADF80E50ADF81440A14200F2BC80DFE8AA
:1083000001F0473B2F0942362A040023ADF806301E
:10831000ADF80E3002210123ADF80A10ADF80C3093
:10832000072A00F29680012861D03BD3022835D17C
:10833000524C013A2388D200204601A99DB2ADF8E3
:10834000102002F0FDFEBDF80630B3F5827F6FD03D
:10835000002006B070BD0023ADF80630ADF80E3039
:1083600002210023ADF80A10ADF80C30D8E7002345
:10837000ADF80630ADF80E3000210123ADF80A103B
:10838000ADF80C30CCE70023ADF80630ADF80E3078
:108390000023ADF80A30ADF80C30C1E76FF00100F2
:1083A00006B070BDBDF80630002B52D0344C238887
:1083B000D200204601A99DB2ADF8102002F0C0FE07
:1083C000BDF80630B3F5827FC2D123886B40990790
:1083D000BED0FF23A381238803F48273002B46D0F1
:1083E00023891A06FCD4264B00209B89B1E7254C33
:1083F000013A2388D200204601A99DB2ADF8102091
:1084000002F09EFEBDF80630B3F5827FA0D123882E
:108410006B409E079CD0FF23A381238803F48273C3
:108420000BB323891D06FCD4164B00209B8990E7D3
:1084300023886B4099078BD0FF23A381238803F403
:1084400082734BB123891A06FCD40C4B00209B8904
:108450007FE76FF002007CE72389DB07F5D42389EF
:10846000DB07F9D5F1E72389D807FCD5DCE72389B9
:10847000DB07FCD5B7E76FF003006AE7003C00407C
:10848000003001400038004001281BD00FD30228E3
:108490000AD149B3012934D12A4B002A4CD14FF4D7
:1084A00080711046598370476FF00100704711B317
:1084B000012926D1244B002A34D04FF400621A83BC
:1084C0000020704749B101291BD11F4B002A2ED033
:1084D0004FF480621A83002070471A4BEAB14FF4C0
:1084E000805208461A837047184B8AB14FF40042F5
:1084F00008461A837047134B32B1042208461A8388
:1085000070476FF00200704704211046598370478E
:108510004FF400411046598370474FF48051104684
:10852000598370474FF400611046598370474FF4E8
:1085300080611046598370474FF480721A8300207F
:10854000704700BF00040240000C024000000240DF
:1085500001281BD018D302280CD10D4B89B2998168
:108560001A8802F4827242B11A891106FCD49889E1
:1085700080B270476FF0010070471A89D207F6D4B5
:108580001A89D207F9D5F2E7024BE7E7024BE5E794
:10859000003C004000300140003800402DE9F84325
:1085A0000128089D4AD040D302283AD1DFF808E1DB
:1085B000DFF80891384CDFF80881384F6668002EE4
:1085C00066D1BE892768DFF8FCC027F00106266067
:1085D0004CF82050002A52D0E26046F48067636075
:1085E000D8F8006026F00102C8F8002000293CD02D
:1085F000C8F80C1042F4806671462046C8F8043072
:1086000002F004FB4046494602F000FBFDB147F092
:10861000110346F0010223600020C8F80020BDE8E5
:10862000F8836FF00100BDE8F883DFF88CE01C4CA4
:10863000DFF894801B4F4FF0F259BFE74FF0F25E26
:10864000DFF88890184CDFF88880184FB6E727F0DD
:10865000100343F0010346F001022360C8F8002034
:1086600060680028FCD1BDE8F883114AC8F80C20E6
:1086700026F48066FF2126F001061170BCE70D4A42
:10868000E26027F48067FF2027F001071070A6E75B
:108690006FF00200BDE8F88340600240003C0040FB
:1086A0004064024000300140586002400038004001
:1086B000D0020020D102002000003910400E00201E
:1086C00088600240C4020020586402403900002043
:1086D0007060024010B50548054902F097FA054B55
:1086E0001B6813B1BDE81040184710BD406402403C
:1086F00000003910C402002010B506484FF0F251B6
:1087000002F084FA044B5B6813B1BDE810401847CF
:1087100010BD00BF58600240C402002010B50548DB
:10872000054902F073FA054B9B6813B1BDE8104090
:10873000184710BD4060024000003910C4020020FC
:1087400020B9044A044B1080188070474FF0FF3066
:10875000704700BFD4020020D20200204FF0FF304B
:10876000704700BF4FF0FF30704700BF00207047D8
:108770004FF0FF30704700BF4FF0FF30704700BF31
:108780004FF0FF30704700BF4FF0FF30704700BF21
:108790004FF0FF30704700BF4FF0FF30704700BF11
:1087A0004FF0FF30704700BF4FF0FF30704700BF01
:1087B0004FF0FF30704700BF4FF0FF30704700BFF1
:1087C0004FF0FF30704700BF4FF0FF30704700BFE1
:1087D0004FF0FF30704700BF01283CD830B50C4641
:1087E00087B0054669B9012805D1102002F074F957
:1087F000002007B030BD084602F06EF9204607B0F1
:1088000030BD01214FF0005002F062FB0024032232
:108810003C23012D8DF804200293059406A90BD169
:10882000202341F8183D0D4802F030FA02A910202B
:1088300002F03AF92946D8E7102341F8183D0748D5
:1088400002F024FA204602A902F02EF92046012166
:1088500002F042F9CCE74FF0FF30704700000240D1
:1088600010B5044668B1012808D1042002F06AF965
:108870002146102002F042F9002010BD4FF0FF30D9
:1088800010BD042002F04EF92046012102F036F915
:10889000204610BD022848D82DE9F0414E1EB6F5FD
:1088A000803F84B044D21746234A984652F820505D
:1088B000224B9D42044631D003F580639D422DD06A
:1088C0001F4B012153F8200002F002FB2846012132
:1088D000002202F0CFFC1B4A0296532300262846B2
:1088E00001A9ADF8043042F82470ADF80C60ADF881
:1088F000066002F065FC01210A46284602F0BAFC37
:108900002846012102F0A8FC0F4B414613F8240031
:10891000FFF7A4F8304604B0BDE8F081084B012110
:1089200053F8240002F0E0FAD0E74FF0FF30704730
:108930006FF00100EFE700BFD4160408000001400B
:10894000EC160408D8020020E016040810B54FF019
:108950008040012102F098FC00B910BD4FF080402A
:10896000012102F09DFC024BBDE810401B68184736
:10897000D802002010B50748012102F085FC00B99B
:1089800010BD0448012102F08BFC034BBDE81040F0
:108990005B68184700040040D802002010B5074863
:1089A000012102F071FC00B910BD0448012102F060
:1089B00077FC034BBDE810409B681847000C004053
:1089C000D802002070B5044604EB4404114EC4EBF9
:1089D000C40484B001211020A40002F079FA00251B
:1089E0004FF6FF73304601A9013C0293ADF80440F5
:1089F000ADF80C50ADF8065002F0E2FB01210A463A
:108A0000304602F037FC3046012102F025FC2846B2
:108A100004B070BD0010004010B5044684B0C0B969
:108A20000120014602F060FA4FF6FF72A7230A48C0
:108A3000029201A9ADF80430ADF80C40ADF8064043
:108A400002F0BEFB0448012102F006FC204604B0FF
:108A500010BD4FF0FF30FAE700000140044A516AB0
:108A600089B2536A5B1A9BB28342FAD900207047DD
:108A7000000001402DE9F04F83469DB0002840F0F2
:108A80000F81894A894B8A48DFF85CE2894E8A491E
:108A90008A4F8B4DC2F800B0C2F804B0C2F808B0DB
:108AA000C2F80CB00324C3F800B0C3F804B0C3F894
:108AB00008B0C3F80CB0C0F800B001A8AEF8004090
:108AC0004FF0020AC7F800B085F800B081F800B096
:108AD000C6F800B0C6F804B0C6F808B0C6F80CB0C6
:108AE00002F028F901A977488DF80840CDF804A0D4
:108AF0008DF80BB002F0CAF8042301A97148019364
:108B000002F0C4F801A97048CDF804A0102402F0C6
:108B1000BDF801A96C48019402F0B8F801A96948B0
:108B2000019402F0B3F8202301A9664801930124BF
:108B300002F0ACF801A965480194654DDFF8A091F9
:108B4000DFF89881634F02F0A1F801A95F48CDF8E2
:108B500004A002F09BF821464FF440708DF80840C5
:108B60008DF80AB0DA4602F0BFF95C4685F800B02D
:108B70005946FF2020414A08013210F0010FD2B2BD
:108B80004FF0060304F101040DD011F0010F18BFDE
:108B9000484617F80A1008BF404601F021FF29781F
:108BA0000131C9B22970082C0AF10C0AE1D1CB07B6
:108BB000494FDFF8389148BF013103A800243970CC
:108BC00001F0FEFE06224FF4004303A80392059332
:108BD0000494069401F0E0FE07A801F0D3FE3B7870
:108BE0003E488DF821405B08012507A98DF83030FB
:108BF00009940B948DF8205001F09CFE07A9384889
:108C000001F098FE2946354801F036FF284601F06C
:108C10003DFF2946314801F0D9FE2946304801F090
:108C2000D5FE29464FF4800002F03AF921462D483E
:108C300001F0E2FF0DA801F0CDFF3B7829480D942B
:108C4000EB404FF4805C4FF4804E4FF400320DA99E
:108C50004FF480684FF480771193CDF850C0CDF871
:108C600054E01792109412940F96CDF83890CDF8E6
:108C70004C80169701F076FF29461A4801F0BCFF98
:108C80002A461848102101F0DBFF05213820FEF7A5
:108C9000E5FE124801F0EAFE20461DB0BDE8F08F67
:108CA0004FF0FF30F9E700BFE40200200C03002082
:108CB00020030020F8020020F402002028030020F6
:108CC00008030020000802400000024000040240A7
:108CD0001C030020F8160408240300200020014093
:108CE00000210140106402403E00002008230140A2
:108CF00007289ABF024B33F810004FF0FF3070473F
:108D0000E402002008B5024801F0B0FE002008BDD2
:108D1000002001402DE9F04F3048314983B001F087
:108D200075FF304B1B78002B51D12F4A2F4B1278F7
:108D300019782F4B0192154615FB01F1C9B22D4848
:108D40002D4A1C784B0018441A4401F01F034909AE
:108D5000002C37D0294D2A4EB5F800A0DFF8A880A6
:108D600002EB440E4FF0010C40F6B83912E05445C6
:108D70001FDC0BF1FF3B22F802BC0133DBB2202BDE
:108D800000F1020006F1020602D101310023C9B24E
:108D9000724517D03588048832F802BB2C1B002C92
:108DA0000CFA03F7B8BF6442BBF1000FDFD17F2C90
:108DB000E3DD58F8214005803C4322F8029C48F846
:108DC0002140DAE7019B13B903B0BDE8F08F0D48ED
:108DD00003B0BDE8F04F01F049BE00BF106402408F
:108DE00039008010F4020020080300202403002032
:108DF0001C030020E40200200C0300203E000020A1
:108E0000F8020020002001402803002012230B80DC
:108E100000487047D417040804230B8000487047AB
:108E2000D0170408704700BF704700BF704700BFED
:108E3000704700BF704700BF704700BF704700BF5A
:108E4000704700BF704700BF704700BF704700BF4A
:108E5000704700BF704700BF704700BF704700BF3A
:108E6000704700BF704700BF704700BF01207047C8
:108E7000704700BF00207047704700BF0020704758
:108E80000020704765230B800048704720180408B5
:108E900010B50C4B8CB01B68ADF8043002A81B0C4D
:108EA0000C468DF80630FEF78FFD0028ABBF02A8F8
:108EB00001A822462246044902F048FE02480CB0AE
:108EC00010BD00BF04180408B4B30020F0B5174B60
:108ED000174C0E4693E8070085B001AF3D4603C529
:108EE0002A802278EAB1203A5F2A8CBF002301232E
:108EF00001220132ABB114F8011FA1F120035F2B55
:108F00008CBF0023012371B1202AF2D10848002B25
:108F100008BF38463246074902F018FE054805B03A
:108F2000F0BD3846F6E70248F4E700BF0818040829
:108F3000E03F0008B4B3002030B5084B084C0D46A4
:108F400093E8070085B001AB83E8070018462A467E
:108F5000214602F0FBFD204605B030BD1418040880
:108F6000B4B30020022901D00020704708B508469C
:108F7000002100F093FE002008BD00BF012901D0B0
:108F80000020704708B50846002100F027FE0020A9
:108F900008BD00BF10B50221044604F071FF204651
:108FA000812104F06DFF002010BD00BF002000F003
:108FB00025BC00BF002000F021BC00BF012000F054
:108FC0001DBC00BF10B502210B460446402204F030
:108FD00027FF204681214022022304F021FF044A7A
:108FE00004480221402304F067FF002010BD00BFA9
:108FF00058A8002098A80020F0B5174B174C0E4633
:1090000093E8070085B001AF3D4603C52A8022786A
:10901000EAB1203A5F2A8CBF0023012301220132EA
:10902000ABB114F8011FA1F120035F2B8CBF00230B
:10903000012371B1202AF2D10848002B08BF38461D
:109040003246074902F082FD054805B0F0BD3846BA
:10905000F6E70248F4E700BF08180408E03F0008FC
:10906000B4B30020F0B5174B174C0E4693E8070039
:1090700085B001AF3D4603C52A802278EAB1203A87
:109080005F2A8CBF0023012301220132ABB114F807
:10909000011FA1F120035F2B8CBF0023012371B1BD
:1090A000202AF2D10848002B08BF3846324607492B
:1090B00002F04CFD054805B0F0BD3846F6E7024821
:1090C000F4E700BF08180408E03F0008B4B300202C
:1090D000F0B5174B174C164693E8070085B001AF63
:1090E0003D4603C52A802278EAB1203A5F2A8CBF28
:1090F0000023012301220132ABB114F8011FA1F1B9
:1091000020035F2B8CBF0023012371B1202AF2D1F1
:109110000848002B08BF38463246074902F016FDC2
:10912000054805B0F0BD3846F6E70248F4E700BF51
:1091300008180408E03F0008B4B30020F0B501208F
:10914000254C83B0014601F0ABFE032600232046E8
:1091500069464FF4D85202278DF806308DF8073053
:1091600000928DF805608DF8047001F08FFD2046A7
:1091700008210A2201F0ECFD204609210A2201F013
:10918000E7FD20460B210A2201F0E2FD20460A22DB
:109190000C2101F0DDFD01254FF480636946204676
:1091A00000938DF804708DF805608DF8075001F07C
:1091B0006DFD0A210A46204601F0CAFD29464FF4FA
:1091C000804001F091FE2946802001F075FE28467E
:1091D00001F056FD03B0F0BD00000240432008211D
:1091E000FEF73CBC08B50A4803F058FE38B90848F9
:1091F00004F0F6FE0648BDE8084006F013BC04483B
:1092000006F08AFB0248BDE8084006F00BBC00BF30
:1092100098A8002080B2FFF721BC00BF4FF47A73FA
:1092200003FB00F080B2FFF719BC00BF30B5104D52
:1092300083B00420012101F033FE01240023032226
:10924000284669468DF805208DF806308DF80730E0
:1092500000948DF8044001F019FD2846214601F0E4
:1092600073FD4FF45460FFF7F9FB03B030BD00BF4E
:1092700000080240034811B1012101F067BD01213E
:1092800001F062BD0008024002287DD870B54FF0A1
:10929000A04282B03E4D3F4B1668009304463E4AC2
:1092A0003E4B2846012102F085FC002000F0A6FA82
:1092B0000CB9330332D43A4B3A4A009301213A4B6A
:1092C000334802F08DF9324804F088FE4CF25030F9
:1092D000FFF7C4FB2E4804F07FFE344B1B78422B73
:1092E00016D0334B186910F4806406D0002128484A
:1092F00003F0B6FD002002B070BD2548012103F047
:10930000E5FE0121224803F0ABFD204602B070BD0E
:10931000284B93F90030002BE8DCE2E72846FFF702
:109320000DFF21491E4A1F4BC5F8E41528460121AF
:10933000C5F8E825C5F8EC3503F00EFB284603F028
:1093400057FD284604F01CF908214320FEF786FB50
:1093500002210B46012403262846402285F81041AD
:1093600085F8126104F05CFD284681214022022329
:1093700004F056FD284602210F4A402304F09CFDCC
:10938000204600F03BFAA8E74FF0FF30704700BFDF
:1093900098A80020581704082CB30020A41804082B
:1093A00088180408E8170408A0170408D63F000826
:1093B00000000240D73F000858A80020064B1B7849
:1093C000422B01D000207047044B187810F0800F1A
:1093D00018BF0020704700BFD43F0008D53F0008E9
:1093E0000020704738B50D4C2178054661B90C4C0A
:1093F000217841B1284603F0CDFF2846217802F0BC
:1094000089FF0023237038BD03F0C4FF284621786C
:1094100002F080FF00232370E9E700BF8B050020E6
:10942000840500202DE9F84F704C237813B90020F3
:10943000BDE8F88F06460D4605F020F90028F6D065
:109440006B4F3B78022B6DD0012B18D0002BEED147
:10945000DFF8D081B8F800309BB20BB1237813BB92
:10946000DFF8C481634A98F8003012786249634893
:1094700003F004F801233B700020BDE8F88FDFF80B
:10948000A881304698F8001005F000F901285DD950
:10949000042800F090800238C0B2012853D93B78EC
:1094A000002BD5D0C3E7FEF7B1FA554AB8F8003023
:1094B00015889BB2AD089D4228BFB8F80050B8F897
:1094C0000030ADB25B1B2EB29BB2002EA8F800306C
:1094D00018DD4C484C4CDFF854E1002180468C46A6
:1094E0000288038801339BB292B23F2B01F1010144
:1094F0005EF82220038088BFA8F800C0B14244F87B
:10950000042BEDD1AC00414B414D1B783E493B480B
:10951000E4B222462C7002F099FF02233B70FEF762
:1095200089FA84E7DFF8E480304698F8001005F007
:10953000ADF80028B3D0012805D0042846D0022871
:1095400046D00328ABD100233B7081E72B4B98F822
:10955000002003EB4213D3F8A458AD08F3D02D4EEE
:1095600033889BB2C3F140039D4298D2FEF74EFA76
:10957000DFF884B0284CDFF8B8905BF804ABCAF38E
:10958000031010305146FBF77BFC70B9228823880A
:1095900001339BB23F2B238088BF2080338892B257
:1095A00001339BB249F822A03380013DE5D1FEF79B
:1095B00041FA3D7056E7194A98F800301278304663
:1095C000294603F089F90028BDD068E7144AF3E77B
:1095D0000F4A98F80030127808480B4902F036FF1D
:1095E0003B78002B3FF434AF21E700BF8505002016
:1095F0008A0500207E05002058A8002098A8002099
:109600002C030020820500203C0500208B05002053
:109610007D05002030030020860500203303002054
:109620003203002080050020840500203403002040
:10963000380400202DE9F04F89B0DFF89CC1DFF835
:109640009CB1DFF89CA1DFF89C91DFF89C81584F1A
:10965000584E91F83820584D0390584800230C4636
:109660000121ACF800302B70ABF80030AAF80030C4
:1096700089F80030A8F800303B80338001704AB18F
:1096800094F84310012911D0012A03D094F84C30EA
:10969000012B72D0FFF792FE2B781BB1D4F88030EB
:1096A0001B6C9847002009B0BDE8F08F94F8441077
:1096B0000329E9D11B01E01890F852100A0661D481
:1096C000B0F85400ADF814003D4A3E48DFF81CE104
:1096D0000490BDF8140010803B4805908EF80010EF
:1096E0002344583399789B88080659D413808EF800
:1096F00000100398CDF818C0079202F0C7FD334B55
:10970000049A187011780398049302F0BFFD079A29
:10971000049B1288197894F820E094F82130019283
:109720002B4A1070022072460090039802F064FDEC
:10973000274B059894F821E01978007894F82020B8
:109740000190022300930398734602F055FD012215
:109750002049DDF818C02A70184A0023ACF8003000
:109760000B70ABF80030AAF8003089F80030A8F888
:1097700000303B80338013708CE794F84D20032A2F
:1097800088D197E7104A05920E4A0492B0F8542007
:109790000D48DFF858E002700A4A1170084A9FE746
:1097A00005980370049B19709EF80010A1E700BF94
:1097B0003404002082050020850500207C0500205F
:1097C0002C030020330300207E0500208B050020A1
:1097D000840500208A050020300300208605002033
:1097E0002E030020380500208005002032030020D1
:1097F000003018BF01204042704700BFF0B511494A
:10980000DFF864E0104F114E114D124C124A002344
:10981000AEF800303B8033802B7023800B801380A8
:1098200038B90E4A012111700D4A03461370002009
:10983000F0BD0C4A09491370094A0B7001231370DB
:109840000020F0BD34040020860500202E030020F7
:109850003805002080050020820500207C050020BE
:10986000850500208A0500203003002010B504463D
:10987000FFF7A4FD0CB1002010BD034B1878003099
:1098800018BF012010BD00BF850500202DE9F04F55
:10989000DFF8648198F8003083B0002B69D04F4C1A
:1098A00023889BB23E2B074668D9DFF84091DFF84A
:1098B0004CB14B4D4B4ED9F8E435002B4AD0FEF756
:1098C000A5F89BF80030002B3FD123889BB2002BDA
:1098D0003BD098F80030002B37D0404B1B889BB210
:1098E000102B4FF0010368D83C4AB2F800E08BF827
:1098F000003013881FFA8EFECEEB03039BB20FFAE3
:109900008EFE1380BEF1000F4FEA8E03019316DD29
:1099100000213548DFF8DCC08A462A882B880133CD
:109920009BB292B23F2B01F101015CF822202B8007
:1099300088BFA5F800A0714540F8042BEDDB019B22
:109940002A48294A812104F0DDFAFEF773F898F8D5
:10995000003073B1234B1A88194642F20F739A42B2
:1099600038D823889BB201323E2B3280A3D88A4656
:1099700006E04FF0FF3003B0BDE8F08FDFF864A0E1
:10998000FEF744F81A4A1B4813889BB2591C89B247
:109990001180118840F823708BB23F2B84BF0023C5
:1099A0001380238801339BB22380FEF743F8002005
:1099B000AAF8000003B0BDE8F08F8BF80030074B29
:1099C000064A1B88103B9BB21380402301934FF043
:1099D000100E9DE76FF00100CDE700BF800500206D
:1099E00082050020880500203C05002098A8002062
:1099F0003404002034030020850500207C0500206D
:109A000038B5114C23889BB2D3B10546FDF7FEFF54
:109A10000E4A0F481188138801339BB23F2B1380E5
:109A200084BF00231380238889B2013B50F82110A2
:109A300029609BB22380FDF7FDFF208880B238BDEE
:109A40004FF0FF3038BD00BF300300202E03002050
:109A5000380400202DE9F84F534D284603F01EFA34
:109A6000002840F08C80D5F8E435002B00F084808D
:109A7000DFF85C81FDF7CAFF98F80030002B3CD07E
:109A8000D5F8DC43C4F38F04002C36D0DFF84491C2
:109A9000B9F800309BB2C3F1400322B29A422CDAEB
:109AA000DFF80CB1414FDFF830A15BF8046BC6F36F
:109AB000031010303146FBF7E3F9013CA4B222B2A7
:109AC00080B939883B8801339BB23F2B3B8088BFEC
:109AD0003880B9F8003089B201339BB24AF821606E
:109AE000A9F80030002AE0DC002388F800302E4876
:109AF0002F4A0221402304F0DFF9FDF79BFFD5F840
:109B0000E435002B38D0FDF781FF2A4B1A78002A64
:109B100030D129490A8892B262B3284A12784AB3EE
:109B20000A8892B2102A4FF001022FD91A700B88BE
:109B3000103B9BB20B8010264023214C214D224F1D
:109B40000020A446864621882288013292B289B23A
:109B50003F2A00F1010057F82110228088BFACF89D
:109B600000E0B04245F8041BEDDB0F48154A8121A7
:109B700004F0C8F9FDF75EFF0020BDE8F88F284625
:109B8000124902F03DF90020BDE8F88F0E881A70E6
:109B90000B88B6B29B1B36B29BB2002E0B804FEAED
:109BA0008603CADCE1E700BF98A8002086050020F4
:109BB00058A800207C050020800500208505002095
:109BC000820500203C050020340300202CB3002037
:109BD000380500203003002038040020F8B5284B59
:109BE000284CD3F8E43500222270002B39D0FDF741
:109BF0000DFF2378002B30D1234A13889BB263B327
:109C0000224B1B784BB313889BB2102B4FF00103F0
:109C100028D923701388103B9BB213801026402351
:109C20001B4C1C4D1C4F0020A446864621882288D0
:109C3000013292B289B23F2A00F1010057F8211097
:109C4000228088BFACF800E0B04245F8041BEDDB91
:109C50000B48104A812104F055F9BDE8F840FDF7A2
:109C6000E9BEF8BD168823701388B6B29B1B36B2C6
:109C70009BB2002E13804FEA8603D1DCE8E700BFD9
:109C800098A800207C050020800500208505002084
:109C9000820500203C050020340300202DE9F04718
:109CA000254C264DD4F8E43501222A70002B40D0F3
:109CB000FDF7ACFE2B78002B37D0D4F8DC43C4F38F
:109CC0008F04002C31D01E4F3B889BB2C3F1400360
:109CD00022B29A4229DADFF870A01A4EDFF86C80BF
:109CE0005AF8049BC9F3031010304946FBF7C8F833
:109CF000013CA4B222B270B93188338801339BB2DF
:109D00003F2B338088BF30803B8889B201339BB2C0
:109D100048F821903B80002AE2DC00232B700648A3
:109D2000094A0221402304F0C7F8BDE8F047FDF7D7
:109D300081BEBDE8F08700BF98A80020380500204C
:109D4000300300208605002058A800203804002099
:109D50002DE9F047044686B0002840F0AE80584810
:109D6000DFF87C910221072200F0F2FF5448032122
:109D7000072200F0EDFF53480821072200F0E8FF1A
:109D8000072209214F4800F0E3FF684600F0D2FFA8
:109D9000012502264FF00408694649488DF8046001
:109DA0008DF80540CDF800808DF8065000F06EFF6C
:109DB0004FF48073694643488DF8046000938DF832
:109DC000065000F063FF082369463D488DF80460A3
:109DD00000938DF8075000F059FF4FF40073694667
:109DE0003848009306AF00F051FF2946302001F0BB
:109DF0007BF847F6122629464FF4F01001F068F878
:109E000047F8106D4FF00C0A39462F48ADF80C405A
:109E1000ADF80E40ADF81040ADF81440ADF812A00A
:109E200001F042FA394629480296C9F80060ADF8B7
:109E300012A0ADF80C40ADF80E40ADF81040ADF8F2
:109E4000144001F031FA41462620C9F80460FDF7BC
:109E500005FE2A461C481E4F1E4E40F2255101F0B9
:109E600093FA41462720FDF7F9FD2A46174840F2AC
:109E7000255101F089FADFF86CC0DFF86CE0164A72
:109E8000164B11488CF8004029468EF800403C7073
:109E9000347014701C708CF801408EF801407C7096
:109EA000747054705C7001F061FA0848294601F042
:109EB0005DFA204606B0BDE8F0874FF0FF30F9E7C5
:109EC00000000240000C02400044004000480040F6
:109ED000940500209C060020A80600208C05002088
:109EE000A0060020900500209806002001281CD81C
:109EF00070B5114E335CDBB10446FDF787FD0F4AA8
:109F00000F48115D135D0133DBB23F2B135584BF46
:109F10000023135501EB8411335D455C013BDBB23B
:109F20003355FDF787FD284670BD4FF0FF30704771
:109F30006FF0010070BD00BF900500209405002067
:109F40001806002001284BD82DE9F84F264D2B5C30
:109F500013443F2BFBDC16468A460446FDF756FDAC
:109F60008EB32248224FDFF88C90DFF88C80721E6F
:109F70001AFA82F20AF1FF318446A6014FF0000E70
:109F800001E091421FD010F804A0035D11F801BF59
:109F90000133DBB23F2B035588BF0CF804E02B5D87
:109FA0000133DBB2B244012B07F80AB02B55E8D1DC
:109FB000012C0DD1B9F80C309BB243F080039142D3
:109FC000A9F80C30DFD1FDF735FD0020BDE8F88F92
:109FD000B8F80C309BB243F08003A8F80C30D0E7FF
:109FE0004FF0FF30704700BF9C060020A8060020FD
:109FF000980500200048004000440040284B1A8883
:10A00000910670B52AD4264B1A8812061ED5254C07
:10A010002278E2B12278BAB1FDF7F8FC224A23484F
:10A0200011781378455C0133DBB23F2B137084BF8A
:10A03000002313702378013BDBB22370FDF7FAFC99
:10A04000174BADB29D8070BDFF229A8070BD9A897A
:10A0500022F080021204120C9A8170BD9C88E4B236
:10A0600021462020FAF700FF05460028CBD1104EEC
:10A0700033783F2BC7D8FDF7C9FC0E4A0E4811783C
:10A08000137844540133DBB23F2B137088BF157033
:10A0900033780133DBB23370FDF7CCFCB3E700BF9C
:10A0A000004400409C0600208C05002098050020FC
:10A0B0009005002098060020180600202A4B1A88D8
:10A0C000910670B52CD4284B1A88120620D5274C3F
:10A0D0006278F2B16278CAB1FDF798FC244A25484B
:10A0E000517853780133DBB23F2B537084BF002388
:10A0F000537063780144013BDBB291F840506370C8
:10A10000FDF798FC184BADB29D8070BDFF229A8080
:10A1100070BD9A8922F080021204120C9A8170BDDF
:10A120009C88E4B221462120FAF79EFE05460028CD
:10A13000C9D1114E73783F2BC5D8FDF767FC0F4A84
:10A140000F48517853780133DBB23F2B537088BFEF
:10A150005570737801440133DBB281F8404073706D
:10A16000FDF768FCAFE700BF004800409C060020F8
:10A170008C050020980500209005002098060020FE
:10A18000180600205C4B19688A8A088B92B2D007A7
:10A1900010B40FD55A69920771D51A7D6FF300027A
:10A1A0001A758B885DF8044B23F4E0631B041B0CC9
:10A1B0008B80704702F0020080B218B31A7912F057
:10A1C000010F1A8A92B25FD1002A6DD0588A1A8A7A
:10A1D00080B292B2904208D29A682AB1588A80B26C
:10A1E000441CA4B25C82125C0A825A8A1B8A92B214
:10A1F0009BB29A4245D38B8823F480631B041B0CCB
:10A200008B803EE002F08404802C40D0842C5FD010
:10A21000540636D5D868002833D00C8A598A1A8A51
:10A2200089B292B29142E4B205D25A8A92B2511CDA
:10A2300089B25982845459692F4A88072ED4508A8A
:10A24000118A89B280B20139884207DA5169490717
:10A2500017D5528A92B2012A13D194B919680A8883
:10A2600022F480621204120C0A800A8892B242F42C
:10A2700000720A801A7D42F002021A7501E01B7911
:10A280000B825DF8044B7047012AFAD1E7E7588A40
:10A290001A8A80B292B290429ED3F2E7137D11687F
:10A2A0006FF3000313757CE7088880B240F40070F8
:10A2B0000880187D40F002001875888820F4E0605E
:10A2C0000004000C8880197D62F300011975D8E73D
:10A2D0000A8892B242F400720A801A7D42F00202A9
:10A2E0001A758A8822F4E0621204120C8A801A7DA0
:10A2F00060F300021A75C4E7AC06002038B51A4CAA
:10A30000206800F051FD194B034005461BBB184B5C
:10A310002B40C3B9174B2B4053B12068164900F0AE
:10A320004BFD6FF006032068A361012100F024FDBE
:10A3300020684FF4E061002200F02CFD237D6FF3D4
:10A340000003237538BD20680C4900F035FD6FF01F
:10A350000403A361DEE720684FF0012100F02CFD2B
:10A360006FF00503A361D2E7AC06002000010010E6
:10A3700000020010000400100004000100020001AF
:10A38000644B596A8A8A088B92B2D00710B411D5EF
:10A390009A6B920776D593F838206FF3000283F812
:10A3A00038208B885DF8044B23F4E0631B041B0CFE
:10A3B0008B80704702F0020080B220B393F828200F
:10A3C00012F0010F9A8E92B262D1002A72D0D88E0A
:10A3D0009A8E80B292B2904208D2DA6A2AB1D88EAE
:10A3E00080B2441CA4B2DC86125C0A82DA8E9B8E98
:10A3F00092B29BB29A4248D38B8823F480631B04A9
:10A400001B0C8B8041E002F08404802C43D0842C10
:10A4100068D0540639D5186B002836D00C8AD98EEE
:10A420009A8E89B292B29142E4B205D2DA8E92B299
:10A43000511C89B2D9868454996B364A880731D425
:10A44000D08E918E89B280B20139884207DA916B41
:10A4500049071AD5D28E92B2012A16D1ACB9596ADF
:10A460000A8822F480621204120C0A800A8892B2CE
:10A4700042F400720A8093F8382042F0020283F816
:10A48000382002E093F828300B825DF8044B7047C7
:10A49000012AFAD1E4E7D88E9A8E80B292B2904225
:10A4A0009BD3F2E792F83830516A6FF3000382F8D9
:10A4B000383076E7088880B240F40070088093F85E
:10A4C000380040F0020083F83800888820F4E0600B
:10A4D0000004000C888093F8381062F3000183F8C0
:10A4E0003810D2E70A8892B242F400720A8093F8D8
:10A4F000382042F0020283F838208A8822F4E06291
:10A500001204120C8A8093F8382060F3000283F85A
:10A510003820BAE7AC06002038B51B4C606A00F062
:10A5200043FC1A4B034005462BBB194B2B40D3B9B8
:10A53000184B2B4053B1606A174900F03DFC6FF097
:10A540000603606AE363012100F016FC606A4FF4C1
:10A55000E061002200F01EFC94F838306FF3000335
:10A5600084F8383038BD606A0C4900F025FC6FF083
:10A570000403E363DCE7606A4FF0012100F01CFC98
:10A580006FF00503E363D0E7AC0600200001001084
:10A59000000200100004001000040001000200018D
:10A5A0002DE9F843B2F100080446894656DD0D78DE
:10A5B000002D4FD08C4600271CF8012F0137002AB0
:10A5C000FAD1B845D8BF904645DC13F0020F14BF4E
:10A5D0003027202713F0010318BF002627D0294673
:10A5E0005DB1DCB123684846197023680136013338
:10A5F000236010F8011F0029F6D1B8F1000F0ADD21
:10A6000084B3236845461F702368013D03F10103AD
:10A610002360F8D146443046BDE8F8830120FAF7BC
:10A6200035FF19F8011F01360029F7D1E5E7B8F128
:10A63000000F1FDD04B3236842461F702368013AF0
:10A6400003F101032360F8D1464699F800504FF01A
:10A650000008C4E72F46C7EB0808B6E72027002606
:10A660000D78BCE7444601203946FAF70FFF013C5C
:10A67000F9D1CFE71E46B2E7454601203946FAF741
:10A6800005FF013DF9D1DFE72DE9F04685B00D4624
:10A690000C4681460C9E00294DD0003318BF012383
:10A6A0000A2A18BF0023002B38D100218DF80B1087
:10A6B000002C4DD00E990DF10A05A1F13A0EB4FB14
:10A6C000F2F102FB11440EEB0407092CD8BF274618
:10A6D0003037AA460C4605F801790029EFD11C460F
:10A6E0004BB94846514632460D9BFFF759FF20446F
:10A6F00005B0BDE8F086BEB10D9B9B0714D5B9F13E
:10A70000000F28D0D9F800302D221A70D9F8003067
:10A710000133C9F80030013E0124E2E70029BABF45
:10A720004C4201230023C0E72D230AF8013C0024FA
:10A730000AF1FF3AD5E732460D9B302469468DF881
:10A7400001508DF80040FFF72BFF05B0BDE8F08603
:10A750000DF10B0AC3E72D210120FAF797FEDAE786
:10A760002DE9F0470D46097888B006460592002984
:10A7700000F0AB804FF0000A41F6B407D146C0F6B6
:10A7800004074FF06108252944D168786C1C002823
:10A7900037D025283DD02D2803BFA878AC1C012335
:10A7A0000023302808D1621C10781446302843F06A
:10A7B000020302F10102F7D0A0F13001CAB2092A66
:10A7C0004FD8651C00222C4615F8010B02EB8202C3
:10A7D00001EB4202A0F130015FFA81FCBCF1090FEC
:10A7E000F1D9732820D064282ED078283BD058285F
:10A7F00046D075284DD0632858D06178651C002953
:10A80000C1D116B1336800221A70504608B0BDE8B5
:10A81000F0872546A6B13268117033680133336082
:10A820000AF1010A2C46E8E705980168051D002990
:10A8300008BF394630460595FFF7B2FE8244DCE793
:10A840000120FAF723FEEBE7059D304629688DE8E5
:10A850000C0104350A2201230595FFF715FF8244F8
:10A86000CBE70022BDE7059D304629688DE80C0145
:10A870000435102200230595FFF706FF8244BCE74C
:10A8800005984FF0410E0168051D8DE80C403046DB
:10A89000EFE7059D304629688DE80C0104350A2252
:10A8A00000230595FFF7F0FE8244A6E705993046A0
:10A8B000D1F800E00D1D07A98DF81D908DF81CE062
:10A8C0000595FFF76DFE824497E78A4699E700BF3A
:10A8D0000EB400B584B005AB53F8041B01901A46C2
:10A8E00001A80393FFF73CFF04B05DF804EB03B04D
:10A8F000704700BF00B583B002AB43F8040D1846A3
:10A90000FFF72EFF03B05DF804FB00BF40F0BF600F
:10A91000024B40F40030D860704700BF00ED00E00B
:10A9200021F0604121F07F01014B0843986070479E
:10A9300000ED00E0F0B544680A6891F804C0D1F871
:10A940000CE00E698D684F790D4B24F0407424F4AF
:10A950008074224342EA0C22426084684EEA060276
:10A960002A432340134343EA470383600A7DC36AB3
:10A97000013AD2B223F4700343EA0253C362F0BD3A
:10A98000FDF7FFC0002301220275036003714371CC
:10A990008360C3600361704770B490E84400064D63
:10A9A0008468C168054B6868324322430A43034008
:10A9B00013436B6070BC704700230140E030FCFF24
:10A9C0000023036043608360C3607047836819B9E4
:10A9D00023F001038360704743F0010383607047F5
:10A9E000092970B41CD9A1F10A0404EB4404C56818
:10A9F0000726A640A34025EA06042343062AC3608F
:10AA00001AD90C2A25D90D3AC46A02EB82021F23F7
:10AA1000934024EA030391401943C16270BC70471C
:10AA200001EB410605690724B440B34025EA04045C
:10AA30002343062A0361E4D8013A446B02EB820205
:10AA40001F23934024EA030391401943416370BCE0
:10AA50007047073A046B02EB82021F23934024EAFB
:10AA6000030391401943016370BC7047836843F04E
:10AA700080438360704700BF836819B923F48073F3
:10AA80008360704743F4807383607047054A53685E
:10AA900018B923F400535360704743F400535360D4
:10AAA000704700BF00230140F0B491E8C000094D99
:10AAB0008C68CB682A6847EA06010C4340F6FE71B1
:10AAC00023438140834022EA010213432B60F0BC00
:10AAD000704700BF0074004039B9074901230A6874
:10AAE000834022EA03030B607047034901230A688D
:10AAF000834013430B6070470074004041B908491C
:10AB000000094A680123834022EA03034B6070472F
:10AB1000034900094A680123834013434B6070478F
:10AB20000074004082B00022054B01920193019B0A
:10AB3000083318440190019B196002B0704700BFB0
:10AB40000074004082B00022054B01920193019BEA
:10AB5000143318440190019B196002B0704700BF84
:10AB6000007400402DE9F04182B08B6A0193CB68FC
:10AB70004F698E69CD690C6A4A6AD0F800C0DFF867
:10AB800050E098460B6848EA030848EA07073E4346
:10AB900035432C43019B0E6B0D69224313434A6BD3
:10ABA0004C6813438A6B0CEA0E0E134343EA0E0300
:10ABB00003604269CB6A896822F00702334313437A
:10ABC000436145608460C16002B0BDE8F08100BFB0
:10ABD0003F801CF00023036043608360C360036117
:10ABE00043618361C361036243628362C36203633F
:10ABF00043638363704700BF036819B923F00103FF
:10AC00000360704743F001030360704710B4094BC1
:10AC1000094C0A4AA04294BF1846104611F0005F42
:10AC200021F0F02121F0821114BFC16081605DF834
:10AC3000044B7047006002400F6402400064024011
:10AC40000B060CD54369AAB143F080038029436108
:10AC50000FD0036801F01E0119430160704780297D
:10AC600007D0002AF5D1036801F01E0123EA010193
:10AC70000160704723F0800380294361F3D170475E
:10AC8000014B5861704700BF003C014000222DE994
:10AC9000F0471346D1F800E001274FF0030C04E021
:10ACA0000133102B02F1020229D007FA03F404EA5F
:10ACB0000E05A542F4D104680E79D44004F00304D3
:10ACC000B4420CFA02F806F1FF3A07D0046824EA0D
:10ACD000080404600468964026430660BAF1010F38
:10ACE0000FD9C568CC7925EA0805C560C5689440C8
:10ACF00001332C43102BC46002F10202D5D1BDE810
:10AD0000F087866891F805908C790CFA02FA26EAA9
:10AD10000A068660866809FA02F949EA060686602C
:10AD2000466826EA0505456045689C40A4B22C4368
:10AD30004460D6E700234FF6FF720260037143714F
:10AD40008371C371704700BF0183704741837047AF
:10AD5000CB0800EB830001F0070110B48900046AFE
:10AD60000F238B4024EA03030362036A5DF8044B5C
:10AD70008A40134303627047038829B923F40073A0
:10AD80001B041B0C038070479BB243F400730380C9
:10AD9000704700BF83889BB21AB923EA0101818002
:10ADA0007047194381807047838A028B98B240EACA
:10ADB000024020F07F407047C94389B281827047CA
:10ADC000014B1860704700BF20000E4210B4214CA8
:10ADD000A36803F00C03042B1BD0082B1CD01E4BC4
:10ADE00003601C4A1D499468C4F303140C5DE340DE
:10ADF00043609468C4F382240C5D23FA04F48460F5
:10AE000092685DF8044BC2F342328A5CD340C3605F
:10AE10007047134B0360E4E76368616813F4800FC5
:10AE2000636818BF0E4C01F03F020CBF0A49B4FB27
:10AE3000F2F1C3F3881308BFB1FBF2F101FB03F297
:10AE4000044B5B68C3F3014301335B00B2FBF3F3D4
:10AE50000360C6E7003802400024F40040000020F0
:10AE600000127A0000F44073B3F5407F09D108491D
:10AE70008B6820F0704223F4F81322F440721343DD
:10AE80008B60034A136FC0F30B00184310677047C1
:10AE900000380240014B1860704700BF3C0E47422B
:10AEA000044A136B19B923EA000010637047184372
:10AEB0001063704700380240044A536B19B923EA03
:10AEC00000005063704718435063704700380240D9
:10AED000044A136C19B923EA000010647047184340
:10AEE0001064704700380240044A536C19B923EAD1
:10AEF00000005064704718435064704700380240A7
:10AF0000044A136919B923EA000010617047184315
:10AF10001061704700380240044A536919B923EAA6
:10AF2000000050617047184350617047003802407C
:10AF3000044A136A19B923EA0000106270471843E3
:10AF40001062704700380240044A536A19B923EA74
:10AF5000000050627047184350627047003802404A
:10AF600010B41E4983B00023CA2453224C624A62A3
:10AF70000193CB685B0615D44FF0FF33CB6000E044
:10AF80004AB9CA68019B01330193019BB3F5803F25
:10AF900002F04002F4D1114BDB6813F0400301D101
:10AFA000184614E00D4B9A6822F040029A609968A6
:10AFB00002680A439A6082681A6141681A6942EA23
:10AFC00001421A61DA6822F08002DA600120034B44
:10AFD000FF225A6203B05DF8044B7047002800401E
:10AFE00000217F22FF2380E80E00704730B4504BD1
:10AFF00082B0002836D19D6815F0400566D1CD702D
:10B000000A78092A4FF0000407D90A3AD2B201346B
:10B01000092AE4B2F9D82401E4B24B782243092B7F
:10B020004FEA02404FF0000207D90A3BDBB201327F
:10B03000092BD2B2F9D81201D2B289781343092967
:10B040004FEA032272D900230A39C9B20133092910
:10B05000DBB2F9D81B01DCB240EA050313432143FC
:10B0600019430CE09A6812F040022CD1CA7048785B
:10B070000B788978000240EA0343194311432C4CB2
:10B080000023CA205322606262620093E3685B0679
:10B090001FD44FF0FF33E36000E048B9E068009A46
:10B0A00001320092009AB2F5803F00F04000F4D1E6
:10B0B0001F4BD86810F040000BD11D4BFF225A6285
:10B0C00002B030BC7047CA781204D0E7CD782D04A6
:10B0D00096E7174A01F07F3121F0FE411160D368F5
:10B0E000532123F080030024CA20D36001945062CE
:10B0F0005162D36823F0A003D360114600E04AB93F
:10B10000CA68019B01330193019BB3F5003F02F034
:10B110002002F4D1064BD86810F0200002D1FF22A3
:10B120005A62CAE7FF225A620120C6E7002493E769
:10B13000002800400023C370037043708370704781
:10B140002DE9F0410B88B1F80280B1F804C0CA883B
:10B15000B1F808E04F898E89CC890588098A48EAC8
:10B16000030343EA0C03134343EA0E033B43334315
:10B1700043EA040205F4415313439BB20380838BDB
:10B1800023F400631B041B0C83830182BDE8F08160
:10B19000038829B923F040031B041B0C038070476C
:10B1A0009BB243F040030380704700BF83889BB28B
:10B1B0001AB923EA010181807047194381807047E1
:10B1C000224A038890429BB212D002F580629042DC
:10B1D0000ED0B0F1804F0BD0A2F58032904207D054
:10B1E00002F58062904203D002F58062904203D162
:10B1F0004A8823F070031343154A90421ED002F58B
:10B20000806290421AD00A8970B423F440730F4CC4
:10B210004E680D889BB21343A0420380C662058529
:10B2200006D00C4B984203D00123838270BC704738
:10B230008B7A03860123838270BC704703800B885E
:10B240004A68C2620385012383827047000001407F
:10B250000010004000040140038829B923F00103D5
:10B260001B041B0C038070479BB243F00103038057
:10B27000704700BF83899BB21AB923EA010181811B
:10B280007047194381817047038A828911EA03005C
:10B2900092B203D0114214BF01200020704700BFBA
:10B2A000C94389B201827047028A8B88F0B592B295
:10B2B000CE880F8904460D4622F440523243A889B5
:10B2C00049892282A2893B4392B20B4322F4B052B5
:10B2D00022F00C029BB21343A381A38A9BB223F4F6
:10B2E0004073034385B0A3826846FFF76FFD1D4B93
:10B2F0009C4229D003F580639C4225D0029AA38901
:10B30000A6891BB2002B2B6802EB8202B4BF5B0044
:10B310009B0002EB8202B2FBF3F0134A36B2A2FBAF
:10B3200000356D096423002E05FB13034FEA051554
:10B330000CDB1B013233A2FB0323C3F343132B4368
:10B340009BB2238105B0F0BD039AD8E7D900323112
:10B35000A2FB0131C1F3421242EA05039BB22381F1
:10B3600005B0F0BD001001401F85EB51838929B95C
:10B3700023F400531B041B0C838170479BB243F4DE
:10B3800000538381704700BF10B401F01F04C1F364
:10B3900042110123012903FA04F311D002290CBF41
:10B3A0001030143032B902685DF8044B22EA03030E
:10B3B0000360704702685DF8044B134303607047F5
:10B3C0000C30EFE710B5D0F8E83504461B69984714
:10B3D000032384F81231002010BD00BF08B50422F9
:10B3E00090F81211D0F8E83580F8131180F8122186
:10B3F000DB689847002008BD08B5D0F8E435DB6964
:10B4000003B19847002008BD08B5D0F8E4351B6AA1
:10B410009847002008BD00BF08B5D0F8E4355B6A46
:10B420009847002008BD00BF002110B50B46044618
:10B43000402202F0F5FC802120464022002302F049
:10B44000EFFC0122D4F8E83584F81221A0785B687B
:10B450009847002010BD00BF10B582B06946044671
:10B4600000F052FB9DF8001001F01F03012B18D0D3
:10B4700010D3022B07D0204601F0800102F068FDB6
:10B48000002002B010BD2046694600F0D3FA00202B
:10B4900002B010BD2046694600F012F9002002B04B
:10B4A00010BD2046694600F0A3FA002002B010BD8E
:10B4B00038B5044649B990F81131022B19D094F8E7
:10B4C0001631012B0CD0002038BDD0F8E4355B6973
:10B4D000002BF8D090F81221032AF4D19847F2E714
:10B4E000204A236912685A60002384F8163100202C
:10B4F00038BDD0F83821D0F824319A4210D9C1781B
:10B500000129D0F82811A2EB030208BFC918C0F81E
:10B51000382108BFC0F8281192B200F0A1F8CEE798
:10B52000D0F83C21B2FBF3F503FB15255DB993423E
:10B5300009D8D0F840319A4205D22A4600F090F856
:10B54000C4F84051BBE7D4F8E435DB681BB194F88C
:10B550001221032A03D0204600F0A2F8AFE72046CC
:10B560009847F8E7B0B3002010B5044629B990F821
:10B570001131032B0CD0002010BDD0F8E4359B69AD
:10B58000002BF8D090F81221032AF4D19847F2E763
:10B59000D0F89023D0F87C339A4212D9C17801298F
:10B5A000D0F88013A2EB030204BFC918C0F88013BF
:10B5B0009A42C0F8902328BF1A4692B200F058F879
:10B5C000D9E7D0F8E4351B691BB190F81221032AA2
:10B5D00003D0204600F054F8CDE79847F9E700BFC4
:10B5E0002DE9F0410446164698460D46069FFDF7A4
:10B5F000A5FD20462946C4F8E485C4F8E875C4F8DA
:10B60000EC6502F0D3F9D4F8E8351B68984720467A
:10B61000BDE8F041FDF7E2BDD0F8E43510B50446D1
:10B620001B689847D4F8E8359B689847002010BD00
:10B6300008B5D0F8E4355B689847002008BD00BF26
:10B6400038B5134602250A46C0F83C31C0F83831F7
:10B6500080F81151002102F055FC002038BD00BFD8
:10B6600008B513460A46002102F04CFC002008BD34
:10B6700008B513460A46002102F01EFC002008BD52
:10B6800010B50021042304460A4680F811310B4608
:10B6900002F038FC204602F067F9002010BD00BF20
:10B6A00010B50021052304460A4680F811310B46E7
:10B6B00002F002FC204602F057F9002010BD00BF46
:10B6C00030B54B78052BA1B00D4604465DD01BD993
:10B6D000082B00F098806BD9092B37D0552B59D106
:10B6E0000B78C02B56D14B88002B53D1CD88802DA1
:10B6F00050D12A466846B54924F0A4FA2046694646
:10B700002A46FFF79DFF0BE0012B69D00BD3032BDB
:10B7100040D14B88012B00F04081022B00F01181B9
:10B72000002021B030BD90F81231023B012B32D8FD
:10B73000A74BD0F81821002119600AB102221A6023
:10B740002046A3490222FFF77BFFE9E78978A14D54
:10B75000012929701ED890F81231022B7BD0032BBF
:10B7600019D1002900F0278190F81011012900F06B
:10B770001A81FFF75DFF297884F810112046FFF742
:10B780004BFF2046FFF77CFFCAE78B8813B9CB88B5
:10B79000002B46D02046802102F0DAFB0021204613
:10B7A00002F0D6FB204602F0DFF8002021B030BDC9
:10B7B000062BEFD149880B0A013B062BEAD801A2E0
:10B7C00052F823F0C3B8010887B8010875B801081A
:10B7D00095B7010895B7010895B7010895B7010815
:10B7E00090F81231023B012BD5D84B88012B97D111
:10B7F000D0F8E43500229B68C0F81821984720460D
:10B80000FFF73EFF8CE7CA88012AC3D190F81231B6
:10B81000022B1CD0032BBED100F58871FFF710FF5F
:10B820007EE790F812318D78032B05F07F05B1D0BB
:10B8300080F81451294602F0C7FB2046FFF720FF8D
:10B84000002D00F0B480022384F8123168E76249C9
:10B85000FFF7F6FE64E7002900F0A580012103232D
:10B8600080F8101180F81231FFF7D6FE2046FFF75E
:10B8700007FF55E7C9B2052900F2B280DFE801F001
:10B88000595149413931D0F8E43580789B6A69468D
:10B890009847022343700146C4F8F005BDF8002024
:10B8A000002A3FF43DAFEB88002B3FF439AF9342C1
:10B8B00028BF13461A462046ADF80030FFF7C0FEF9
:10B8C0002EE7D0F8EC3580781B6869469847EB88FE
:10B8D000402B014603D094F81221012ADED1082220
:10B8E000E2E7D0F8EC3580789B69694698470146D5
:10B8F000D4E7D0F8EC3580785B6969469847014613
:10B90000CCE7D0F8EC3580781B696946984701464A
:10B91000C4E7D0F8EC358078DB6869469847014683
:10B92000BCE7D0F8EC3580789B68694698470146BB
:10B93000B4E7D0F8EC3580785B68694698470146F3
:10B94000ACE78B8813F0FF0F7FF4EAAE1B0A0269A5
:10B95000013B5268042B07D8DFE803F01B17130FD5
:10B960000300052363F306121C4B012184F8161112
:10B9700020461A60FFF784FED2E6042363F3061222
:10B98000F2E7032363F30612EEE7022363F30612E2
:10B99000EAE7012363F30612E6E7D0F8E425C0F8EE
:10B9A0001831936898472046FFF76AFEB8E60123EE
:10B9B00084F81231B4E6022380F8101180F81231B5
:10B9C000FFF736FE2046FFF75BFEA9E6BC18040829
:10B9D000F4060020F806002000070020B0B3002085
:10B9E000D0F8E4358078DB6A6A469847014655E727
:10B9F00038B590F81231032B044603D10B79012B93
:10BA00000D460BD9802102F0A3FA2046002102F056
:10BA10009FFA204601F0A8FF002038BDD0F8E43599
:10BA20009B689847EB88002BF6D12046FFF728FE4D
:10BA3000F2E700BF38B54B788A88012B0C460546E3
:10BA4000D1B222D018D3032B14D190F81231022B8B
:10BA500016D0032B3BD163881BB94A0601D002F0F4
:10BA600077FAD5F8E43521469B682846984728465A
:10BA7000FFF706FE002038BD90F81231022B12D1DC
:10BA80004A06F7D002F064FAF4E790F81231022B7C
:10BA9000F6D0032B1BD16388002BEBD14B06E6D0ED
:10BAA00002F074FADDE7032B11D113061BD401EB6E
:10BAB000810100EBC10191F87633F3B9114B0022FB
:10BAC0001A6028460F490222FFF7BAFDD2E780210B
:10BAD00002F03EFA0021284602F03AFA284601F028
:10BAE00043FF002038BD01F07F0101EB810100EB35
:10BAF000C10191F81E31002BE0D0024B01221A60E7
:10BB0000DFE700BFFC06002090F8CC350B7090F802
:10BB1000CD354B7090F8CF2590F8CE3503EB02234E
:10BB20004B8090F8D12590F8D03503EB02238B8021
:10BB300090F8D32590F8D23503EB02239BB2012273
:10BB4000CB80C0F8403180F81121704700B30378F2
:10BB500030B4F3B10446002314F8015F0133DBB2C3
:10BB6000002DF9D15B000233DCB2032513800C7089
:10BB70004D7004785CB1022300255A1CD2B2CC541B
:10BB80008D5410F8014F0233DBB2002CF5D130BCDC
:10BB9000704702242346E8E70123C0F8F437002069
:10BBA000704700BF0023C0F8F4371846704700BF45
:10BBB000002070472DE9F041069F144605460E46C9
:10BBC0009846FDF7BBFA0020FDF730FB002240232A
:10BBD0000121A37122706270A27084F82020E170AC
:10BBE000217784F821102846217900F093FB6179B0
:10BBF000284600F08FFB3146C4F87C80C4F8807082
:10BC0000284602F0B9FCD4F880301B6898472846D3
:10BC1000BDE8F041FDF7E2BA0B7F0022013B70B5B1
:10BC20000C468A7405460A2B00F28D80DFE803F08B
:10BC3000141C2A334B5A678E708206008B7B0133AB
:10BC4000DBB2022B8B7340F2A3804B780B7008227F
:10BC50008A740223184670BD1431627900F0A8FB83
:10BC6000022323770023F5E7497902F00FFD01282D
:10BC700000F09280032866D105230B22A37422775B
:10BC80000023E7E723798968A28900F0CBFB04232E
:10BC900023770023DEE7097902F0F8FC012800F0A1
:10BCA0008E8004286AD0032808D0284602F0EAFCD7
:10BCB000524A238A1288C01A904244D90B23237710
:10BCC0000023184670BD4B7900EB4313012283F823
:10BCD000A92863798968A28900F07EFB062323776F
:10BCE0000023B7E7497902F0D1FC01286AD0042883
:10BCF00070D0022825D1052323770023AAE700214D
:10BD000023790A4600F08EFB082323770023A1E75E
:10BD10004B7900EB4313002193F8A92882F001022C
:10BD200083F8A92863790A4600F056FB0A23237793
:10BD300000238FE7497902F0A9FC012822D00228CC
:10BD400044D00328BAD00023184670BD097902F008
:10BD50009DFC0128064615D00328AFD0284602F0E6
:10BD600091FC264A238A1288C01A9042A6D8042E33
:10BD7000E9D163782370A67403236BE7637823709B
:10BD8000002367E7637823700D232377002361E79F
:10BD900001230B7700235DE7237D628B23F07F0374
:10BDA000DBB2EAB1154A41F288311180FBB90523B3
:10BDB0002377284602F066FC002320824AE7092305
:10BDC000237772E707232377002343E709232377A9
:10BDD00000233FE7637823700C232377002339E7A0
:10BDE000064A322111802BB907232377E1E7032389
:10BDF0002377DEE709232377DBE700BF0407002072
:10BE000070B594B002260C468DF80F60054602F01E
:10BE100035FC237868BB002B46D0B34200D0267097
:10BE2000D4F880301B699847002601234022A27174
:10BE3000E370237784F82130217926706670A6702C
:10BE400084F82060284600F065FA6179284600F001
:10BE500061FAD4F880305B689847E36F28465B68E6
:10BE600004F120019847284600F060FA267014B0CB
:10BE700070BD0A2BFBD801A252F823F0A9BE01081D
:10BE8000EBBE010821BE01086FBE010861BF0108B9
:10BE90007FBF010899BF0108DFBE0108BFBE0108CE
:10BEA0006FBE0108C9BF0108284602F0E7FB002861
:10BEB000DDD0012323706420FDF7B0F9D7E7D4F873
:10BEC00080309B6B98470128D1D1E36F28461B68CF
:10BED000214698470028CAD105232370C7E7284682
:10BEE0002146FFF799FE14B070BDD4F880309B68EE
:10BEF00098470021284600F0C9F980216071284642
:10BF000000F0C4F92071284602F0B2FB0646002872
:10BF1000ADD1D4F88030DB689847284602F0A2FB08
:10BF2000D4F88030C0B284F8210004229B692270CA
:10BF30009847A079217994F8202094F82130019035
:10BF40000096284600F058F9617994F8202094F87A
:10BF50002130A47901940096284600F04DF986E737
:10BF6000A378092B83D8DFE813F0D900C800FD00BF
:10BF70009100B3009C007A00630057005000E36F0B
:10BF800028469B68214698478DF80F009DF80F3092
:10BF90004BB9062323706AE7E36F2846DB68214626
:10BFA00098478DF80F009DF80F30DBB21A1F012A59
:10BFB00040F20081062B7FF45AAFD4F880300A2279
:10BFC0001B682270984752E7012200234021E2704B
:10BFD000227784F8212023706370A37084F82030C6
:10BFE000A1712846217900F095F96179284600F081
:10BFF00091F9D4F880305B689847E36F28465B6816
:10C0000004F12001984714B070BDD4F880305B6B08
:10C010009847082323702AE72846214694F83920B8
:10C0200000F04CFC00287FF422AF0923A3701EE728
:10C0300094F83220002A00F0C480FF2100912846A5
:10C0400004AB214600F0F4FB00287FF410AFD4F8D5
:10C05000803004A81B6B98470823A37007E794F867
:10C060003120002A00F0BD80FF210091284604AB5A
:10C07000214600F0DDFB00287FF4F9AED4F88030D3
:10C0800004A8DB6A98470723A370F0E628462146F8
:10C09000092200F069FA00287FF4E9AE0423A370B6
:10C0A000E5E694F83020002A00F09380FF2100910B
:10C0B000284604AB214600F0BBFB00287FF4D7AE36
:10C0C000D4F8803004A89B6A98470623A370CEE674
:10C0D00028462146E28E00F047FA00287FF4C7AEDA
:10C0E000D4F8803004F134005B6A04F13E0104F1BD
:10C0F000500298470523A370B9E62846214612222C
:10C1000000F0D4F900287FF4B2AED4F8803004F106
:10C110002200DB6998470223A370A8E6284621463F
:10C12000082200F0C3F9064600287FF4A0AE94F878
:10C130002930A371284602F09BFAA3796179009611
:10C140000122A270284601933246334600F080F85F
:10C15000A37921790193009628463246334600F0B0
:10C1600077F884E628462146012200F099FB06462E
:10C1700000287FF47CAE0220FDF750F80122D4F8AD
:10C18000803084F820201B6A98470323217994F893
:10C190002020009601962846A370334600F058F8F8
:10C1A000617994F82020009601962846334600F0E5
:10C1B0004FF85CE6D4F880305B6C98470A23237014
:10C1C00055E6D4F880300B481B6B98470823A370C2
:10C1D0004DE6D4F8803007489B6A98470623A37041
:10C1E00045E6D4F880300348DB6A98470723A370FC
:10C1F0003DE600BF3C1904082DE9F04100EB410584
:10C2000000EB4114B5F8705A9DF818C0BDF81CE059
:10C2100084F89028264605F07F080027C5F3C0154E
:10C2200084F8918884F8925884F8933884F895C8F3
:10C23000A4F896E804F6880486F8A87886F8A97821
:10C240000BB90123237300F095FF0020BDE8F081B6
:10C2500070B54C01BDF8145012B1061986F890283B
:10C26000021902F68802D689AE4200D05DB90444B4
:10C2700004F68804E27A9A4201D003B1E37200F036
:10C2800079FF002070BDD581F1E700BFB0F9703AA9
:10C29000002B1DDAB0F9723A002B25DAB0F9743AA6
:10C2A000002B24DAB0F9763A002B23DAB0F9783A89
:10C2B000002B22DAB0F97A3A002B21DAB0F97C3A75
:10C2C000002B20DAB0F97E3A002B1FDAFF207047EE
:10C2D0000022134600EB43036FEA41416FEA5141EC
:10C2E000A3F8701A1046704701221346F2E70222A3
:10C2F0001346EFE703221346ECE704221346E9E76F
:10C3000005221346E6E706221346E3E70722134613
:10C31000E0E700BF072907D800EB4100B0F8703A0A
:10C32000C3F30E03A0F8703A00207047002380F892
:10C33000743A80F8753A80F8763A80F8773A80F85F
:10C34000783A80F8793A80F87A3A80F87B3A80F83F
:10C350007C3A80F87D3A80F87E3A80F87F3A184639
:10C36000704700BFC87801280ED002280AD10B7F81
:10C370000D2B18D00B2B13D00C2B03D10123CB701A
:10C38000032070470120704730B40D788A6007247D
:10C3900002224D700C708B810877CA7030BC7047D8
:10C3A0000123CB70704701230020CB7008777047C2
:10C3B000F8B500EB42144FF0000E03260825C4F830
:10C3C0009C1884F892E884F898681146C4F8A0583C
:10C3D00002F060F9C0B2F8BDF8B503F1150400EB46
:10C3E000431500EB44164FF0000E85F892E8C6F8AE
:10C3F000FC15C5F8A02862B9012185F8A918022208
:10C4000000EB4414194684F8F82502F043F90020A3
:10C41000F8BD00EB431292F8A928002A18BF0222A7
:10C42000EEE700BFF8B500EB43152C4601270226C6
:10C43000C5F89C1885F8927885F898681946C4F86C
:10C44000A02802F027F90020F8BD00BFF8B500EBE6
:10C4500043152F4695F8A958C7F89C18002D4FF0A2
:10C46000000618BF022587F89268C7F8A028194669
:10C4700087F8985802F00EF93046F8BDF8B500EB91
:10C480004316354696F8A868C5F89C18002E18BFC4
:10C490000226012785F89278C5F8A028194685F864
:10C4A000986802F0F7F80020F8BD00BFF8B516460E
:10C4B00000234FF480724FF0800E0627CA820B8350
:10C4C0004E8381F814E04F75334600F2F4520C4667
:10C4D0000546FFF747FF00B1F8BD95F8F43584F83D
:10C4E000223095F8F53584F8233095F8F72595F83E
:10C4F000F63503EB0223A38495F8F83584F826304B
:10C5000095F8F93584F8273095F8FA3584F828300D
:10C5100095F8FB3584F82930082EDDD995F8FD25EE
:10C5200095F8FC3503EB0223638595F8FF2595F814
:10C53000FE3503EB0223A38595F8012695F8003616
:10C5400003EB0223E38595F8023684F8303095F842
:10C55000033684F8313095F8043684F8323095F893
:10C56000053684F83330F8BD2DE9F04F0023154629
:10C5700000F2F45A4FF0800E06274FF400760B833A
:10C580008DB052464D8381F814E04F75CE822B4614
:10C5900004468946FFF7E6FE8046002840F00F81FA
:10C5A000002D45D0DFF878E21EF0030F0CBF012309
:10C5B0000023082D94BF002303F00103002B00F09B
:10C5C000028104F5BF630EF10402524588BF734532
:10C5D00000F2F9802F1FC7F38D0701374FEA870C50
:10C5E0001FFA8CFC714652460346013398B252F84A
:10C5F000046B41F8046B8742F7D8654518D004EB0B
:10C600000C030CF1010292B293F8F4350EF80C30E1
:10C61000954283490CD9A0180CF102039BB290F803
:10C62000F40588549D4203D9E21892F8F425CA54BF
:10C6300094F8F43589F8343094F8F53589F83530C4
:10C6400094F8F63594F8F72503EB022292B2A9F894
:10C65000362094F8F83589F8383094F8F91589F8C7
:10C66000391094F8FA1589F83A1094F8FB1589F8FE
:10C670003B1094F8FC1589F83C10092D40F29F807E
:10C68000022B00F29380674B67490A931B78019352
:10C69000B1F800C0099109F13E034FF0090E0B9368
:10C6A00009F15007964580F085809AF800309A4449
:10C6B0009E449AF80130042B1FFA8EFEF2D19AF8AC
:10C6C00003509AF80240022DECD89AF800300293F9
:10C6D0009AF805309AF8041003939AF806300493F8
:10C6E0009AF80730059302299AF808300693D9D8AA
:10C6F00063B208930B9E1BB203EBC30200201B0125
:10C700000793324403468B424DDA9AF80060B244F4
:10C7100076449AF801B0BBF1050F1FFA86FEF2D1FC
:10C72000019EB346089EB3455CD09DF80860167024
:10C73000042656709DF80C6056719DF81060967135
:10C740009DF81460D6719DF818609470D5701171C1
:10C7500016720194079E4FF0080C1CFB03639AF8B5
:10C760000060FE543B449AF801605E709AF80260E3
:10C770009E709AF80360DE709AF805C09AF804601B
:10C7800006EB0C269E809AF806609E719AF804309B
:10C790009AF805C00130C0B203EB0C2C43B28B42B7
:10C7A0001FFA8CFCB1DBB9F836207BE71E4B0993EE
:10C7B0001C4B0A93099A002313800A9A137040466F
:10C7C0000DB0BDE8F08F681E80B200F2F450174A39
:10C7D000204404F2F35313F8011F02F8011F8342AF
:10C7E000F9D125E79AF804609AF805B006EB0B2614
:10C7F000B445D8DC9DF808601670042656709DF884
:10C800000C6056719DF8106096719DF81460D67199
:10C810009DF818609470D570117116729AE700BF78
:10C8200018B40020060700200807002017B40020D5
:10C830002DE9F843BDF820404C8342F440724FF09C
:10C8400080094FF0060C40F2094E00F2F4571E46E4
:10C85000CA8281F8149081F815C0A1F818E03A4610
:10C8600023468046FFF77EFD18B998F8F535032B6F
:10C8700001D0BDE8F88398F8F435023B9C42A8BF8C
:10C880001C46A4B244B10246BB18023292B29B7855
:10C8900006F8013B9442F7D800233370BDE8F883D3
:10C8A00030B400240525CA824D750C750C834C8369
:10C8B0002246234630BCFFF755BD00BF30B40024EC
:10C8C0000925CA824D750C750C834C83224623467C
:10C8D00030BCFFF747BD00BF70B4453300EB4313D6
:10C8E00000240A83022612064FF001050E754D75CD
:10C8F000CC824C834FF000024CBF1C725C7270BC47
:10C900001346FFF72FBD00BF30B4C4786CB900EBFD
:10C91000820003339B10D0F8D05006D0224601325B
:10C9200051F8040B28609342F9D1002030BC7047C5
:10C930000332921030B4D0F8D05009D0084600230A
:10C9400001332C6840F8044B9A42F9D101EB820183
:10C95000084630BC704700BFF0B5012440220023D8
:10C96000A14284708280C37000F06E81002900F0C3
:10C9700050814278C3604FF4006101610678002A5B
:10C9800000F075814FF460674FF488644FF4806164
:10C9900003F5106E03F53065012AC0F818E045650F
:10C9A0007ED003F5126E03F53265022AC0F81CE052
:10C9B000856575D003F5146E03F53465032AC0F858
:10C9C00020E0C5656CD003F5166E03F53665042AC4
:10C9D000C0F824E0056663D003F5186E03F53865EA
:10C9E000052AC0F828E045665AD003F51A6E03F50B
:10C9F0003A65062AC0F82CE0856651D003F51C6E16
:10CA000003F53C65072AC0F830E0C56648D003F559
:10CA10001E6E03F53E65082AC0F834E005673FD076
:10CA200003F5206E03F54065092AC0F838E0456734
:10CA300036D003F5226E03F542650A2AC0F83CE0C1
:10CA400085672DD003F5246E03F544650B2AC0F8E5
:10CA500040E0C56724D003F5266E03F546650C2A31
:10CA6000C0F844E0C0F880501AD003F5286E03F5F2
:10CA700048650D2AC0F848E0C0F8845010D003F58E
:10CA80002A6E03F54A650E2AC0F84CE0C0F88850BB
:10CA900006D003F52C6503F54C620565C0F88C20C3
:10CAA0004161C0F8CC40002E00F0AF8003F5A062D9
:10CAB000012EC0F8902000F0BF8003F5A462022E82
:10CAC000C0F894204BD003F5A862032EC0F898203C
:10CAD00045D003F5AC62042EC0F89C203FD003F58E
:10CAE000B062052EC0F8A02039D003F5B462062E3E
:10CAF000C0F8A42033D003F5B862072EC0F8A820F0
:10CB00002DD003F5BC62082EC0F8AC2027D003F569
:10CB1000C062092EC0F8B02021D003F5C4620A2EED
:10CB2000C0F8B4201BD003F5C8620B2EC0F8B820A3
:10CB300015D003F5CC620C2EC0F8BC200FD003F545
:10CB4000D0620D2EC0F8C02009D003F5D4620E2E9D
:10CB5000C0F8C42003D003F5D862C0F8C82003F59C
:10CB6000805103F50052022EC0F8D010C0F8D42036
:10CB70004BD903F54052032EC0F8D82045D003F519
:10CB80008042042EC0F8DC203FD003F5A042052EE1
:10CB9000C0F8E02039D003F5C042062EC0F8E420EA
:10CBA00033D003F5E042072EC0F8E8202DD003F57E
:10CBB0000042082EC0F8EC2027D003F51042092EC1
:10CBC000C0F8F02021D003F520420A2EC0F8F4204E
:10CBD0001BD003F530420B2EC0F8F82015D003F51A
:10CBE00040420C2EC0F8FC200FD003F550420D2E11
:10CBF000C0F8002109D003F560420E2EC0F80421D0
:10CC000003D003F57043C0F80831C0F80C71002060
:10CC1000F0BD1B4DC1724FF4A0610C260622C180ED
:10CC2000184F194C1949DFF874E006702B46427012
:10CC3000C560C0F810E0ABE603F58053C0F8D03013
:10CC4000C0F80C710020F0BD4FF4A0740223082638
:10CC500004224FF0A045C172C48003720670427076
:10CC60002B460B4F0B4C0C49DFF834E0E0E7134642
:10CC70004FF460674FF488644FF4806110E700BFA1
:10CC800000000440000E044040040440000404403E
:10CC9000000E005040040050000400500008044002
:10CCA0000008005070B5037A012B82B005464FF0A2
:10CCB000000150D0C3684C4CDA6842F04002DA60A0
:10CCC00003200191FCF7A6FAEB681A69019206E0CD
:10CCD000FCF7A0FAEB68013C1A69019219D0019A9D
:10CCE000002A4FF00300F3DA01993F4A41F00101B5
:10CCF0000191019919611969019103E01969019183
:10CD0000013A02D00199C907F8D40320FCF782FA4E
:10CD1000EB686A7A002A0CBF4FF434114FF4741197
:10CD200099631420FCF77AFAEB68EA78012A06D1B5
:10CD30009E68052262F3440646F020069E60DA688B
:10CD40002A4942F440726FF080440020DA605C614E
:10CD5000996102B070BDC368427A0E46996B66F362
:10CD600010410AB141F480119963DA681E4C6FF3E7
:10CD700086126FF396526FF351426FF3D342DA602B
:10CD8000032000230093FCF745FAEB681A69009230
:10CD900006E0FCF73FFAEB68013C1A69009219D0F3
:10CDA000009A002A4FF00300F3DA00990E4A41F08E
:10CDB00001010091009919611969009103E0196955
:10CDC0000091013A02D00099C807F8D40320FCF77B
:10CDD00021FAEB68EA78012AB1D1052262F3440610
:10CDE00046F020069E60A0E7400D0300040800D036
:10CDF000C268936843F0010393600020704700BF4E
:10CE0000C268936823F0010393600020704700BF5D
:10CE100000B583B000230193019A104B42F0200229
:10CE20000192019A01F01F0122F4F86242EA811294
:10CE30000192C168019A0A610A69019203E00A69D4
:10CE40000192013B02D0019A9206F8D40320FCF72C
:10CE5000E1F9002003B05DF804FB00BF400D0300C2
:10CE6000C26808B5D36801296FF35D736FF39E73D1
:10CE700008D009B943F08043D3603220FCF7CEF9E3
:10CE8000002008BD43F00053F6E700BFC3685869AF
:10CE900000F0010080F00100704700BFC3685869CE
:10CEA00000F00100704700BFC3685A6998691040DC
:10CEB000704700BFF0B5044683B0FCF7B7F9D4F86B
:10CEC0000C31626900261E60237A012B136816BF9D
:10CED000012166F3010361F301031360D4F8CC2050
:10CEE00013686FF382036FF341036FF3C3036FF3B0
:10CEF000451343F4807515600A20FCF78FF9D4F8C8
:10CF0000CC306FF308251D601420FCF787F96269A7
:10CF100013686FF382031360E37A012B374600F046
:10CF2000C180E1680A68674B22F4006200200A6051
:10CF30000090009A42F020020092009A22F4F862D7
:10CF400042F480620092009A0A610A69009203E04A
:10CF50000A690092013B02D0009A9006F8D403209F
:10CF6000FCF758F900230193019AE168554B42F010
:10CF700010020192019A0A610A69019203E00A69AA
:10CF80000192013B02D0019AD206F8D40320FCF7AB
:10CF900041F92378002B69D0D4F890104FF0FF327C
:10CFA00000238A60CB60217801295FD9D4F89410DE
:10CFB0008A60CB602178022958D9D4F898108A6009
:10CFC000CB602178032951D9D4F89C108A60CB60BA
:10CFD000217804294AD9D4F8A0108A60CB6021783E
:10CFE000052943D9D4F8A4108A60CB60217806299A
:10CFF0003CD9D4F8A8108A60CB602178072935D9AC
:10D00000D4F8AC108A60CB60217808292ED9D4F8E6
:10D01000B0108A60CB602378092B27D9D4F8B410DC
:10D0200000238A60CB6021780A291FD9D4F8B81070
:10D030008A60CB6021780B2918D9D4F8BC108A609B
:10D04000CB6021780C2911D9D4F8C0108A60CB604C
:10D0500021780D290AD9D4F8C4108A60CB602178D0
:10D060000E2903D9D4F8C8108A60CB60E26816494B
:10D0700000234FF0FF356FF08040936155615061A0
:10D080009161E3789169002B14BF0023102343F0D2
:10D090000C5343F4001343F008030B430020936147
:10D0A00003B0F0BD8023E022E16863F30F0662F372
:10D0B0000F07C0F26006C0F260074B628E62C1F8D3
:10D0C00000712FE7400D0300040800D038B5054675
:10D0D0000C46FCF7CFF8D5F8CC2013686FF3820329
:10D0E0006FF341036FF3C3036FF34513D90406D401
:10D0F000012C0FD0C820BDE83840FCF78FB8002CB9
:10D10000F8D1194664F30C311160C820BDE83840ED
:10D11000FCF784B843F480511160C820BDE8384062
:10D12000FCF77CB84269136861F301031360704730
:10D1300043695869704700BF38B505460A20D5F8DD
:10D14000CC2013686FF382036FF341036FF3C303C3
:10D150006FF3451343F480741460FCF75FF8D5F85F
:10D16000CC306FF308241C601420FCF757F8012022
:10D1700038BD00BFF0B500EB81034FF0FF32D3F8AC
:10D1800090504B01AA600E46C118C27891F89518CC
:10D19000012A14BF002404240022032913D8DFE845
:10D1A00001F002530247C11801F688018F7A44F456
:10D1B000936444F00104002F43D1097B44F0400400
:10D1C00009B144F02004D0F814E0EC60DEF8184017
:10D1D000C7680121B1402143CEF81810B96918443D
:10D1E00041F00073BB6190F8907890F8916890F8E6
:10D1F000924890F8933890F8951867F39C5266F32C
:10D20000CE2200F6880064F3CF32A3F10203B3FA12
:10D2100083F35B09C08963F3514261F3934260F386
:10D220000A02032908BF42F000522A600020F0BD24
:10D23000C11844F4D36491F8921844F00104002911
:10D24000C1D044F48074BEE7C11844F4087491F866
:10D25000921844F001040029B5D044F4C074B2E738
:10D26000F0B54C01021902F69806B36887B00025A4
:10D270007BB1B2F896785A1E3A44B2FBF7F292B2FA
:10D28000B2F5807F61D93B024FF4807EB360724675
:10D2900002E04FF0010E7246061996F892C8BCF1F2
:10D2A000000F05D0B6F8963803FB02F3C6F8A03895
:10D2B00001F1150700EB471200EB810192F8F8C568
:10D2C000D1F8906063F312056EF3DC456CF35E7584
:10D2D0003561C578D0F814E002F5BE62012D04BFB7
:10D2E000D26872613268DEF8085005F0010585F0F9
:10D2F000010565F35D7242F000426FF39E72326089
:10D30000C278FAB9044404F68804A27AD2B9CBB13F
:10D31000627B032A25D8DFE802F0021B021BC568E6
:10D32000EC6A0394DA1CA4B2C2F38F02944218D2BE
:10D33000AA6942F02002AA61C27800EB4710D0F837
:10D34000FC0592B1002007B0F0BDC2F3090EA3E7BF
:10D35000DEF810400194DA1CA4B2C2F38F029442AA
:10D3600011D300EB4710D0F8FC05D1F8D0409BB2A8
:10D3700003339B10E6D00022013250F8041B2160D9
:10D380009342F9D1DEE7C468A26942F08062A261EB
:10D39000C278D2E700EB810186B0D1F89020136803
:10D3A00043F0404359030AD541690969C1F3074174
:10D3B00009B96FF3DF730020136006B07047C168CE
:10D3C000C96AC1F307410029F3D00020136006B0F9
:10D3D000704700BF00EB81014FF00043D1F890206F
:10D3E000012161F3DC4313611368002043F0004323
:10D3F00060F39E7313607047D0F80C31F0B50022D3
:10D40000044600691A60036862F3CC230360E17A82
:10D41000012983B000F08E80E16800230093009A18
:10D42000544B42F020020092009A22F4F86242F437
:10D4300080620092009A0A610A69009203E00A6918
:10D440000092013B02D0009A9006F8D40320FBF72B
:10D45000E1FE00230193019AE168464B42F010027D
:10D460000192019A0A610A69019203E00A69019234
:10D47000013B02D0019AD206F8D40320FBF7CAFE82
:10D48000256900224FF0FF332A616A61AB61EA61CE
:10D4900063783BB3174604F11401FF2651F8043FAB
:10D4A00018680028ACBF00204FF0904018601F6142
:10D4B0009E60637801329342F0D89BB100221746F8
:10D4C00004F15001FF2651F8043F18680028ACBF52
:10D4D00000204FF0904018601F619E606378013219
:10D4E0009342F0D82B6943F480732B61E378012BCE
:10D4F00004D1214B402262F359432B63E2681F4859
:10D500006FF0804100239361516151619061E37834
:10D510009169002B14BF4FF400634FF4016343F48F
:10D52000701343F4405343F008030B43002093610E
:10D5300003B0F0BD0668E1681346C022802562F39F
:10D540000F034FF4800265F31F4346F0030665F3B3
:10D550000F024FF4A07706604D628A62C1F8043171
:10D5600067F30F036FF31F43C1F80831C1F80C31A3
:10D5700053E700BF400D030003010100040800D081
:10D5800010B4C2680C4C00236FF08041936151616C
:10D5900051619461C07891695DF8044B984208BF6D
:10D5A000102343F4701343F4605343F008030B4318
:10D5B00000209361704700BF040800D003699B6896
:10D5C000C3F34103022B07D0032B03D0012B01D05F
:10D5D000032070470220704701207047036981696A
:10D5E0009A680868C2F34102022A06BF032262F366
:10D5F0000A006FF30A0008605A6842F480725A60A9
:10D600000020704770B44B78012B4FF000041FD0FE
:10D610000D7800EB85020123AB40526D63F31F448C
:10D6200013681D040DD48E68CD78C98866F30A038B
:10D6300065F3934361F3995343F0805343F40043FC
:10D6400013600269D36923430020D36170BC704723
:10D650000A7800EB8205934063F30F04AA69DFE7C1
:10D6600030B44B780022012B144612D00B7800EB1B
:10D670008305012199406D6D61F31F4401696FF3CA
:10D68000CF322A60CB6923EA04030020CB6130BC8F
:10D690007047097800EB81058B4063F30F04AD6997
:10D6A000ECE700BFF0B54B780A78012B2AD000EBED
:10D6B00082024B69566D8C6832683569F3B1234438
:10D6C000013BB3FBF4F3C3F3090304FB03F4C4F31A
:10D6D00012049BB263F3DC4564F312053561C37831
:10D6E000012B5CD0CB78012B54D00B7800EB83005E
:10D6F00042F00442436D1A600020F0BD0123C4F3E0
:10D700001204E7E700EB82024C69966932683569DA
:10D71000002C4BD08F6891F803E064F31205E319F5
:10D72000013BBEF1010FB3FBF7F363F3DC4508BF28
:10D730006EF35E753561C378012B46D0CB78012B33
:10D740003CD04CB106690F78756B0123BB402B436D
:10D750007363CB78012B31D00B7800EB830342F05D
:10D7600004429B691A60CB78012BC5D1C278CD6881
:10D770000978002AC0D1A3B200EB810003339B10CB
:10D78000D0F8D000B8D0013255F8041B01609342A4
:10D79000F9D1B1E74B7973B142F00052A5E70B78AC
:10D7A0000C6900EB83035B6D5C619BE764F312051E
:10D7B00063F3DC45BEE742F0805296E703699B685D
:10D7C000DB0509D442F00052C6E70B780D6900EB87
:10D7D00083039B695D61BCE742F08052BCE700BFF8
:10D7E000F0B44A78012A82B02DD00B784A6900EB58
:10D7F00083035C6D23682569009502B38A684A61DA
:10D8000002F07F029DF802609DF80050012762F34C
:10D81000060567F3C4068DF802608DF80050009A83
:10D820002261C278BA4241D00A7800EB820043F00C
:10D830000443426D1360002002B0F0BC70478A6858
:10D8400002F07F02DEE784694D692368266900964D
:10D85000002D32D08A689DF80060954284BF02F0A6
:10D860007F054A619DF8022098BF05F07F050127DA
:10D8700065F3060667F3C4028DF800608DF8022098
:10D88000009A2261C278012A24D043F00443236025
:10D89000C378002BCFD14B69002BCCD0006909781D
:10D8A000426B01238B4013434363C4E70A780C693E
:10D8B00000EB8202526D5461B6E79DF800709DF84E
:10D8C000026065F3060762F3C4068DF800708DF8F8
:10D8D0000260D5E70A780D6900EB82029269556112
:10D8E000D3E700BF4B78012B0B7800EB830006D009
:10D8F000426D136843F4001313600020704782697F
:10D900001368002BF6DA43F0804343F400131360EE
:10D91000002070474B78CA78012B0B7800EB83000E
:10D92000A2F102020CBF8069406D0368012A6FF307
:10D93000555398BF43F0805303600020704700BFE9
:10D9400002699369D0691840000C704700EB8101AF
:10D9500002694B6D9B68506918407047036998696C
:10D96000DB69184080B2704710B4012383B04FF0D8
:10D97000000263F3C402C024002318210093436D06
:10D980008DF802208DF803408DF80010009A1A617E
:10D99000C278012A06D100F2CC5058614FF08022A3
:10D9A00019681A6003B05DF8044B704738B5044637
:10D9B000FEF7D2FF62780121002384F8121184F867
:10D9C0001431002A00F00A824020012A84F81D1137
:10D9D00084F81C31A4F8223184F81F31C4F82831AE
:10D9E000C4F83031C4F8240100F00A82022A84F815
:10D9F000451184F84411A4F84A1184F84731C4F859
:10DA00004C01C4F85031C4F8583100F0E3800225CD
:10DA1000032A84F86D1184F86F31C4F87401C4F8D6
:10DA20007831C4F8803184F86C51A4F8725100F058
:10DA3000D1800325042A84F8951184F89731C4F81D
:10DA40009C01C4F8A031C4F8A83184F89451A4F81A
:10DA50009A5100F0BF800425052A84F8BD1184F88E
:10DA6000BF31C4F8C401C4F8C831C4F8D03184F857
:10DA7000BC51A4F8C25100F0AD800525062A84F8F7
:10DA8000E51184F8E731C4F8EC01C4F8F031C4F8CA
:10DA9000F83184F8E451A4F8EA5100F09B8006259F
:10DAA000072A84F80D1284F80F32C4F81402C4F85F
:10DAB0001832C4F8203284F80C52A4F8125200F044
:10DAC00089800725082A84F8351284F83732C4F88B
:10DAD0003C02C4F84032C4F8483284F83452A4F806
:10DAE0003A5277D00825092A84F85D1284F85F320B
:10DAF000C4F86402C4F86832C4F8703284F85C5226
:10DB0000A4F8625266D000230925012040210A2A88
:10DB100084F8850284F88452A4F88A5284F8873203
:10DB2000C4F89032C4F89832C4F88C1252D00A2546
:10DB30000B2A84F8AD0284F8AF32C4F8B412C4F8EA
:10DB4000B832C4F8C03284F8AC52A4F8B25241D012
:10DB50000B250C2A84F8D50284F8D732C4F8DC12DD
:10DB6000C4F8E032C4F8E83284F8D452A4F8DA52A7
:10DB700030D00C250D2A84F8FD0284F8FF32C4F859
:10DB80000413C4F80833C4F8103384F8FC52A4F822
:10DB900002531FD00D250E2A84F8250384F827335D
:10DBA000C4F82C13C4F83033C4F8383384F8245341
:10DBB000A4F82A530ED00E2584F84D0384F84F3371
:10DBC000C4F85413C4F85833C4F8603384F84C5381
:10DBD000A4F85253002340210120022A84F875330F
:10DBE00084F87433A4F87A3384F87733C4F8803334
:10DBF000C4F8883384F89D3384F89F33C4F8A8337D
:10DC0000C4F8B033C4F87C13C4F8A41384F89C039C
:10DC1000A4F8A20340F2E2800220032A84F8C5336C
:10DC200084F8C733C4F8CC13C4F8D033C4F8D8335D
:10DC300084F8C403A4F8CA0300F0D0800320042AA7
:10DC400084F8ED3384F8EF33C4F8F413C4F8F833F0
:10DC5000C4F8003484F8EC03A4F8F20300F0BE80AA
:10DC60000420052A84F8153484F81734C4F81C14E9
:10DC7000C4F82034C4F8283484F81404A4F81A042E
:10DC800000F0AC800520062A84F83D3484F83F3447
:10DC9000C4F84414C4F84834C4F8503484F83C043C
:10DCA000A4F8420400F09A800620072A84F865341C
:10DCB00084F86734C4F86C14C4F87034C4F8783449
:10DCC00084F86404A4F86A0400F088800720082A15
:10DCD00084F88D3484F88F34C4F89414C4F89834DC
:10DCE000C4F8A03484F88C04A4F8920476D00820F8
:10DCF000092A84F8B53484F8B734C4F8BC14C4F8DD
:10DD0000C034C4F8C83484F8B404A4F8BA0465D0A4
:10DD100009200A2A84F8DD3484F8DF34C4F8E414D6
:10DD2000C4F8E834C4F8F03484F8DC04A4F8E2045D
:10DD300054D00A200B2A84F8053584F80735C4F836
:10DD40000C15C4F81035C4F8183584F80405A4F887
:10DD50000A0543D000230B2040210C2A84F82D35DE
:10DD600084F82F35C4F83835C4F8403584F82C05CC
:10DD7000A4F83205C4F8341530D00C200D2A84F8EC
:10DD8000553584F85735C4F85C15C4F86035C4F8C7
:10DD9000683584F85405A4F85A051FD00D200E2AC2
:10DDA00084F87D3584F87F35C4F88415C4F8883547
:10DDB000C4F8903584F87C05A4F882050ED00E22B4
:10DDC00084F8A53584F8A735C4F8AC15C4F8B03587
:10DDD000C4F8B83584F8A425A4F8AA252046FFF78E
:10DDE0000FF82046FEF75EFF20460021FFF738F8C7
:10DDF0002046FFF701FB2046BDE83840FEF7F8BF9C
:10DE000084F8753384F87433A4F87A3384F877335C
:10DE1000C4F87C03C4F88033C4F88833DEE700BF5D
:10DE2000F8B50C0617D401EB8104E40006190027AD
:10DE300006F55D7486F8741386F87573C6F87C234E
:10DE400086F87733022B04BF002323712146FFF7A6
:10DE5000D9FB0020F8BD01F07F0101EB8104E40053
:10DE60000619012706F58E7486F81C1186F81D71B7
:10DE7000C6F8242186F81F31A6F82211E2E700BF78
:10DE8000CAB208B513060DD401EB810300EBC3033E
:10DE900003F55D73D20919705A701946FFF7E0FB5C
:10DEA000002008BD01F07F0101EB810300EBC303FB
:10DEB00003F58E73EEE700BFF8B501F07F0505EBC3
:10DEC0008504E4000119002781F87453C1F8802308
:10DED000C1F88833C1F88C7381F87573C37801F584
:10DEE000607E012B08BFEDB201F55D7108BFCEF871
:10DEF00004201DB1FFF7D6FB0020F8BDFFF770FC32
:10DF00000020F8BD2DE9F84301F07F0505EB8504FD
:10DF1000E40006194FF001094FF0000806F58E7174
:10DF200086F81C5186F81D91C6F82821C6F82C21C8
:10DF3000C6F83481C6F8303125B1FFF7B3FB0020B5
:10DF4000BDE8F883FFF74CFC0020BDE8F88300BF74
:10DF5000CAB2130610B50FD401EB810300EBC30363
:10DF600003F55D73D209012419705A709C7019462B
:10DF7000FFF7B8FC002010BD01F07F0101EB810329
:10DF800000EBC30303F58E73ECE700BFCAB21306C0
:10DF900010B50FD401EB810300EBC30303F55D73F0
:10DFA000D209002419705A709C701946FFF7B2FC10
:10DFB000204610BD01F07F0101EB810300EBC3039C
:10DFC00003F58E73ECE700BF02690020136861F36C
:10DFD0000A10034313607047704700BF704700BFCB
:10DFE0002DE9F04F85B00546FEF750FF18B9002027
:10DFF00005B0BDE8F08F2846FEF756FF00900028D8
:10E00000F5D0C0F3074707F0080303F0FF00002B2B
:10E0100040F090807C0730D49DF80040A10702D5E5
:10E02000EB6802225A61009B002BC0F2E881C3F327
:10E030000726320700F1B481270700F1A781E10626
:10E0400000F17E81F20600F1E380B30600F1C480A6
:10E05000009BC3F3074818F0100F40F0B28018F08F
:10E06000200FC5D0694B1B6828461B6A9847EB6890
:10E070004FF400125A610120BAE72846FFF76EFC00
:10E080000746002854D005F1180A2E464FF0000824
:10E0900022E0180703D5DAF8002008239360D90698
:10E0A00003D5DAF80020102393605A0603D5DAF876
:10E0B000002040239360980703D5DAF8002002235C
:10E0C0009360DB0940F0DD817F0808F101080AF167
:10E0D000040A06F128062BD0F907F5D529695FFA5D
:10E0E00088F408694B6B05EB8402E3409269DB011D
:10E0F0009268DBB203431340DBB2DA07C9D5434A67
